:020000040800F2
:1000000000000120816A0008EF330008F133000886
:10001000F3330008F5330008F73300080000000050
:10002000000000000000000000000000F93300089C
:10003000FB33000800000000FD330008FF33000818
:10004000D16A0008D16A000801340008D16A0008AA
:10005000D16A0008D16A00080D3400081D34000878
:10006000D16A00082D340008D16A00083534000830
:10007000413400084D340008D16A0008D16A0008F4
:10008000593400085D340008D16A0008D16A0008BC
:1000900000000000D16A000869340008D16A000835
:1000A000D16A0008D16A0008D16A0008D16A000844
:1000B000D16A0008D16A0008D16A0008D16A000834
:1000C000D16A0008D16A00086D340008D16A0008BE
:1000D000D16A000879340008D16A0008D16A0008A2
:1000E000D16A0008D16A000885340008D16A000886
:1000F000D16A00080000000000000000D16A00087A
:10010000D16A0008D16A000891340008D16A000859
:10011000D16A0008D16A0008D16A0008D16A0008D3
:10012000D16A0008D16A0008D16A0008D16A0008C3
:08013000D16A0008D16A000841
:1001400010B5054C237833B9044B13B10448AFF311
:1001500000800123237010BDA005002000000000D6
:10016000E41F030808B5034B1BB103490348AFF371
:10017000008008BD00000000A4050020E41F030863
:1001800014214160704714207047406A7047000096
:1001900081010008870100088B010008A101000807
:1001A00010B5044604F1100000F05CFCC4F8F8003F
:1001B0000148C4F87C0110BD90010008F8B5E6B014
:1001C00004460D4616461F460A4906A800F0CAFE18
:1001D00070996F9A05910492009733466E996D9AC3
:1001E000039102922A466C990191214600F060F831
:1001F00067B0F0BD9C010008F8B5E6B004460D46B6
:1002000016461F46094906A800F0ACFE6F996E9A83
:100210000491039200976D996C9A02910192334672
:100220002A46214600F087F867B0F0BD9C0100081F
:1002300038B500281CBF01680029184A23D1184B83
:100240001C684FF6F0710C404CF24025AC421FBFC9
:100250001B6819404CF27024A14212D1114D29683B
:1002600079B911490B68C3F30B03B3F58A6F1FBF4C
:100270000968C1F30B0140F28343994204BF012195
:10028000117028B905E0094B994204BF0121117092
:100290004068BDE8324002F073BC00BFBC050020DE
:1002A00000ED00E0002004E00010005C0000374892
:1002B0002DE9F04104460D46216816464A681F465E
:1002C00090478046B8F5403F2ED122680A9993683E
:1002D000204698478046B8F5403F25D12368089AC4
:1002E0000799D3F80CC02046E0478046B8F5403F58
:1002F0001AD12368069A39461F692046B8478046B6
:10030000B8F5403F10D1236829465D693246204642
:10031000A8478046B8F5403F06D123680B9A099953
:100320009D692046A847804621680A682046904774
:100330004046BDE8F0812DE9F04104460D462168B4
:1003400016464A681F4690478046B8F5403F2ED172
:1003500022680A999368204698478046B8F5403F3E
:1003600025D12368089A0799D3F80CC02046E047A6
:100370008046B8F5403F1AD12368069A39461F696E
:100380002046B8478046B8F5403F10D1236829463B
:100390005D6932462046A8478046B8F5403F06D101
:1003A00023680999DD6900222046A8478046216814
:1003B0000A68204690474046BDE8F0814FF440303F
:1003C00070470000F0B50C4685B0114600281A466B
:1003D0001CBF0568002D0B4B11D082B104B971B957
:1003E0000D9860B10F9E0E9F0A9B02900496039792
:1003F0000B980C9E009001962046A847034618468D
:1004000005B0F0BD020003002DE9F04F0646D0B064
:100410000868F56DD6F860E0726EB76EF36E00BADC
:1004200000906C46486800BA60600DF1400888682A
:1004300000BAA060C86800BAE060086900BA20612C
:10044000486900BA6061886900BAA061C86900BAE9
:10045000E061086A00BA2062486A00BA6062886A8D
:1004600000BAA062C86A00BAE062086B00BA2063F2
:10047000486B00BA6063886B00BAA063C86B00BAAF
:10048000E063402058F80C1C58F820CC58F838ACE1
:100490008CEA010158F840CC8AEA01018CEA010992
:1004A0004FEAF979401E48F8049BEBD187EA020035
:1004B00000EA0E00784010EBF5610098DFF824C4E4
:1004C00041186144C81882EABE032B404FEAF0612C
:1004D00053405918636859186144CF194FEAB5035E
:1004E00083EABE01014081EABE0111EBF765A16814
:1004F0004D196544A91883EAB0023A404FEAF16504
:100500005A405519E26855194FEAB70282EAB00716
:1005100065440F4005EBBE0E97EAB00717EBFE658A
:1005200027697D194FEAB10782EA0701654401EAAC
:100530000E01EB18514011EBF36561694D194FEA5B
:10054000BE0187EA010E65440EEA030E15EBB0000A
:100550008EEA070E0EEBF065D4F818E0754465449A
:10056000AA1881EAB30505404FEAF26E4D40AE4449
:10057000E569AE44E64477444FEAB00080EAB30E42
:100580000EEA020E8EEAB30E0EEBF765D4F820E009
:1005900075446544691880EAB2053D404FEAF16E42
:1005A0004540AE44656AAE44E6440EEBB3034FEA01
:1005B000B70787EAB20E0EEA010E8EEAB20E0EEB14
:1005C000F365D4F828E075446544281887EAB10536
:1005D0001D404FEAF06E7D40AE44E56AAE44E6440D
:1005E0000EEBB2024FEAB30383EAB10E0EEA000E3D
:1005F0008EEAB10E0EEBF265D4F830E07544654436
:10060000EF1983EAB00515404FEAF76E5D40AE443E
:10061000656BAE44E6440EEBB1014FEAB20282EAEA
:10062000B00E0EEA070E8EEAB00E0EEBF165D4F8AE
:1006300038E075446544EB1882EAB7050D404FEA8F
:10064000F36E5540AE44E56BAE44E6440EEBB000AD
:100650004FEAB10181EAB70E0EEA030E8EEAB70E39
:100660000EEBF065D4F840E07544654481EAB30EC2
:10067000AA180EEA000E4FEAF2658EEA010E7544E2
:10068000DDF844E04FEAB000754480EAB30E6544FB
:100690000EEA020E15EBB7078EEAB30E0EEBF76506
:1006A000DDF848E04FEAB202754480EA020E654484
:1006B0000EEA070E69188EEA000E0EEBF165DDF802
:1006C0004CE07544654405EBB3034FEAB70E1427BD
:1006D0000DF1500CDFF810528EEA010B82EA0B0B81
:1006E0000BEBF36A5CF804BBDA44AA44504483EA97
:1006F000B10B4FEAF06A8EEA0B0BDA445CF804BBEC
:10070000DA44AA44524480EAB30B4FEAF26A8BEA15
:10071000B10BDA445CF804BBDA444FEAB000AA44F7
:1007200080EA020BD6448BEAB30B0BEBFE6A5CF853
:1007300004BBDA444FEAB202AA4482EA0E0B0AEB87
:10074000B10180EA0B0B0BEBF16A5CF804BBDA44F5
:100750007F1DAA44282F0AEBB3034FEABE0EBBD37A
:100760003C2F61D3502F4DD204EB870CC7F15407B7
:100770005E4CA7FB04A504465D4FA8088EEA010A5B
:1007800082EA0A0A5CF804BB0AEBF3655D447D1952
:100790002C1983EAB10A4FEAF4658EEA0A0A554435
:1007A0005CF804AB5CF804BB55447D19AA1884EAD4
:1007B000B30A4FEAF2658AEAB10A55445D444FEA4A
:1007C000B4047D1984EA020AAE448AEAB30A0AEB49
:1007D000FE655CF804AB55444FEAB2027D1982EA2B
:1007E0000E0A15EBB10184EA0A0A5CF804BB0AEBB5
:1007F000F1655D447D1915EBB303401E4FEABE0E53
:10080000BCD12046F46D1B19F365336EC9183166EF
:10081000716E71447166B36ED218B266F16E401893
:10082000F06650B0BDE8F08F4EEA010B0EEA010A07
:100830000BEA020B4BEA0A0A0AEBF36554F827A00D
:10084000DFF8B0C0554443EAB10B654403EAB10A8E
:100850000BEA0E0B28184BEA0A0A7F1C0AEBF0651C
:1008600054F827A0554440EAB30B654400EAB30AA4
:100870000BEAB10BAA184BEA0A0A7F1C0AEBF265D5
:1008800054F827A055444FEAB00040EA020B6544F3
:1008900000EA020A0BEAB30BAE444BEA0A0A7F1CD9
:1008A0000AEBFE6554F827A055444FEAB20242EA2B
:1008B0000E0B654402EA0E0A0BEA000B15EBB101C0
:1008C0004BEA0A0A7F1C0AEBF16554F827A055444D
:1008D0007F1C65443C2F05EBB3034FEABE0EA3D348
:1008E00040E700BF9979825AA1EBD96ECDCCCCCC30
:1008F000D6C162CADCBC1B8F00B581B00168074A53
:10090000914200D110B9064801B000BD7C212EF003
:1009100018F94FF4003001B000BD00BF040A000810
:10092000030002002DE9F0410B4A92E8F85188B02B
:10093000694681E8F8510268084B9A4200D118B91B
:10094000074808B0BDE8F0811422083000F04FFBE2
:1009500008B0BDE8F08100BFE4090008040A0008FF
:1009600003000200152904D20268044B9A4200D108
:1009700008B903487047083000F048BB040A000873
:100980000300020010B481B013460268074CA24273
:1009900000D118B901B010BC0548704701B000F192
:1009A000240210BC083000F035BB00BF040A000868
:1009B0000300020010B481B013460268074CA24243
:1009C00000D118B901B010BC054870470A4601B003
:1009D00000F1240110BC083000F070BB040A0008CC
:1009E000030002000123456789ABCDEFFEDCBA9816
:1009F00076543210F0E1D2C3000000000000000085
:100A000000000000F9080008250900086509000831
:100A100085090008B509000809040008810F0008CD
:100A2000CD0F0008890F0008F0B5A3B004460B48AD
:100A300002900D4616461F46094B0822402104A885
:100A400000F0D1FA28980190009733462A462146B3
:100A500002A800F01BF823B0F0BD00BF040A000894
:100A6000180A000810B5040008BF002408D0054883
:100A7000054B20600822402104F1080000F0B3FA81
:100A8000204610BD040A0008180A00082DE9F041AC
:100A900004460E46216817464A681D469047804620
:100AA000B8F5003F19D12268069993682046984707
:100AB0008046B8F5003F10D123683146DE683A46DB
:100AC0002046B0478046B8F5003F06D12368079A14
:100AD00029461D692046A847804621680A682046A5
:100AE00090474046BDE8F08110B500F033FA4FF46E
:100AF000403400280EBF034C4FF4C0712EF021F893
:100B0000204610BD0200030010B5044600F022FA92
:100B100008B9054810BD0021A160D0F87C211168FA
:100B200088474FF4403010BD0200030070B5044602
:100B30000D4600F00FFA064E40B1D0F87C01416836
:100B40008847A84224BF65604FF44036304670BDE8
:100B5000020003002DE9FF4715000C4600D02CB120
:100B6000064600F0F7F95FEA000801D16448C3E0E7
:100B7000D8F8F80001684A689047B0F5003F17D1EF
:100B8000D8F87C118A68404690478146B9F1810FB8
:100B900080F09E80A94508F1FC0A17D2D8F8F80029
:100BA0000368D3F80CC02A462146E047B0F5003F61
:100BB00040F08E80D8F8F8000368D3F810C06A4679
:100BC0005146E047B0F5003F76D10AE0002004E04E
:100BD000215C0AF800100098401C00900098A84280
:100BE000F6D34FF0000C4749474A484B01AC0098F8
:100BF000844558D2D3E9007001ADC5E90070107882
:100C000000281ABF042086464FF0000E085854F8FA
:100C10000E5028443E4D05600127D0F800E0876063
:100C2000019D4F681AF80C007D408EEA050585F09D
:100C3000040E65680F687D4085F0FC05754485F0FD
:100C4000A30568400AF80C000CF1010CCFE7D3E9CA
:100C5000004501A8C0E9004510782E4D002814BFBA
:100C60004FF0040E4FF0000E01A8744651F80EE04C
:100C70000459A6440127CEF80050DEF80040CEF813
:100C800008704D68019F40687D406C400D68684069
:100C900084F0040480F0FC00041984F057040AF87E
:100CA0000C400CF1010CCC45D1D3D8F8F800016808
:100CB0004A689047B0F5003F0AD1D8F8F8000368B9
:100CC000D3F80C804A465146C047B0F5003F01D0EA
:100CD000114811E0002006E05AF8201081F06A3136
:100CE0004AF82010401CB0EB990FF5D3B06840F0E3
:100CF0000100B0604FF4403004B0BDE8F08700BFA1
:100D0000020003002C610308BC0500202C0F000822
:100D1000ADBE4ED70DBE75A10100030038B50C461F
:100D2000017A1546CA0702D500F014F908B9084837
:100D300032BDD0F8F80003682146DC682A46A04797
:100D4000B0F5003F01D0034832BD4FF4403032BD12
:100D500002000300010003002DE9F84191B00546AF
:100D60000E461746402101A82DF0EBFE297AC80750
:100D700004D5284600F0EEF8040002D1DFF8A48084
:100D80004BE0D4F8F800DFF8A0800368D3F810C077
:100D90006A4601A9E047B0F5003F3ED1D4F8F8001B
:100DA00001684A689047B0F5003F36D1D4F87C110D
:100DB0008A6820469047D4F8F830024618461B68E7
:100DC000D3F80CC004F1FC01E047B0F5003F24D19A
:100DD000D4F87C0141688847D4F8F83002461846B8
:100DE0001B68D3F80CC001A9E047B0F5003F14D14F
:100DF000D4F8F8000268696893689847B0F5003F36
:100E00000BD1D4F8F80003681C693A463146A04774
:100E1000B0F5003F08BF4FF44038404612B0BDE87F
:100E2000F08100BF02000300010003002DE9F8413A
:100E3000A5B0074688461646402115A82DF081FE2C
:100E400000220492402105A82DF07BFE387AC107CC
:100E50005ED5384600F07EF8050059D0D5F8F80088
:100E60002D4C0368D3F810C06A4605A9E047B0F5D9
:100E7000003F3CD1D5F8F80001684A689047B0F5CA
:100E8000003F34D1D5F87C118A6828469047D5F8C0
:100E9000F830024618461B68D3F80CC005F1FC0177
:100EA000E047B0F5003F22D1D5F87C014168884782
:100EB000D5F8F830024618461B68D3F80CC005A9CF
:100EC000E047B0F5003F12D1D5F8F8000268796824
:100ED00093689847B0F5003F09D1D5F8F80003684A
:100EE0001D6904AA15A9A847B0F5003F01D0204606
:100EF0000FE00A4B0A490B4A0396029101924046C1
:100F00001C68049B009415AA796800F0E5F900E0DC
:100F1000054826B0BDE8F0810100030034610308F4
:100F2000936E030026C703000200030004B0010112
:100F300000170145E90A0008090B00082D0B0008FD
:100F4000BD030008550B00081D0D0008590D0008D1
:100F50002D0E00080168024A914218BF0020704718
:100F6000340F000810B5040008BF002404D0034863
:100F70002060204609688847204610BD340F0008CD
:100F800020225C302DF0D9BDF0B58468A308002282
:100F900004F0030407E000F15C0555F8226035BA5F
:100FA00041F82250521C9A42F5D300220BE000F186
:100FB0005C0502EB830755F82360D500C5F11805E1
:100FC000EE40CE55521CA242F1D3F0BD30B5C468FC
:100FD00003690022E31AD5188C5C0544521C082AC8
:100FE0002C77F8D330BD0360C1600261704738B51B
:100FF000044615460022626023685A689047002024
:101000006061A061A5604FF4003032BD81604FF493
:10101000003070472DE9F84304462079D4F80C805D
:10102000450748BF244845D466691D46A8F101001C
:1010300000EAD60306EBC506B6EBC50F666102D221
:10104000A669761CA6611746A66906EB5576A661C9
:101050000E46E918884225D2A8EB03094A463146D4
:10106000F8182DF06AFD2268136839460FE04246F1
:1010700038462DF062FD23681A68394620469047AD
:1010800007E0311811F00300F1D1226813682046FF
:101090009847484600EB0809A9F10101A942F0D39D
:1010A000002300E000202A1A3118F8182DF045FD21
:1010B0004FF40030BDE8F283040002002DE9FC4F3C
:1010C000024685B0D0681369DFF86CC1DFF86C8127
:1010D000A0EB030A506840F004005060002703A80A
:1010E00002900DF10C0ED8E9003403A8544DC0E96C
:1010F00000342878534D00280CBF00230423994660
:101100005CF803305EF80940234401261D601C682A
:101110009E60DCF80430039DDCF80090DEF804608B
:101120005D406540484C654089EA0606474C66408C
:101130007519474C6540D8E9006B03AC0028C4E939
:10114000006B0EBF002404200424029E5CF8000003
:10115000345920183F4C04600126046886600398C7
:10116000029E43406340384C7068634089EA000047
:10117000364C6040034438484340280018BF0120E3
:101180005B1E9B41042F2CBFC0B2D80F02F1140389
:1011900053F8200007F00303C3F10303DB00D8403A
:1011A0000DF807007F1C082F9DD315460C466A6971
:1011B000AB69E868D20842EA4372401E00EA0207BF
:1011C000002302409B420AD8524508D28020E055B5
:1011D0007F1C574516D2AAEB0701E01910E08020CA
:1011E000E05500E0E355E8687F1C8742FAD32A689F
:1011F000136828469847BAF1000F03D0514620469D
:101200002DF09FFC2A68069E059F93686946284634
:1012100098472A68D2F8009021462846C8472B688C
:10122000DA683946284690470EB1A86830604FF416
:10123000003007B0BDE8F08F2C6103085C12000895
:10124000BC0500205FC5109304850012FC68017A7C
:10125000C0F524FF24AF33D426AF698B04B001015D
:1012600000170145F8B501240094002300240DE087
:10127000009D065D0F5D7E40F643761CF60F86F0FE
:10128000010635400095641C009DEB189442EFD395
:101290001846F2BDF8B5002301240094002A11E09D
:1012A000009C85188F1815F8016C17F8015C6E40CA
:1012B000F643761CF60F86F0010634400094009C3D
:1012C000E318521EECD11846F2BD0000651200086A
:1012D00095120008010000002DE9F84F1D46DDF8C9
:1012E00028900B9F0D9C4FF0FF3300930E469246C3
:1012F000D9F800B0804632465146D847834664B399
:10130000D9F8043032465146404698476FEA0B02FE
:10131000521C42EA0B0200996FEAD2735B1C19401F
:10132000C2430091521C024300996FEAD2735B1CC6
:101330001940009186F05531484087EA000181F05C
:101340005531216080F05531C943491C0843009A4A
:101350006FEAD070401C82430092D9F8080001283F
:1013600009D17540E943491C0D4300986FEAD572D5
:10137000521C90430AE0F11C85EA9102D243521CB0
:10138000154300986FEAD5735B1C984386F0AA3624
:10139000009086EA0B0686F0AA33F243DB430C98F2
:1013A000C2F3C0725B1C42EAD3720099D243521C52
:1013B00091430091774000998843009987F0AA37BC
:1013C0000F403843BDE8F28F00000000000000002D
:1013D00001F0FF01102A2BDB10F0070F08D010F8E6
:1013E000013B013A8B422DD010F0070F42B3F6D1EA
:1013F000F0B441EA012141EA014122F007047FF003
:1014000000070023F0E80256083C85EA010586EA59
:10141000010685FA47F5A3FA87F586FA47F6A5FA95
:1014200087F68EB9EED1F0BC01F0FF0102F00702A1
:1014300032B110F8013B013A83EA010313B1F8D14C
:101440000020704701387047002D06BF354603382D
:10145000073815F0010F07D1013015F4807F02BF66
:10146000013015F4C03F0130F0BC0138704700BFB7
:10147000034613F8012B002AFBD1181A01387047D4
:1014800081F0004102E000BF83F0004330B54FEA35
:1014900041044FEA430594EA050F08BF90EA020FA2
:1014A0001FBF54EA000C55EA020C7FEA645C7FEA35
:1014B000655C00F0E2804FEA5454D4EB5555B8BF58
:1014C0006D420CDD2C4480EA020281EA030382EAC9
:1014D000000083EA010180EA020281EA0303362D5B
:1014E00088BF30BD11F0004F4FEA01314FF4801C2E
:1014F0004CEA113102D0404261EB410113F0004F40
:101500004FEA03334CEA133302D0524263EB4303F6
:1015100094EA050F00F0A780A4F10104D5F1200E94
:101520000DDB02FA0EFC22FA05F2801841F10001EF
:1015300003FA0EF2801843FA05F359410EE0A5F1C3
:1015400020050EF1200E012A03FA0EFC28BF4CF0F4
:10155000020C43FA05F3C01851EBE37101F00045AA
:1015600007D54FF0000EDCF1000C7EEB00006EEBB7
:101570000101B1F5801F1BD3B1F5001F0CD3490841
:101580005FEA30004FEA3C0C04F101044FEA445298
:1015900012F5800F80F09A80BCF1004F08BF5FEA1F
:1015A000500C50F1000041EB045141EA050130BDFF
:1015B0005FEA4C0C404141EB0101013C28BFB1F511
:1015C000801FE9D291F0000F04BF01460020B1FA5C
:1015D00081F308BF2033A3F10B03B3F120020CDA2F
:1015E0000C3208DD02F1140CC2F10C0201FA0CF00D
:1015F00021FA02F10CE002F11402D8BFC2F1200C72
:1016000001FA02F120FA0CFCDCBF41EA0C01904027
:10161000E41AA2BF01EB0451294330BD6FEA040470
:101620001F3C1CDA0C340EDC04F11404C4F120025B
:1016300020FA04F001FA02F340EA030021FA04F36D
:1016400045EA030130BDC4F10C04C4F1200220FAC4
:1016500002F001FA04F340EA0300294630BD21FA02
:1016600004F0294630BD94F0000F83F4801306BFC8
:1016700081F480110134013D4EE77FEA645C18BFBC
:101680007FEA655C29D094EA050F08BF90EA020F53
:1016900005D054EA000C04BF1946104630BD91EA4B
:1016A000030F1EBF0021002030BD5FEA545C05D14E
:1016B0004000494128BF41F0004130BD14F580048D
:1016C0003CBF01F5801130BD01F0004545F0FE4101
:1016D00041F470014FF0000030BD7FEA645C1ABF36
:1016E000194610467FEA655C1CBF0B46024650EA6D
:1016F000013406BF52EA033591EA030F41F4002199
:1017000030BD00BF90F0000F04BF0021704730B51E
:101710004FF4806404F132044FF000054FF00001F3
:1017200050E700BF90F0000F04BF0021704730B5B4
:101730004FF4806404F1320410F0004548BF404289
:101740004FF000013EE700BF42004FEAE2014FEADE
:1017500031014FEA02701FBF12F07F4393F07F4FB9
:1017600081F06051704732F07F4208BF704793F0BC
:101770007F4F04BF41F40021704730B54FF46074CF
:1017800001F0004521F000411CE700BF50EA0102D2
:1017900008BF704730B54FF000050AE050EA01027B
:1017A00008BF704730B511F0004502D5404261EBEB
:1017B00041014FF4806404F132045FEA915C3FF42C
:1017C000D8AE4FF003025FEADC0C18BF03325FEAC9
:1017D000DC0C18BF033202EBDC02C2F1200300FA7A
:1017E00003FC20FA02F001FA03FE40EA0E0021FA9F
:1017F00002F11444BDE600BF70B54FF0FF0C4CF48D
:10180000E06C1CEA11541DBF1CEA135594EA0C0F3E
:1018100095EA0C0F00F0DEF82C4481EA030621EA79
:101820004C5123EA4C5350EA013518BF52EA0335B4
:1018300041F4801143F4801338D0A0FB02CE4FF066
:101840000005E1FB02E506F00042E0FB03E54FF096
:101850000006E1FB03569CF0000F18BF4EF0010E8E
:10186000A4F1FF04B6F5007F64F5407404D25FEA8A
:101870004E0E6D4146EB060642EAC62141EA55513D
:101880004FEAC52040EA5E504FEACE2EB4F1FD0C7F
:1018900088BFBCF5E06F1ED8BEF1004F08BF5FEAFD
:1018A000500E50F1000041EB045170BD06F00046AF
:1018B00046EA010140EA020081EA0301B4EB5C045C
:1018C000C2BFD4EB0C0541EA045170BD41F4801154
:1018D0004FF0000E013C00F3AB8014F1360FDEBF79
:1018E000002001F0004170BDC4F10004203C35DA55
:1018F0000C341BDC04F11404C4F1200500FA05F3D8
:1019000020FA04F001FA05F240EA020001F0004278
:1019100021F0004110EBD37021FA04F642EB0601EE
:101920005EEA430E08BF20EAD37070BDC4F10C0418
:10193000C4F1200500FA04F320FA05F001FA04F2DC
:1019400040EA020001F0004110EBD37041F10001C8
:101950005EEA430E08BF20EAD37070BDC4F12005D3
:1019600000FA05F24EEA020E20FA04F301FA05F23B
:1019700043EA020321FA04F001F0004121FA04F2E3
:1019800020EA020000EBD3705EEA430E08BF20EAB3
:10199000D37070BD94F0000F0FD101F000464000ED
:1019A00041EB010111F4801F08BF013CF7D041EA6F
:1019B000060195F0000F18BF704703F00046520073
:1019C00043EB030313F4801F08BF013DF7D043EA44
:1019D0000603704794EA0C0F0CEA135518BF95EAFA
:1019E0000C0F0CD050EA410618BF52EA4306D1D181
:1019F00081EA030101F000414FF0000070BD50EAA0
:101A0000410606BF1046194652EA430619D094EA29
:101A10000C0F02D150EA013613D195EA0C0F05D113
:101A200052EA03361CBF104619460AD181EA030167
:101A300001F0004141F0FE4141F470014FF000001F
:101A400070BD41F0FE4141F4780170BD70B54FF0BA
:101A5000FF0C4CF4E06C1CEA11541DBF1CEA13553A
:101A600094EA0C0F95EA0C0F00F0A7F8A4EB05041C
:101A700081EA030E52EA03354FEA013100F0888013
:101A80004FEA03334FF0805545EA131343EA1263DC
:101A90004FEA022245EA111545EA10654FEA002691
:101AA0000EF000419D4208BF964244F1FD0404F54A
:101AB000407402D25B084FEA3202B61A65EB0305A6
:101AC0005B084FEA32024FF480104FF4002CB6EB63
:101AD000020E75EB030E22BFB61A754640EA0C00E3
:101AE0005B084FEA3202B6EB020E75EB030E22BF23
:101AF000B61A754640EA5C005B084FEA3202B6EB64
:101B0000020E75EB030E22BFB61A754640EA9C0022
:101B10005B084FEA3202B6EB020E75EB030E22BFF2
:101B2000B61A754640EADC0055EA060E18D04FEAB0
:101B3000051545EA16754FEA06164FEAC30343EA50
:101B400052734FEAC2025FEA1C1CC0D111F4801F1D
:101B50000BD141EA00014FF000004FF0004CB6E716
:101B600011F4801F04BF01430020B4F1FD0C88BFB5
:101B7000BCF5E06F3FF6AFAEB5EB030C04BFB6EBC0
:101B8000020C5FEA500C50F1000041EB045170BDB3
:101B90000EF0004E4EEA113114EB5C04C2BFD4EBE0
:101BA0000C0541EA045170BD41F480114FF0000E64
:101BB000013C90E645EA060E8DE60CEA135594EAE0
:101BC0000C0F08BF95EA0C0F3FF43BAF94EA0C0FE3
:101BD0000AD150EA01347FF434AF95EA0C0F7FF458
:101BE00025AF104619462CE795EA0C0F06D152EAAC
:101BF00003353FF4FDAE1046194622E750EA410690
:101C000018BF52EA43067FF4C5AE50EA41047FF4A0
:101C10000DAF52EA43057FF4EBAE12E74FF0FF3C05
:101C200006E000BF4FF0010C02E000BF4FF0010CD6
:101C30004DF804CD4FEA410C7FEA6C5C4FEA430C4F
:101C400018BF7FEA6C5C1BD001B050EA410C0CBF9E
:101C500052EA430C91EA030F02BF90EA020F002000
:101C6000704710F1000F91EA030F58BF994208BF67
:101C700090422CBFD8176FEAE37040F00100704724
:101C80004FEA410C7FEA6C5C02D150EA013C07D17B
:101C90004FEA430C7FEA6C5CD6D152EA033CD3D0C6
:101CA0005DF8040B704700BF8446104662468C46C0
:101CB0001946634600E000BF01B5FFF7B7FF0028F3
:101CC00048BF10F1000F01BD4DF808EDFFF7F4FF1C
:101CD0000CBF012000205DF808FB00BF4DF808EDA7
:101CE000FFF7EAFF34BF012000205DF808FB00BFCA
:101CF0004DF808EDFFF7E0FF94BF012000205DF8EC
:101D000008FB00BF4DF808EDFFF7CEFF94BF0120A0
:101D100000205DF808FB00BF4DF808EDFFF7C4FF99
:101D200034BF012000205DF808FB00BF4FEA410CE2
:101D30007FEA6C5C02D150EA013C0AD14FEA430CC5
:101D40007FEA6C5C02D152EA033C02D14FF0000002
:101D500070474FF0010070474FEA410212F5001240
:101D600015D211D56FF47873B3EB625212D94FEAE2
:101D7000C12343F0004343EA505311F0004F23FACC
:101D800002F018BF404270474FF00000704750EA21
:101D9000013005D111F0004008BF6FF000407047DE
:101DA0004FF00000704700BF4FEA4102B2F1E0433C
:101DB00024BFB3F5001CDCF1FE5C0DD901F0004C32
:101DC0004FEAC0024CEA5070B2F1004F40EB830082
:101DD00008BF20F00100704711F0804F21D113F1AE
:101DE0003872BCBF01F00040704741F480114FEAE7
:101DF0005252C2F11802C2F1200C10FA0CF320FA70
:101E000002F018BF40F001004FEAC1234FEAD3238C
:101E100003FA0CFC40EA0C0023FA02F34FEA4303F6
:101E2000CCE77FEA625307D150EA01331EBF4FF07F
:101E3000FE4040F44000704701F0004040F0FE409A
:101E400040F40000704700BF80F0004002E000BF97
:101E500081F0004142001FBF5FEA410392EA030F95
:101E60007FEA226C7FEA236C6AD04FEA1262D2EBDF
:101E70001363C1BFD218414048404140B8BF5B42E4
:101E8000192B88BF704710F0004F40F4000020F07D
:101E90007F4018BF404211F0004F41F4000121F093
:101EA0007F4118BF494292EA030F3FD0A2F10102DD
:101EB00041FA03FC10EB0C00C3F1200301FA03F11B
:101EC00000F0004302D5494260EB4000B0F5000F3E
:101ED00013D3B0F1807F06D340084FEA310102F1FD
:101EE0000102FE2A51D2B1F1004F40EBC25008BFAF
:101EF00020F0010040EA03007047490040EB000079
:101F0000013A28BFB0F5000FEDD2B0FA80FCACF179
:101F1000080CB2EB0C0200FA0CF0AABF00EBC250A6
:101F200052421843BCBFD0401843704792F0000F94
:101F300081F4000106BF80F400000132013BB5E7E7
:101F40004FEA41037FEA226C18BF7FEA236C21D05D
:101F500092EA030F04D092F0000F08BF08467047C2
:101F600090EA010F1CBF0020704712F07F4F04D190
:101F7000400028BF40F00040704712F100723CBFA3
:101F800000F50000704700F0004343F0FE4040F4CD
:101F9000000070477FEA226216BF08467FEA23638B
:101FA0000146420206BF5FEA412390EA010F40F476
:101FB000800070474FF0000304E000BF10F00043C2
:101FC00048BF40425FEA000C08BF704743F09643A9
:101FD00001464FF000001CE050EA010208BF7047C4
:101FE0004FF000030AE000BF50EA010208BF70474B
:101FF00011F0004302D5404261EB41015FEA010C60
:1020000002BF84460146002043F0B64308BFA3F157
:102010008053A3F50003BCFA8CF2083AA3EBC25339
:1020200010DB01FA02FC634400FA02FCC2F1200258
:10203000BCF1004F20FA02F243EB020008BF20F08F
:102040000100704702F1200201FA02FCC2F12002F5
:1020500050EA4C0021FA02F243EB020008BF20EAEA
:10206000DC7070474FF0FF0C1CEAD0521EBF1CEA18
:10207000D15392EA0C0F93EA0C0F6FD01A4480EA06
:10208000010C400218BF5FEA41211ED04FF00063EF
:1020900043EA501043EA5111A0FB01310CF000401B
:1020A000B1F5000F3EBF490041EAD3715B0040EA41
:1020B000010062F17F02FD2A1DD8B3F1004F40EB11
:1020C000C25008BF20F00100704790F0000F0CF0E4
:1020D000004C08BF49024CEA502040EA51207F3AA8
:1020E000C2BFD2F1FF0340EAC250704740F4000083
:1020F0004FF00003013A5DDC12F1190FDCBF00F074
:1021000000407047C2F10002410021FA02F1C2F121
:10211000200200FA02FC5FEA310040F1000053EABD
:102120004C0308BF20EADC70704792F0000F00F00B
:10213000004C02BF400010F4000F013AF9D040EA11
:102140000C0093F0000F01F0004C02BF490011F4A5
:10215000000F013BF9D041EA0C018FE70CEAD153A3
:1021600092EA0C0F18BF93EA0C0F0AD030F0004C23
:1021700018BF31F0004CD8D180EA010000F00040D7
:10218000704790F0000F17BF90F0004F084691F095
:10219000000F91F0004F14D092EA0C0F01D14202CF
:1021A0000FD193EA0C0F03D14B0218BF084608D198
:1021B00080EA010000F0004040F0FE4040F40000E2
:1021C000704740F0FE4040F4400070474FF0FF0C75
:1021D0001CEAD0521EBF1CEAD15392EA0C0F93EABC
:1021E0000C0F69D0A2EB030280EA010C49024FEA0E
:1021F000402037D04FF0805343EA111143EA1013C7
:102200000CF000408B4238BF5B0042F17D024FF47E
:10221000000C8B4224BF5B1A40EA0C00B3EB510F59
:1022200024BFA3EB510340EA5C00B3EB910F24BF42
:10223000A3EB910340EA9C00B3EBD10F24BFA3EBC7
:10224000D10340EADC001B0118BF5FEA1C1CE0D18F
:10225000FD2A3FF650AF8B4240EBC25008BF20F042
:10226000010070470CF0004C4CEA50207F32C2BF96
:10227000D2F1FF0340EAC250704740F400004FF033
:102280000003013A37E792F0000F00F0004C02BF64
:10229000400010F4000F013AF9D040EA0C0093F02E
:1022A000000F01F0004C02BF490011F4000F013B88
:1022B000F9D041EA0C0195E70CEAD15392EA0C0FF0
:1022C00008D142027FF47DAF93EA0C0F7FF470AF28
:1022D000084676E793EA0C0F04D14B023FF44CAF6B
:1022E00008466EE730F0004C18BF31F0004CCAD100
:1022F00030F000427FF45CAF31F000437FF43CAF3C
:102300005FE700BF4FF0FF3C06E000BF4FF0010C5D
:1023100002E000BF4FF0010C4DF804CD4FEA40023F
:102320004FEA41037FEA226C18BF7FEA236C11D089
:1023300001B052EA530C18BF90EA010F58BFB2EB3C
:10234000030088BFC81738BF6FEAE17018BF40F0BC
:10235000010070477FEA226C02D15FEA402C05D170
:102360007FEA236CE4D15FEA412CE1D05DF8040BF5
:10237000704700BF844608466146FFE70FB5FFF788
:10238000C9FF002848BF10F1000F0FBD4DF808ED40
:10239000FFF7F4FF0CBF012000205DF808FB00BF31
:1023A0004DF808EDFFF7EAFF34BF012000205DF88B
:1023B00008FB00BF4DF808EDFFF7E0FF94BF0120D8
:1023C00000205DF808FB00BF4DF808EDFFF7D2FFD5
:1023D00094BF012000205DF808FB00BF4DF808ED18
:1023E000FFF7C8FF34BF012000205DF808FB00BFE5
:1023F0004FEA40024FEA41037FEA226C02D15FEAD2
:10240000402C08D17FEA236C02D15FEA412C02D133
:102410004FF0000070474FF0010070474FEA400254
:10242000B2F1FE4F0FD34FF09E03B3EB12620DD902
:102430004FEA002343F0004310F0004F23FA02F06C
:1024400018BF404270474FF00000704712F1610F13
:1024500001D1420205D110F0004008BF6FF00040EA
:1024600070474FF00000704742000ED2B2F1FE4FAD
:102470000BD34FF09E03B3EB126209D44FEA002353
:1024800043F0004323FA02F070474FF0000070471A
:1024900012F1610F01D1420202D14FF0FF307047BB
:1024A0004FF00000704700BF53B94AB9002908BF78
:1024B00000281CBF4FF0FF314FF0FF3000F06AB929
:1024C000ADF1080C6DE904CE00F006F8DDF804E08B
:1024D000DDE9022304B070472DE9F047089D0C4662
:1024E000002B4ED194468C458646B2FA82F262D9D0
:1024F0004AB1C2F12003914020FA03F30CFA02FC26
:10250000194300FA02FE4FEA1C471FFA8CF6B1FB92
:10251000F7F44FEA1E4307FB141143EA014304FB9F
:1025200006F199420AD91CEB030304F1FF3080F055
:102530001281994240F20F81023C6344591A1FFAFA
:102540008EF3B1FBF7F007FB101143EA014300FBE8
:1025500006F69E420AD91CEB030300F1FF3180F01E
:10256000FC809E4240F2F980634402389B1B40EAA3
:10257000044000211DB1D3400022C5E90032BDE86E
:10258000F0878B4205D90DB1C5E90001002108464D
:10259000F5E7B3FA83F1002946D1A34202D3904272
:1025A000C0F0F080861A64EB03030120002DE6D012
:1025B000C5E90063E3E7002A40F09080A1EB0C043A
:1025C0004FEA1C481FFA8CF70121B4FBF8F64FEADA
:1025D0001E4308FB164443EA044307FB06F09842F7
:1025E00008D91CEB030306F1FF3402D2984200F233
:1025F000CD8026461C1A1FFA8EF3B4FBF8F008FBB8
:10260000104443EA044300FB07F79F4208D91CEB40
:10261000030300F1FF3402D29F4200F2B080204653
:10262000DB1B40EA0640A5E7C1F120068B4022FAF9
:1026300006F71F4320FA06FC04FA01F343EA0C03F1
:10264000F44000FA01F8380C4FEA1349B4FBF0FEED
:102650001FFA87FC00FB1E4449EA04440EFB0CF9F8
:10266000A14502FA01F20AD93C190EF1FF3A80F0B5
:102670008480A14540F28180AEF1020E3C44A4EB7F
:1026800009041FFA83F9B4FBF0F300FB134449EA91
:10269000044403FB0CFCA44507D93C1903F1FF30AB
:1026A00067D2A44565D9023B3C4443EA0E40A0FBF7
:1026B0000293A4EB0C049C42CE469C4651D34ED0D0
:1026C00055B1B8EB0E0364EB0C0404FA06F6CB40EC
:1026D0001E43CC40C5E90064002150E7C2F120034D
:1026E00020FA03F10CFA02FC24FA03F394400C43A1
:1026F0004FEA1C4800FA02FE1FFA8CF7B3FBF8F011
:1027000008FB1031230C43EA014300FB07F1994217
:1027100008D91CEB030300F1FF362CD299422AD9C9
:10272000023863445B1AA4B2B3FBF8F108FB11331F
:1027300044EA034401FB07F3A34208D91CEB040459
:1027400001F1FF3613D2A34211D902396444E41ACD
:1027500041EA004139E70446F0E6084606E7C84585
:10276000AED2B9EB020E63EB070C0138A8E7314695
:10277000EDE7034699E73046D4E7D6467FE7634462
:1027800002384DE70646234608460FE7023E6344FB
:1027900030E700BF704700BF00487047001BB74BD1
:1027A00070B50C4601F0ECF9104E05460821304694
:1027B00005F08AFA012804D001F0E2F9431BA34294
:1027C00007D30821094805F07FFA431E58425841B3
:1027D00070BD72B60821304605F076FA012800D0A7
:1027E00030BF62B6BFF36F8FE0E700BF0004004860
:1027F00008B5002210214FF0904005F06BFA054813
:102800000022202105F066FABDE80840022001F010
:10281000BFB900BF0004004810B50C4C01221021C4
:10282000204605F057FA052001F0B2F920460122B2
:10283000202105F04FFA4FF090400122102105F0C1
:1028400049FABDE81040022001F0A2B90004004896
:1028500070B54FF090400C46164610210022144DE2
:1028600005F038FA00232B701248B3B222462146F5
:1028700006F024FCD8B901F083F941F2873604460A
:102880002B783BB1BDE87040012210214FF0904001
:1028900005F020BA01F074F9031BB342F2D872B606
:1028A0002B7803B930BF62B6BFF36F8FE8E770BD16
:1028B000BD05002020070020014B01221A7070473F
:1028C000BD050020004870473861030813B5114B5F
:1028D0000446186800909B88ADF804300120FFF78B
:1028E0009BFF062269460120FFF7B2FF0120FFF798
:1028F0007FFF9DF80430112B08D19DF80520122A86
:1029000004D101202370627002B010BD00231A466A
:102910001846F7E7002003080CB4F0B5ADB032ABB1
:1029200006AF53F8042B059305460E46384696210C
:102930002CF056F89528C1BF42F62E63ADF8AA30A8
:102940002E23ADF8AC3000F037F83C24042D4FF4C2
:102950007A7E1449B0FBFEFCB0FBF1F14EF6602329
:10296000B0FBF3F3B3FBF4F204FB1232BCFBF4F361
:1029700004FB13C30EFB1C049ABF0B48405D3F20B1
:10298000CDE90040CDE9026708482BF0A9FF084BCC
:102990001B6898682BF0CEFE2DB0BDE8F04002B069
:1029A000704700BF80EE360096610308746103082B
:1029B000CC03002001F0ECB801F0E2B81348144A4F
:1029C00008B54FF00043C0E9002304224261012210
:1029D0000023C2614FF480510722C0E90233C0E9ED
:1029E0000933C0E90C1203610383837680F8203039
:1029F00080F82C30826380F83C30C36404F0BCF86B
:102A000018B1BDE8084000F099BB08BDC005002022
:102A1000002401400268084B9A4282B00AD14FF06C
:102A2000B0431A6E42F400721A661B6E03F4007310
:102A30000193019B02B07047002401400268054BDE
:102A40009A4201BF4FF0B042136E23F40073136635
:102A5000704700BF0024014030B585B00024054612
:102A6000CDE901440394FFF7A9FF144804F018FCD2
:102A700008B100F063FB1148039401A9CDE90154AA
:102A800004F0D8F908B100F059FB0C4804F032FB0F
:102A900008B100F053FB4FF0FF31084804F06CF927
:102AA000064804F0DFFB054804F0C0F9044603487B
:102AB00004F082FB204605B030BD00BFC0050020F9
:102AC000014B024A1A607047C005002000240140F3
:102AD00008B50948FFF7C0FF68B1084BB3F8AA3042
:102AE0004FF6FF72934216BF40F6E442044B534345
:102AF000B3FBF0F398B208BD002000B40075FF1FCF
:102B0000D8084C0013B50023ADF80630FFF7E0FFFE
:102B100004461948FFF7A0FF184BB3F8C820B3F8D4
:102B2000A8108A4204FB00F018D040F6E443B0FB42
:102B3000F3F364205B1A4343521A93FBF2F31E3300
:102B40001BB2ADF80630BDF806305BB21B02ADF823
:102B50000630BDF8060000B202B010BD4FF47A7224
:102B600040F6FF73B0FBF3F35343A3F53923A3F50A
:102B70000C6340F6C412E0E7001000B00075FF1FC0
:102B80004FF0B04382B09A6A22F480529A629A6CF3
:102B900042F480529A649B6C03F480530193019B2E
:102BA000002002B070474FF0B04307B59A6C42F076
:102BB00004029A649A6C02F004020192019A9A6CDF
:102BC00042F001029A649B6C002203F0010311465B
:102BD00000930B20009B04F001FC0B2004F030FC60
:102BE000002211460C2004F0F9FB0C2004F028FC14
:102BF000002211460D2004F0F1FB0D2004F020FC12
:102C0000002202210F2004F0E9FB0F2004F018FC41
:102C100000221146102004F0E1FB102004F010FC0B
:102C200000221146112004F0D9FB112003B05DF8F9
:102C300004EB04F005BC000008B504F045FE10B13B
:102C40006FF0040008BD064B9A6942F040429A6159
:102C50004CF2FA321A6104F049FE0028F2D0EFE794
:102C600000400058F0B585B000230D46009306469D
:102C7000A8B3FFF7E1FF044670BB04F025FE88BB54
:102C80001A481B4A02230193D0F8E01506F1784355
:102C900002EA8121B3FBF1F701FB1733DB0A029350
:102CA000D0F8E00505F178410139314402EA80228B
:102CB000B1FBF2F002FB1011C3EBD12301336946E3
:102CC00001A8039304F092FE20B1022814BF6FF014
:102CD0000104012404F00AFE204605B0F0BD6FF0A7
:102CE0000504F9E76FF00404F6E700BF0070FF1F6A
:102CF00000FCFF03014B18600020704724060020F1
:102D00002DE9F04FB0F1006F89B006460F469046AE
:102D1000C0F0C080DFF89091644DD9F8E03505EA45
:102D2000832303F10063013B984200F2B380002942
:102D300000F0B38040EA02035B0740F0AE80FFF78B
:102D40007BFF044690BB04F0BFFD002840F0A88044
:102D5000D9F8E015009705EA812106F17842B2FB27
:102D6000F1F301FB132208F17843013B3344B3FB39
:102D7000F1F001FB1033DB0A01334FEAD22AA3EB57
:102D8000D222012A039388BFC6F30A050AF58037C9
:102D9000C6F108038CBFC5F500654546FF02B34682
:102DA0000693039B9A4505D304F0A0FD204609B085
:102DB000BDE8F08FA6F10803069A1A4495421CD884
:102DC000009B04950193CDF814B04FF00009059BCA
:102DD00009EB0301049B99453DD3009BAB442B4475
:102DE000A8EB0505B5F5006F009328BF4FF400650B
:102DF0000AF1010A07F50067D3E753F8081F5A687C
:102E0000B2F1FF3F08BFB1F1FF3FD5D0284B1868A2
:102E100010B96FF00504C7E727B14FF400623946D7
:102E200011F0E6FFDFF888900099D9F80030CBF375
:102E30000A001844AAB211F0DBFF4FF400613846D3
:102E4000FFF710FF00BBD9F8003001934FF4006387
:102E500005970493B9E7019B07914B440293012026
:102E6000D3E9002304F07CFD88B90799019BD1E9DF
:102E7000000259F80310029B5B689A4208BF88421F
:102E800005D109F10809A2E76FF001048CE76FF0A2
:102E9000030489E74FF0FF3488E76FF0050485E706
:102EA0006FF0040482E700BF0070FF1F00FCFF0307
:102EB00024060020B1F1006F70B510D30B4BD3F88E
:102EC000E0650B4B03EA862303F10063013B994263
:102ED00005D838B192B211F08BFF002070BD4FF0D1
:102EE000FF30FBE76FF00500F8E700BF0070FF1F41
:102EF00000FCFF03B0F1006F10B40DD3084BD3F802
:102F0000E045084B03EA842303F10063013B984248
:102F100002D810BCFFF7A6BE4FF0FF3010BC7047C0
:102F20000070FF1F00FCFF034FF0B04382B0DA6C6B
:102F30000243DA64DB6C03400193019B02B07047EB
:102F40002DE9F04186B01422002101A82BF066FD86
:102F50000220464EFFF7E8FF0420FFF7E5FF0120BF
:102F6000FFF7E2FF04213046002204F0B3FE002206
:102F700010214FF0904004F0ADFE04230024012501
:102F800002270DEB03013046CDE901354FF0100863
:102F9000CDE9034704F078FD01A93046CDE901856C
:102FA000CDE9037404F070FD202301A93046CDE97A
:102FB0000135CDE9037404F067FD01A94FF090409D
:102FC000CDE90185CDE9034404F05EFD08224FF40C
:102FD000881301A93046CDE901234FF00308CDE95C
:102FE000034704F051FD4FF4441301A94FF0904002
:102FF000CDE90183CDE9035704F046FD4FF440537A
:1030000001A93046CDE90135CDE9034804F03CFD86
:103010004FF404134021CDE901131548039501A98C
:1030200004F032FD22460F21062004F0D7F90620D5
:1030300004F006FA22460F21072004F0CFF90720FA
:1030400004F0FEF922462146092004F0C7F90920C0
:1030500004F0F6F922462146092004F0BFF90920C0
:1030600004F0EEF906B0BDE8F08100BF00040048AE
:103070000008004800B59BB04822002108A82BF0AA
:10308000CDFC1822002102A82BF0C8FC04F03CFE65
:103090004FF0B0420120D2F8903023F01803C2F86C
:1030A0009030D2F8003423F4C06343F40073C2F8C4
:1030B0000034D2F8003403F4C0630193019B24234D
:1030C000089381230B930023CDE91003B02208A8B5
:1030D000CDE9122304F090FF08B172B6FEE74F234A
:1030E000CDE90230CDE90400CDE90600022102A8B5
:1030F00005F01CFA08B172B6FEE71BB05DF804FBE0
:1031000008B503F0E7FCFFF7B5FFFFF719FFFFF77E
:103110004AFD00F0D1FF00F063FE00F089F8064898
:103120000122042104F0D6FD02F07CF900F018FC25
:1031300002F07FF9FCE700BF0004004872B6FEE72A
:1031400000B58DB02C22002101A82BF067FC174898
:10315000174B03601F2383604FF080420023C0E9B8
:103160000433C0E9072383614FF48073436205F0A1
:1031700083FC08B1FFF7E2FF0C4805F0A9FD08B198
:10318000FFF7DCFF4FF00053002207930748089237
:103190004FF4807301A9029206920B9305F0CCFCC8
:1031A00008B1FFF7CBFF0DB05DF804FB2806002047
:1031B0000028004010B5044690B03822002102A833
:1031C0002BF02CFC2268194B9A422CD14FF48033FF
:1031D000029302A84FF480730F9305F0CBFA08B165
:1031E000FFF7ACFF4FF0B0430220D3F8902042F439
:1031F0000042C3F890209A6D42F480629A659B6DFC
:10320000002203F4806311460193019B04F0E6F869
:10321000022004F015F900222A20114604F0DEF8FD
:103220002A2004F00DF910B010BD00BF00280040A6
:103230001148124A08B54FF48273C0E900230023F5
:103240004FF4E062C0E902324FF400712822C0E975
:1032500006120722C0E90433C0E90833C0E90B2392
:1032600083620823436305F0A3FE18B1BDE808405C
:10327000FFF764BF08BD00BF2007002000300140F9
:10328000F0B5054689B01422002103A82BF0C6FB37
:103290002A68374B9A4269D14FF0B04302261A6E22
:1032A00042F480521A661A6E02F480520292029A16
:1032B000DA6C42F00102DA64DA6C02F00102019287
:1032C000019ADA6C42F00202DA64DB6C03F002036A
:1032D00000930524009B0327D02303A94FF09040BF
:1032E000CDE90336CDE9067404F0CEFB2023CDE909
:1032F00003364FF09040002603A90794CDE90567F7
:103300001C4C04F0C1FB1C4826620723C4E90003DF
:1033100080232046C4E90266C4E90436C4E906668F
:1033200004F0EEF808B1FFF709FF144AAC65A56296
:10333000134C0823C4E900231021002380222046D7
:10334000C4E90213C4E90423C4E90633236204F088
:10335000D7F808B1FFF7F2FE002222206C65114673
:10336000A56204F03BF8222004F06AF809B0F0BD31
:1033700000300140C00600201C0002403000024026
:10338000600600207047000008B503F0B9FB044B4D
:103390000120C3F88800BDE8084004F00DBD00BF5F
:1033A0000004005808B503F0B2FB00F095FFFFF7EA
:1033B000C7FDFFF7F8FB00F013FDBDE80840FFF77D
:1033C00037BF08B503F0A3FBFFF7BAFDFFF7EBFB30
:1033D000BDE80840FFF72CBF08B503F091FBBDE83E
:1033E00008400121002004F097BC70477047FEE7B9
:1033F000FEE7FEE7FEE7FEE770477047704770475D
:10340000014805F08BBC00BF28060020024B0120BC
:10341000187004F06DBC00BF721C0020024B01222A
:1034200002201A7004F064BC711C0020082004F013
:103430005FBC0000014804F0D9B900BF2C11002086
:10344000014804F0D3B900BFC0060020014804F0D1
:10345000CDB900BF6006002070470000014804F0AD
:10346000C5B900BFE011002070470000014806F018
:1034700013B800BF20070020014807F091B900BF32
:1034800040120020014805F07DBA00BF2806002048
:10349000014806F092BA00BF181100202DE9F04350
:1034A00089B080460020109E0790894615461F4629
:1034B000FCF7BEFEF0B9104CCDE90090CDE9020456
:1034C00007AB0E480593142304933A464346294616
:1034D0000068FCF777FF2346324604F1140153F8E5
:1034E000044B42F8044B8B42F9D1079B337509B06A
:1034F000BDE8F0830120FAE79A070020286103085D
:103500001FB50E4C00233C2202A8CDE902336275A0
:10351000237500F0DFFA042303AA0094122108485F
:10352000FFF7BCFF0749142220462BF067FAB0FAD8
:1035300080F35B09637504B010BD00BF84070020F1
:10354000B4610308361F0020034A044840F21B53AD
:10355000002106F055BF00BFAE0700208C110020EF
:10356000312BF0B52DD81825102415FB0343194D28
:1035700000244FF0800C4CFA04F6A3F110073142FE
:1035800005EB470714BF4FF0240E4FF0140EA7F8B9
:1035900006E0A3F10807304205EB470714BF4FF0E0
:1035A000240E4FF0140E0134324205EB4306A7F807
:1035B00006E00CBF14272427082CF78003F1010331
:1035C000D9D1054B1B781BB9BDE8F040FFF7BCBF54
:1035D000F0BD00BFAE070020DC1C002010B50024A9
:1035E0000022E3B2114610460134FFF7B9FF322C36
:1035F000F6D1BDE81040FFF7A7BF000070B5044644
:103600000D46FFF7EBFF0F4B04EB440400261C4470
:10361000142000F0BDFAA2786178207812FB05F240
:1036200011FB05F110FB05F0F3B2D2B2C9B2C0B282
:103630000136FFF795FF322EEAD1BDE870400A202F
:1036400000F0A6BA080000202DE9F04106460F461A
:103650002048904600214FF416622BF0DFF91E4AF5
:1036600010254FF0800C2B4600244CFA04F1A3F1F6
:1036700010000F4202EB400014BF4FF0240E4FF039
:10368000140EA0F806E0A3F108000E4202EB400081
:1036900014BF4FF0240E4FF0140E013418EA010F3E
:1036A00002EB4301A0F806E00CBF14202420082CF4
:1036B000C88003F10103D8D11835B5F5986FD2D180
:1036C000064B1B781BB9BDE8F041FFF73DBFBDE8D5
:1036D000F08100BFB4070020AE070020DC1C0020F2
:1036E00000F00F000B4607281ED8DFE800F00407A3
:1036F0000A0F1316191B0022114600E00022104683
:1037000002E0002211461846FFF79EBF0A4600213C
:103710000020F9E700220846F6E70A460021EEE716
:103720000A46F5E70A46E7E770470000024B1878BB
:10373000024B1978FFF7D4BF0600002000000020DC
:1037400070B57248724C0378DBB20B2B33D8DFE8CC
:1037500013F00C00120016001C0024006100900001
:10376000A500B600C500C500C5006A4B1B78DBB2DA
:10377000694A13701FE0684B00221A701BE0674A09
:103780001278012A08BF0123F2E7654B1A78002A54
:1037900040F09080604B0122EFE7614A614B117865
:1037A00039BB61490978012923D119780129CDB2A2
:1037B0001FD1594B1D7003785C4E012B06D05C4D18
:1037C0002A7802F0FF03002A00F08D80524A00237D
:1037D000137023703370FFF701FF564B1B7823B92A
:1037E000554B1A780AB91B7813B1544B01221A7041
:1037F00070BD1278012A05D04B4A127812B11A789E
:10380000002AD8D1444A022111701B78002BD2D152
:103810002323AEE7424A404B157842499DB9424DB9
:103820002D78012D0FD10D78012DEEB20BD11E7028
:10383000434A1578022DEAB212D0032A0FD0012A8A
:1038400015D123220CE01278012A05D0364A1278CD
:1038500012B10A78002AEBD102221A70E8E704229A
:1038600022701A700A78002AA5D1232285E7022245
:10387000F6E72B4B1A783AB9284A1278012AD1B2C6
:1038800002D1254B197096E71B78012B03D0234BEF
:103890001B78002B8FD1204B02226EE7204B1A7829
:1038A00022B9284A1278002A3FF474AF1B78012B02
:1038B000F1D0244B1B78012B7FF47DAFEBE7184B45
:1038C0001A7822B9204A1278042A3FF463AF1B7891
:1038D000012BE0D01C4B1B78052BEDE71A4B1A7817
:1038E000042AF8D156E72A7812B90B4B1B78DBB2C1
:1038F0002370164B20781978FFF7F2FE2B7803B16E
:1039000023782378DBB2337067E700BF3E000020E6
:10391000060000200400002007000020351F0020C2
:10392000631C002041000020420000200100002014
:10393000DC1C0020641C0020651C0020D41C00201E
:10394000EA120020621C0020611C00200000002000
:10395000024803680021596306F0CCBD8C11002099
:1039600038B501240A25294620461435FFF7B8FE4C
:10397000EDB2322000F00CF96E2DF4D10134E4B236
:10398000FFF72CFE082CEDD138BD0000054808B526
:103990000823036005F02EFE18B1BDE80840FFF7CC
:1039A000CDBB08BD181100204FF0B04307B55A6ECB
:1039B00042F001025A665B6E002203F0010301939C
:1039C00011463220019B03F009FD322003B05DF85F
:1039D00004EB03F035BD00000CB407B5054A05AB98
:1039E0001021019311F0D0FD03B05DF804EB02B09B
:1039F000704700BFC661030830B585B0044602A811
:103A00000D4611F059FBBDF90C30064A0093102108
:103A1000029B2046FFF7E0FF2046FDF729FD2880A6
:103A200005B030BDC66103084FF0B04210B59368D1
:103A300023F40043936011F05BFC104B01241C70D5
:103A400000F0ACF811F064F80D4811F07BF80D4B64
:103A50004FF400421A61002011F07AF8FFF730F8B5
:103A600000F0F8F811F06EF92146204611F08AF9BD
:103A700021462046BDE8104011F06EB92411002007
:103A8000F93900080040005811F092B908B5FFF765
:103A90001FF840F6B83398420CD8B0F5E16F0BD35D
:103AA000FE23A0F5E16058434FF49663B0FBF3F0BA
:103AB000C0B208BDFE20FCE70020FAE77FB56846EB
:103AC00000F0ACF80198FEF7A9FC00B207B05DF871
:103AD00004FB0000194A38B5D2F88035591C044659
:103AE00019D103F01BF8054603F024F8054403F050
:103AF0001BF82B0EE3712B0CA3712B0A6371030EC1
:103B0000E370C0F30742C0F307232571C0B2A2706F
:103B10006370207038BD190AC3718171190C1B0EB6
:103B200041710371D2F88435C370D2F88405C0F3B3
:103B30000722C0F30743000EE9E700BF0070FF1F34
:103B400038B5094BD3F8803503600133054609D1F8
:103B500002F0E4FF044602F0E7FF444002F0EAFF0F
:103B600044402C6038BD00BF0070FF1F01210220BF
:103B700011F0F2B80021022011F0EEB800207047D9
:103B8000024B187808B100F0D3B970472411002017
:103B900082B00190019802B000F066BAF0B589B029
:103BA00002F0CEFF02F0D4FF02F0DAFF012304930B
:103BB0000323069300254FF0B04305950795DA6C73
:103BC000154C42F00202DA64DA6C02F00202029250
:103BD000029ADA6C42F00202DA64DB6C03F0020350
:103BE00001934FF4805703A92046019B03974FF49C
:103BF000005603F049FF03A92046039603F044FF53
:103C00002A463946204604F065F82A4631462046C1
:103C100004F060F809B0F0BD0004004810B5044697
:103C2000FEF770FF074BA36040F30F20FEF7C6F9C5
:103C3000054B064A2360064B6060C4E9032300205D
:103C400010BD00BF0000484200007A440D093E004C
:103C5000AB030500002070470120704708B52AF02B
:103C60003FFF162303604FF0FF3008BD08B52AF070
:103C700037FF16230360FEE770B50D4614460E4667
:103C8000731B9C4201DC204670BDAFF3008006F838
:103C9000010BF5E730B5104600234FF06042834238
:103CA00000DB30BDD2F8804EE50707D5D2F8004ED4
:103CB000E40703D5CC5C156815B114700133EEE749
:103CC00000BFF8E74FF0FF3070474FF400534B60F0
:103CD0000020704701207047002070470B4A116890
:103CE00010B5034609B90A491160106809490A4C20
:103CF0000344091B8B4206D92AF0F2FE0C23036011
:103D00004FF0FF3010BD1360FCE700BF281100200A
:103D1000783F0020000001200008000037B5184B54
:103D200002689A42054628D14FF0B043154C1A6EEE
:103D300042F400621A661B6E134A03F40063019397
:103D4000019B1723C4E90023102100238020C4E92C
:103D500002134FF48073C4E904034FF4806C2023F2
:103D6000C4E906C320464FF40053236203F0C8FBA6
:103D700008B1FFF7E3F96C62A56203B030BD00BF84
:103D8000002C01402C1100200800024010B5044610
:103D900086B01422002101A82AF040FE22680F4BB1
:103DA0009A4218D14FF0B04301A9DA6C42F00102F7
:103DB000DA64DB6C03F0010300930222009B4FF4F2
:103DC0008073CDE901324FF090400123CDE90332F9
:103DD000059303F059FE06B010BD00BF002C014052
:103DE00010B510229CB0002400210DEB02002AF037
:103DF00015FE1C22214608A8CDE9014403942AF0AF
:103E00000DFE342221460FA82AF008FE2B482C4B29
:103E10008460C0E900343B23C0E90334C0E90544B1
:103E200006F034F808B1FFF789F94FF480532348BE
:103E3000049304A906F048F908B1FFF77FF91F4879
:103E400006F054F808B1FFF779F900241B480394F1
:103E500001A9CDE9014406F04FFB08B1FFF76EF967
:103E6000602316480E94002208A9CDE90834CDE954
:103E70000A44CDE90C4406F0A1F808B1FFF75EF959
:103E800000234FF40052CDE914230C4813934FF054
:103E900000720FA9CDE90F33CDE91133CDE9163307
:103EA000CDE91823CDE91A3306F052FB08B1FFF72C
:103EB00045F90248FFF76AFF1CB010BD8C110020C5
:103EC000002C0140014B1868704700BFD81100203A
:103ED0000320704708B501464FF47A720023800230
:103EE000890DFEF7E1FA08BD4FF47A73A0FB0303D6
:103EF000800A40EA83507047034B98689A68904262
:103F0000FBD1C043704700BF0028004008B5FFF751
:103F1000F3FF014B186008BDD811002008B5FFF76A
:103F2000EBFF024B1B68C01A08BD00BFD811002070
:103F3000024B187808B1FFF7DFBF7047DC11002093
:103F400010B5074B074C0122DA654FF4807120460B
:103F500004F0DEFC4FF0FF332363002010BD00BFF0
:103F6000002800402806002002460021014804F0F5
:103F7000E6BE00BF2806002002460121014804F0E9
:103F8000DEBE00BF2806002010B58CB02C22002118
:103F9000044601A82AF042FDFFF7D2FF0C4B0D4862
:103FA0001B681C440023089306934FF00053E4431E
:103FB000079301224FF4807301A902940B9304F03C
:103FC000BBFD08B1FFF7BAF800200CB010BD00BF70
:103FD000D81100202806002038B50546FFF78CFFD1
:103FE00002210446074804F0B1FEC4F309024FF46D
:103FF0007A71A2FB0121920AA30A2A8043EA805027
:1040000038BD00BF280600200148002104F09EBEF4
:10401000280600200148012104F098BE280600204F
:10402000F8B50F4D2E78CEB90E4C4FF0FF37276301
:10403000FFF786F8FFF784FF4FF48071204604F005
:1040400067FC2046276304F025FE32462046022105
:1040500004F075FEFFF75AFF01232B700020F8BD16
:10406000DC11002028060020014610B54FF47A72BA
:1040700000238002890DFEF717FA0146FFF73CFF87
:104080000446FFF739FF031B8B4200D310BD00BF6E
:10409000F7E711F035BA000010B5064C02212046B2
:1040A00004F054FE0221421C2046BDE8104004F0FA
:1040B00046BE00BF280600201648174A08B54FF430
:1040C000E133C0E9002300230C22C0E90233C0E938
:1040D0000523C0E90733C0E90933036107F045F957
:1040E00008B1FFF72BF80B48002107F0B6FA08B12A
:1040F000FFF724F80748002107F0CFFA08B1FFF7CF
:104100001DF8044807F089FA18B1BDE80840FFF728
:1041100015B808BD401200200044004070B596B0AC
:1041200006461422002103A82AF078FC3822002138
:1041300008A82AF073FC3268274B9A424AD102231E
:10414000089308A84FF440230A9304F013FB08B126
:10415000FEF7F4FF4FF0B04300259A6D1F4C42F478
:1041600000329A659A6D02F400320292029ADA6C79
:1041700042F00102DA64DB6C03F001030193019B5E
:104180000C220223CDE9032303A907234FF090401B
:104190000793CDE9055503F077FC114925621423F7
:1041A000C4E900131023C4E9023520468023C4E982
:1041B0000435C4E9065503F0A3F908B1FEF7BEFFC4
:1041C0002520F46700220221A66203F007F92520CA
:1041D00003F036F916B070BD00440040E011002035
:1041E0008000024002680C4B9A4210B5044612D17E
:1041F0004FF0B0420C21936D23F4003393654FF0E0
:10420000904003F0EDFCE06F03F0ECF9BDE81040E6
:10421000252003F023B910BD0044004008B50A462C
:104220000146024806F020FA002008BD4012002096
:1042300013B5114B114C18604FF40013009302ABEF
:1042400013E90600204607F08CF92368DA69D103E8
:10425000FCD4DA695202FCD59A68084842F480021C
:104260009A6007F0C4F906490448012207F032F9C0
:10427000002002B010BD00BFD41200204012002068
:10428000DC12002008B5074B1860FEF78CFCFFF726
:1042900013FF054AD2F8803043F00063C2F8803043
:1042A000002008BDD81200200008005808B54FF0C3
:1042B000B04308489A6B42F400329A639A6B22F436
:1042C00000329A63FFF78EFF112003F0C7F8002039
:1042D00008BD00BF4012002008B5074807F045F8A8
:1042E00008B1FEF72BFF054803F00AF918B1BDE845
:1042F0000840FEF723BF08BD40120020E011002057
:104300000268044B9A4203D1034B00201B681847F4
:10431000704700BF00440040D812002002680B4BD9
:104320009A4210B504460FD1094B1B682BB1D0F847
:10433000902012B907480121984720460549BDE859
:104340001040012207F0C6B810BD00BF0044004075
:10435000D4120020DC12002030B59BB0FEF7B2FA78
:1043600013F076FD48B1012013F01AFE12F016FB8F
:104370000446019020B913F0DFFD01201BB030BDD1
:104380003A4D296812F05AFF6968204612F070FF12
:10439000297A204612F0A0FF697A204612F0D0FF59
:1043A0006969204613F05CF8E868FEF75DF881B2B1
:1043B000204612F0DFFF2969204612F0A7FFA97AF4
:1043C000204612F06FFF0221204613F021F8102141
:1043D000204613F05FF8019812F068FB029018B9BC
:1043E00001A812F03BFBC6E701A812F037FB0298C8
:1043F00012F0C4FE18B902A812F076FCBBE71C4DFF
:10440000029800232B600A2203AB06A912F0A8FC35
:1044100060B129680798FDF71DFD03AB28600A22EB
:10442000029806A912F09CFC0446C0B90024286832
:104430001049FDF717FE4FF07C51FDF713FE286081
:10444000029812F0CBFE054602A812F04DFC13F0C4
:1044500073FD002D91D084F00100C0B28EE7296871
:104460000798FDF7F7FC2860E1E700BF2000002077
:10447000741C002000007A442DE9F04FADF21C4D71
:104480004FF40072002106A82AF0C8FA4FF4007217
:10449000002186A8B74F2AF0C1FA00243E464FF00B
:1044A00000082546B1682846FDF7D4FC716805462A
:1044B0002046FDF7CFFC08F10408B8F5007F04465C
:1044C00006F11006EED14FF070512846FDF7CAFDF7
:1044D0004FF0705106462046FDF7C4FD0024DFF87A
:1044E000948282464FF000092546D8F808003146EC
:1044F000FDF7AEFC0146FDF7B5FD01462846FDF788
:10450000A9FC51460546D8F80400FDF7A1FC014678
:10451000FDF7A8FD01462046FDF79CFC09F10409C2
:10452000B9F5007F044608F11008DED14FF0705154
:104530002846FDF797FD8346FDF706F98E4B0022CE
:104540002CF0E2F9CDE900014FF070512046FDF763
:1045500089FDFDF7F9F8884B00222CF0D5F9FDF71D
:1045600023FC06AD82462C464FF000094FF00008B0
:10457000B968B869FDF76CFCFDF750FF0028B8BFBB
:104580004042FDF71BFD44F8040B01464046FDF791
:1045900061FC09F10409B9F5FE7F804607F11007B7
:1045A000E6D17649FDF712FE06AC07464FF000094A
:1045B0004FF00008394654F8040BFDF749FC01465A
:1045C000FDF750FD01464846FDF744FC08F101089F
:1045D0001FFA88F8B8F17F0F8146EBD16749FDF7E4
:1045E000F5FDFDF7B1F8644B00222CF08DF9CDE913
:1045F000020186ACA04600234FF000092A46296834
:1046000050680493FDF724FCFDF708FF0028B8BFAD
:104610004042FDF7D3FC049B48F8040B01461846C2
:10462000FDF718FC09F101091FFA89F9B9F17E0FAC
:1046300005F104050346E1D15149FDF7C7FD4FF0EF
:10464000000905464FF00008294654F8040BFDF711
:10465000FFFB0146FDF706FD01464846FDF7FAFB64
:1046600008F101081FFA88F8B8F17E0F8146EBD1F6
:104670004349FDF7ABFDFDF767F83F4B00222CF0F7
:1046800043F9404A13889BB2FA2BCDE9040100F2AA
:10469000C680108880B2FDF791FC5146FDF794FE6C
:1046A000394C08B105232370384B1A78384B1B88D6
:1046B0009BB29A4280F08480364B1A78364B1B8826
:1046C0009BB29A4206D235493046FDF787FE08B1C3
:1046D00001232370324C334D238801339BB2238056
:1046E00023889BB20A2B04BF0023238022884FF02B
:1046F0001C0892B208FB02F2DDE90001AE502288EC
:1047000092B208FB0252C2F804B0FDF74DFBB4F8B8
:1047100000B0228892B208FB02521FFA8BFB08FB02
:104720000B5BC2F80CA0B4F800A0CBF808004FF067
:1047300086413846FDF796FC1FFA8AFA08FB0A5AAA
:104740002788CAF81000DDE90201FDF72DFB4FF0C4
:104750008641FDF787FC22880B4C92B2BFB208FB62
:10476000075708FB0255217878612976DDE90401B5
:104770001AE000BF041400200000E03F0000FE42E9
:104780000000FC423C000020EA120020030100204F
:10479000E212002002010020E0120020CDCC4C3FAC
:1047A000041C0020EC120020FDF7FEFA4FF08641B9
:1047B000FDF758FCFDF758FE244BC0B21880237853
:1047C000DFF88C80234C98F80030234F012B1DD14B
:1047D000DFF88890224DB9F80030B9F800204FF08A
:1047E0001C0A9BB292B20AFB03F30AFB0252E8587E
:1047F0009168FDF72FFB3146FDF7F0FD88B10223EC
:10480000237023782378DBB288F800302378DBB27A
:1048100088F800303E600DF21C4DBDE8F08F114865
:104820003BE7B9F80030D7F800909BB20AFB03557C
:104830003046A968FDF70EFB4946FDF7CFFD10B1E4
:1048400003232370E2E72070E0E700BFDE120020C0
:10485000E8120020EA120020E4120020041C0020CC
:10486000EC12002000007A432DE9F04F93B0FEF7E0
:1048700029F813F0EDFA48B1012013F091FB10F084
:10488000A5FF0446069028B913F056FB012013B08B
:10489000BDE8F08F584E3378012BDDB24CD0022D9D
:1048A00063D0002D39D1042111F056FB012120469F
:1048B00011F080FA5149204611F0B0FA50492046D3
:1048C00011F092FA4F49204611F040FA4E49204625
:1048D00011F056FA0221204611F072FB4B49204696
:1048E00011F054FB2146684611F0B2FA484A0D9285
:1048F000484A0E924FF07C5300220CA920460C939C
:104900000F921092119311F0CFFA2946204611F020
:10491000EFFA0321204611F005FB069800243470BD
:1049200010F0EAFF0790002861D106A810F0BCFF44
:1049300007A811F06FF8A7E72946374D11F03AFAAA
:1049400020462E4911F06AFAA968204611F0FEF9B6
:10495000E968204611F014FA696A204611F044FA19
:10496000E96C204611F012FBD7E72B4D012111F025
:1049700021FAE969204611F051FA696A204611F0DE
:1049800033FAA968204611F0E1F9E968204611F0F0
:10499000F7F9A86CFDF768FD81B2204611F010FB15
:1049A000E96C204611F0F2FA2146684611F050FAFF
:1049B0002B6B0C936B6B0D93AB6B0E93EB6B0F939D
:1049C0002B6C10930CA96B6C1193204611F06CFAB0
:1049D000A86AFDF749FDC1B2204611F089FA286A9C
:1049E000FDF742FDC1B2204611F004FB95E711F03E
:1049F000A7F898B900204AE7701C00200000824206
:104A00009A99993FCDCC4C3F000020406666263FE6
:104A1000000020410AD7233C081C00200026DFF8B4
:104A200018A2864DDFF818924FF0210837460798F4
:104A300008A911F0DDF800282FD09DF820305BB1D7
:104A40000A993846FDF706FA099907463046FDF7F8
:104A500001FA0134E4B206469AF80030012B16D16F
:104A60002B880A9A9BB209EB03139A602B88099A48
:104A70009BB209EB03135A602B889BB25A1C92B26B
:104A8000802B2A8003D1FFF7F7FC00232B800F2017
:104A9000FDF790FFB8F10108C9D1079811F070F83F
:104AA000069D0121284611F085F90421284611F0C0
:104AB00053FA6449284611F0B1F96349284611F0C8
:104AC00093F96249284611F041F96149284611F0ED
:104AD00057F90221284611F073FA5E49284611F071
:104AE00055FA2946684611F0B3F95B4A0D925B4AC4
:104AF0000F924FF07C534FF07E520CA928460C9336
:104B00000E931092119311F0CFF90021284611F065
:104B1000EFF90321284611F005FA069907A810F0CD
:104B2000A3FF00283FF401AF079811F009F800280F
:104B30003FF460AF06A810F0B7FEDFF8FCB0DFF876
:104B4000FC80DFF8FCA04FF02109079808A911F0BC
:104B50004FF80546002837D09DF82D3073BB9DF8DF
:104B600020305BB10A993846FDF774F90999074678
:104B70003046FDF76FF90134E4B206469BF8003089
:104B8000012B1BD1B8F800300A9A9BB20AEB031331
:104B90009A60B8F80030099A9BB20AEB03135A6086
:104BA000B8F800309BB25A1C92B2802BA8F80020B3
:104BB00004D1FFF761FC0023A8F800300F20FDF7B7
:104BC000F9FEB9F10109C0D1254B012C94BF002297
:104BD00001221A701B7803F0FF0203B10122214861
:104BE000042103F077F820493846FDF73BFA0746E1
:104BF0002046FDF7E3F9044601463846FDF7E6FA9C
:104C0000194907463046FDF72DFA2146FDF7DEFA31
:104C1000164B1F60164B1860079810F0B1FF044642
:104C200007A810F0F7FE13F087F9002C3FF42EAE22
:104C300085F00100C0B22AE600010020061C002019
:104C400004140020000082429A99993FCDCC4C3F39
:104C5000000020406666263F00002041CDCC4C3E3F
:104C6000631C00200004004800007A445C1C002003
:104C7000581C002000B5ABB014230DF1060202A9A8
:104C8000ADF8063013F06CFB28B1BDF80610002318
:104C90009AB2914202D82BB05DF804FB02AA02EB53
:104CA000C30201331279002A08BF1046F0E710B59D
:104CB00086B010220021044602A8019129F0AEFE20
:104CC000FDF700FE13F0C4F88DF8040013F06AF944
:104CD000031E18BF012301218DF80530009013F049
:104CE0007FF9009813F01EFB009813F093F90098D9
:104CF000FFF7C0FF002840F09980684613F062F982
:104D000013F01AF9009813F0A1F9009813F0BAF90A
:104D10000098FFF7AFFF002840F08C80684613F042
:104D200051F913F009F9009813F0C8F9009813F03D
:104D3000E1F90098FFF79EFF00287FD1684613F045
:104D400041F913F0F9F8009813F0F0F9009813F016
:104D500079FA0098FFF78EFF002873D1684613F0A8
:104D600031F913F0E9F8009813F088FA009813F07D
:104D7000A1FA0098FFF77EFF002867D1684613F07C
:104D800021F913F0D9F8009813F0B0FA009813F055
:104D9000E9F90098FFF76EFF00285BD1684613F031
:104DA00011F913F0C9F8009813F0F8F9009813F00E
:104DB00011FA0098FFF75EFF00284FD1684613F004
:104DC00001F913F0B9F8009813F020FA009813F0E5
:104DD00039FA0098FFF74EFF002843D1684613F0D8
:104DE000F1F813F0A9F8009813F048FA009813F0BE
:104DF00061FA0098FFF73EFFC0BB684613F0E2F887
:104E000013F09AF8009813F071FA01238DF80F301F
:104E100001AB03CB206018686160A060684613F0A6
:104E2000D1F813F089F8002006B010BD01238DF8E9
:104E3000063067E701238DF8073074E701238DF80A
:104E4000083080E701238DF809308CE701238DF8C5
:104E50000A3098E701238DF80B30A4E701238DF881
:104E60000C30B0E701238DF80D30BCE701238DF83D
:104E70000E30C7E702480122102102F02BBF00BF0D
:104E80000004004802480022102102F023BF00BFA6
:104E90000004004810B50A4C23780BB9E37C6BB1D1
:104EA000FEF72EFB0038074B18BF0120400018709A
:104EB0001B78022B02BF00232370E37410BD00BFD8
:104EC000361F0020DC1C002038B5114C2378F3B9C4
:104ED000E37CE3B90F4D2B68012B07D92B68042B1A
:104EE00004D80D4A0421012000F07AFD2B68042B20
:104EF0000DD9FEF705FB0038084B18BF0120400014
:104F000018701B78022B02BF00232370E37438BD96
:104F1000361F0020D81C002020620308DC1C002063
:104F200010B5124C237863B101214FF0904002F08C
:104F3000CBFE0F4B0022187022701B780D4ADBB29B
:104F400013700D4C237863B102214FF0904002F0B2
:104F5000BBFE0A4B0022187022701B78084ADBB295
:104F60001370BDE81040FEF7EBBB00BF721C0020C1
:104F70004200002040000020711C00204100002061
:104F80003F00002010B5164B1A78022A26D91B784C
:104F9000082B23D8FFF768FC1248134A03781178CE
:104FA0005B1A124918BF01230B7003781048DBB25B
:104FB0001370104B104A1C780378E31A18BF0123B2
:104FC00013700E4B04701B7823B100230B700C4937
:104FD0000B701370BDE81040FEF7B2BB10BD00BFF0
:104FE0003E000020631C0020601C0020641C002088
:104FF000E8120020EA120020E9120020DC1C002048
:10500000651C002008B501214FF0904002F05CFEC5
:10501000064B012816BF022218701A701878044B2C
:105020001978BDE80840FEF7E9BA00BF0600002085
:105030000000002038B5324D324C287BFCF7BAFF17
:105040003149FDF70FF8A060687BFCF7B3FF2E49EC
:10505000FDF708F8E060A87BFCF7ACFF2A49FDF7F4
:1050600001F86062E87BFCF7A5FF2849FCF7FAFF2E
:10507000274BE0642361287CFCF79CFF6060687C20
:10508000FCF798FFA061A87CFCF794FFE061E87C46
:10509000FCF790FF2062287DFCF78CFFA062687D02
:1050A000FCF78CFF1849FCF7DDFF2063A87DFCF7B7
:1050B00081FF6063E87DFCF781FF1449FCF7D2FFB4
:1050C000A063287EFCF776FFE063687EFCF776FF3E
:1050D0000D49FCF7C7FF2064A87EFCF76FFF0A4963
:1050E000FCF7C0FF6064E87EFCF764FFA064287FE3
:1050F000FCF760FF074BE06202221A7038BD00BF68
:10510000B5000020081C0020CDCCCC3D0AD7233CA4
:10511000CDCCCC3E701C002038B5114D114C287BF5
:10512000FCF74CFF1049FCF79DFFA060687BFCF783
:1051300045FF0D49FCF796FFE060A87BFCF73EFFBA
:105140000949FCF78FFF6062E87BFCF737FF0749EE
:10515000FCF788FF064BE06401221A7038BD00BFDF
:10516000B5000020081C0020CDCCCC3D0AD7233C44
:10517000701C002070B52A4D2A4E2B7803702A4BE4
:105180001B784370044601214FF0904002F09CFDD3
:105190003378A070E37002214FF0904002F094FD4C
:1051A000224B20711B7863713378012B35D1204B52
:1051B0001868FDF759F91F4BE0801868FDF754F99E
:1051C00080B21D4BA0831B78191F4A424A41A27727
:1051D0001A4A92F82B1084F82B10D26AE262012B43
:1051E00084F8283007D1164B1B8884F82930154BDA
:1051F0001B8884F82A30144B1B7853B1134B1B685F
:105200003BB1134B1B78012B01BF124A23231370B0
:105210002B70114B01221A7070BD0020E080D0E786
:1052200006000020631C00203E000020621C0020BD
:105230005C1C0020581C0020EA120020781C002072
:10524000E2120020DE120020010100206C1C002070
:10525000331F002007000020D41C002008B5FFF7F2
:1052600009FEFFF7E7FE034A00231370024A13709A
:1052700008BD00BF701C0020311F002010B5104B6E
:105280001A78104BD2B25A700024012263211A708E
:1052900083F8331083F834209C63DC631C645C6403
:1052A0009C64DC641C655C6583F82B40DC625C629A
:1052B0009C77FFF7DFFDFFF7D1FF034B1C7010BD9C
:1052C0003E000020781C0020311F002008B5FFF7A9
:1052D00043F8BDE808406420FEF75ABC2DE9F041D0
:1052E00086B00D460446FFF7C5FD01F0F3FBFDF760
:1052F00027FE9620FEF74CFC154F00264FF00508C0
:10530000AE420FD14FF47A70FEF742FC01AB03CBF3
:105310001B8823810F4B2060002261601A7006B049
:10532000BDE8F081FEF71CFB87F80080FEF7FEF970
:105330004FF47A70FEF72CFC01A8FFF7B8FC41F29D
:105340008830FEF725FC0136FFF7C0FFD8E700BF25
:1053500006000020311F002013B50023044601A8D9
:10536000ADF80430FDF7B2FA30B19DF80430237087
:105370009DF805306370012002B010BD022801D8ED
:10538000FFF778BD7047022801D8FFF77BBD704753
:10539000022803D80248102102F0A1BC704700BFC8
:1053A0000004004807B568460FF0ACFE054B1B78BB
:1053B00003F0FF021BB9044B00999963DA6303B051
:1053C0005DF804FB03000020781C002007B5684648
:1053D0000FF098FE054B1B7803F0FF021BB9044B3E
:1053E000009919645A6403B05DF804FB02000020C0
:1053F000781C002007B568460FF084FE064A009B23
:105400001278012A01BF054A00219364D164044A3D
:10541000136003B05DF804FB631C0020781C0020BF
:10542000681C002008B5FEF7FFFABDE8084000F050
:10543000EFBC4FF0FF300FF01FBD7047014B012252
:105440001A707047401D002070470000014BD87053
:10545000704700BF50000020014B1874704700BF18
:1054600050000020002101200FF0CEBC10B50A4AE8
:105470000A4C42F21073002818BF03460848236004
:1054800013600FF09DFF2168054810F021F8BDE87A
:10549000104003480FF0E2BFF80000204C0000204D
:1054A000981E002010B5094C206023680BB9084BEA
:1054B000236008480FF084FF2168064810F008F8C0
:1054C000BDE8104003480FF0C9BF00BFF80000203E
:1054D000A0860100E01C002010B5094C2060236864
:1054E00013B942F21073236006480FF069FF216878
:1054F00004480FF0EDFFBDE8104002480FF0AEBFCA
:10550000FC000020F81C002010B5044688B190F97A
:10551000063073B910480FF053FF104B01221A7078
:10552000FEF712F80E4BE2791A700E4B1868FFF76F
:10553000B9FF0D4B0122002102201A700FF064FC0C
:1055400040F6B830FEF724FB08480FF087FFBDE8AF
:10555000104007480FF082BF441D002006000020C5
:10556000321F0020F8000020301F0020281D0020DE
:10557000F81C00200A460149FDF79CBC00F0030816
:1055800038B50C480FF01CFF06F0E8FC60B90A4C77
:105590000A480125257006F075FB2078294606F09B
:1055A000C9F804480FF05AFFBDE8384004480FF02E
:1055B00055BF00BF981E0020B400002050000020FE
:1055C000801E002006F07EBD30B599B0FEF75EFA71
:1055D000044606F0A9F9002841D101A8FFF7CAFD49
:1055E00054490B78042B544B3BD111221A70534A67
:1055F000107800F0FF0500283DD0002010700A78D8
:10560000042A33D112221A704D4A5968127862F076
:105610007F020A705A6820B200EB400000EB401095
:10562000FE21B0FBF1F0507002224649464C097849
:10563000012988BF00225A70637A33B106F060F9FD
:10564000012802D120460FF0BBFE404B3A48D978E2
:10565000002206F07FF9063001D106F04BF919B0AF
:1056600030BD0A78052AC2D11322BFE70A78052A7D
:10567000CAD11422C7E73648047804F0FF02002C90
:10568000D3D02F4A05701278586862F07F020270FA
:105690005A689DF8040050705A689DF80500907093
:1056A0000A78042A11D15A689DF80600D0705A6809
:1056B0009DF8070010715A689DF808005071062285
:1056C0000878052818BF0978AFE70A78052A2FD18E
:1056D0005A689DF80600D0705A689DF8070010714E
:1056E0005A689DF8080050715A689DF80900907139
:1056F000BDF80A205868120AC2715A68BDF80A003B
:105700001072BDF82000000A5072BDF8200090729F
:105710009DF82200D0729DF82C0010739DF82F0088
:1057200050730C98000A90730C98D0731022C7E73E
:105730000322C5E73E00002044000020301F002067
:105740008C1D0020DC1C0020441D00205000002087
:10575000D41C002013B568460FF0D4FC1A4B009AF5
:1057600019781A4B11B9996B511AD9631849DC6B26
:105770000878844281BF012083F82B00D86BD8625F
:105780001448007810B9186C101A58645C6C0878CA
:10579000844281BF012083F82B00586CD8620E48E8
:1057A0000078012802BF986C121ADA64D86C0A7863
:1057B000904205D9012283F83220DA6C92B21A861F
:1057C000064B1B7802B010BD03000020781C00209F
:1057D0000101002002000020631C0020EA120020CA
:1057E00020B1037813B102480FF038BE704700BFF4
:1057F000741D002008B5104B0122002102201A70F0
:105800000FF002FB0D480FF029FE0D4B1B788BB1FA
:105810000C4B1A7872B9DB7C63B90B4B1A68042AFB
:105820009EBF1A6801321A600021BDE808401020AE
:105830000FF0EABA08BD00BF301F0020E01C0020B6
:10584000321F0020361F0020D81C0020044B1B787C
:10585000022B03D1002108200FF0D6BA704700BFF9
:10586000B4000020044B1B78012B03D000218020C2
:105870000FF0CABA704700BF3E00002008B50021F3
:1058800040200FF0C1FA084B1B7863B1074B1A7820
:10589000012A08D10021022019700FF0B5FABDE8E5
:1058A0000840FFF7A7BD08BD321F0020641C002080
:1058B00008B506F05CFB80B906F022F801280CD18F
:1058C000BFF34F8F0549064BCA6802F4E0621343E9
:1058D000CB60BFF34F8F00BFFDE708BD00ED00E0D8
:1058E0000400FA0538B504460D4607484FF4006138
:1058F000FDF700FB30B92A4621460348BDE8384091
:10590000FDF7FEB938BD00BF00F0030838B5104CF4
:10591000237822781809D2B20CD10E4D2A78237838
:105920009A4206D020781E21FDF7DAFE2378DBB2FA
:105930002B7038BD084C23781E2133B1FDF7D0FE03
:10594000237883F001032370F3E702F00F00F5E7FB
:1059500006000020341F0020F5000020704770472B
:1059600070470000022810B504461CD040282AD0F9
:1059700001282BD1164B1B7843B3FA20FEF708F908
:1059800021464FF0904002F09FF9124B1870FFF73C
:1059900009FD002120200FF037FA00210220BDE888
:1059A00010400FF031BA0C4B1B787BB1FA20FEF798
:1059B000EFF821464FF0904002F086F9074B18703F
:1059C000FFF704FDE5E700210420E8E710BD00BF74
:1059D000721C002003000020711C00200200002027
:1059E00070B505460C46164605F09EFF034620B3EB
:1059F00070BD4A68F05CD0540133DAB2A242F8D3E9
:105A00000F4B0D701B78012B88BF00244C700D4C80
:105A1000637A33B105F074FF012802D120460FF0FC
:105A2000CFFC094B0948D978002205F093FF0630D6
:105A3000DED1BDE8704005F05DBF0449DDE700BF81
:105A4000DC1C0020441D00205000002044000020E9
:105A5000044B1B7823B9044A05210120FFF7C0BF7E
:105A6000704700BFDC1C00202562030810B500242D
:105A700090B03C22214601A8009428F0CFFF454B6E
:105A80002022DA7219788DF8001059788DF80110FB
:105A900099788DF80210D9788DF8031019798DF85E
:105AA000041059798DF8051099798DF80610D97977
:105AB0008DF80710197A8DF80810597A8DF80910A9
:105AC000997A8DF80A108DF80B2021460DF10B0202
:105AD00058180131007B02F8010F1429F8D193F80E
:105AE00020208DF8202093F821208DF8212093F894
:105AF00022208DF8222093F823208DF8232093F87C
:105B000024208DF8242093F825208DF8252093F863
:105B100026208DF8262093F827208DF8272093F84B
:105B200028208DF8282093F829208DF8292093F833
:105B30002A208DF82A2093F82B2093F828108DF82E
:105B40002B20154A19BB93F8291001F0FF00F1B979
:105B5000107093F82C206AB193F83F2052B10DF1E8
:105B60002B0100229818013290F82C0001F8010F47
:105B7000142AF7D109484FF40061FDF7BBF920B9A9
:105B8000064840226946FDF7BBF810B010BD012160
:105B90001170DEE7B50000200001002000F80308C6
:105BA000014940220FF024B900F8030838B5454CEC
:105BB000207963794D2BC0B26AD1C0EB0010800010
:105BC000A379E2790A2838BF0A204D2ADBB267D1CF
:105BD000C3EB03139B004FF47A7202FB03F594F8B6
:105BE0002C30002B64D194F83F30002B60D142F26E
:105BF0001070FFF73BFC344B1868FFF753FC237A17
:105C000032493348DBB20B70324B01221A70637A8F
:105C1000DBB2037094F827302F48DBB203700B78A7
:105C20002E49052B2E4B18BF00221A7094F82830ED
:105C30002C4A03EB83035B00DBB2137094F829302A
:105C4000294A03EB83035B00DBB2137094F82A301C
:105C5000264A0133DBB2DB01138094F82B30244A4F
:105C600003EB83035B00DBB213700023E21892F8AE
:105C70002C20D2B2CA540133142BF7D1A378012BB4
:105C80001FD1E37A202B1CD1BDE83840FFF7F6BACC
:105C90006379482B0ABF4FF46163637958438FE7F8
:105CA000E279482A0ABF4FF46162E279534392E7EE
:105CB0004FF47A735843FFF7F5FB2846FFF70CFCC7
:105CC0009DE738BDB5000020F80000203E00002010
:105CD000DC1C00200600002005000020361F0020EC
:105CE0000001002003010020020100203C000020F0
:105CF0000101002010B590B000213C2201A80091C4
:105D000028F08CFE4022404968460FF071F89DF85B
:105D100000203AB99DF80100072803D19DF8021030
:105D2000012909D0FFF7A2FE4FF47A70FDF730FF8A
:105D3000FFF73CFF10B010BD344B1A7058709970CB
:105D40009DF80310D9709DF8041019719DF8051085
:105D500059719DF8061099719DF80710D9719DF839
:105D6000081019729DF8091059729DF80A1099725D
:105D70009DF80B1001F03F01D9720DF10B0198183D
:105D8000013211F8014F0473142AF8D19DF8202034
:105D900083F820209DF8212083F821209DF82220DF
:105DA00083F822209DF8232083F823209DF82420C7
:105DB00083F824209DF8252083F825209DF82620AF
:105DC00083F826209DF8272083F8262083F82720B3
:105DD0009DF8282083F828209DF8292083F8292081
:105DE0009DF82A2083F82A209DF82B2083F82B2069
:105DF0000DF12B0100229818013211F8014F80F8A3
:105E00002C40142AF7D193E700F80308B5000020CE
:105E10001FB5002403A92046039406F08DF803A9BA
:105E2000012006F089F8434B4348009422464FF482
:105E3000FA710FF067FA414B4148009422464FF443
:105E4000FA710FF05FFA3F4B3F48009401224FF484
:105E5000FA710FF057FA3D4B3D48009401224FF480
:105E6000FA710FF04FFA3B4B3B480094012242F28B
:105E700010710FF047FA2046FCF73CFF08B1FDF720
:105E80005DF9364B009400224FF4FA6134480FF06C
:105E900039FA344A002101200FF072F8324A002109
:105EA00002200FF06DF8314A002104200FF068F84D
:105EB0002F4A002108200FF063F800F065FD2D49FE
:105EC0002D4805F0EFFF2D4805F0DCFE1E480FF0D1
:105ED000C5FA2B4B0021187805F02CFCFFF70AFFC0
:105EE000284A002110200FF04BF8274A00212020DB
:105EF0000FF046F8254A002140200FF041F8244ACF
:105F0000002180200FF03CF8224B23481968234BD6
:105F1000009401220FF0F6F9214B22481968224B18
:105F2000009401220FF0EEF91E480FF097FA04B02A
:105F300010BD00BF5F590008741D002061590008A2
:105F40005C1D002065580008441D00200D59000804
:105F5000281D002055570008101D00204D5800082E
:105F6000801E002089BA0008C9550008C5550008E0
:105F70008155000800000301680000205000002047
:105F8000B4000020C94E0008214F0008854F0008CA
:105F900005500008FC000020F81C00207D58000877
:105FA000F8000020E01C0020F557000838B5074D28
:105FB00000242C60FFF78AF9C820FDF7E9FD286866
:105FC0002146FCF7E3F90028F4D138BD741C002009
:105FD00030B50024A5B07C22214605A8049428F001
:105FE0001DFD53238DF81030012540F20713ADF845
:105FF0001230ADF800408DF81450FDF747FDFE2338
:10600000B0FBF3F000EB400000EB40108DF8150002
:106010006846FFF7A1F99DF800309DF80120134371
:1060200014D158238DF816300724802200212F48E0
:1060300028F0F4FC224604A92C4828F085FD2B4AC0
:1060400021460120FFF7CCFC25B030BD0E232946A8
:1060500001A8CDE901448DF81630ADF80C40FFF7EA
:106060003DF901AB03CB224C1B88CDF81B10ADF8DA
:106070001F30CDF81700FFF729F92068FCF7F4F975
:106080000A254FF47A7380B2B0FBF3F0B0FBF5F35E
:1060900005FB130030308DF821002068FCF7E4F98F
:1060A000642380B2B0FBF3F0B0FBF5F305FB130003
:1060B00030308DF822002068FCF7D6F980B2B0FBB2
:1060C000F5F0B0FBF5F305FB130030308DF823003D
:1060D0002068FCF7C9F980B2B0FBF5F305FB1300AB
:1060E00030308DF8240015249FE700BFB01E00203B
:1060F000741C0020F0B5044693B0B6480D468022CB
:1061000000210EF07FFE2378592B40F01C82052DD4
:1061100058D86378443B162B54D8DFE813F0650158
:1061200053004901530052015300530053005300E0
:10613000AC0053003801530053005300C301530017
:106140005300CD005300530053001700A578482D8D
:1061500011D1A14A14210120FFF742FC41F28830FD
:10616000FDF716FD40F6B830FDF712FD13B0BDE89F
:10617000F040FFF79DBB532D0DD1FFF729FF41F2F2
:106180008830FDF705FD934A1521012013B0BDE8C5
:10619000F040FFF725BC432D16D1002402A88DF84E
:1061A000084005F0E7FC8B4A4C23137007239370DB
:1061B0009DF80830547001204133D07013710521CF
:1061C000FFF70EFC13B0F0BD442DFBD1814C5923D9
:1061D00023705A236370A570FFF7E8FE7F22002129
:1061E000601C28F01BFC012607232570A370E670B5
:1061F0002671FDF74BFC794DFE23B0FBF3F000EB6D
:106200004000042300EB40106071A3712868FCF784
:106210002BF90A274FF47A7380B2B0FBF3F0B0FB8E
:10622000F7F307FB13003030E0712868FCF71CF926
:10623000642380B2B0FBF3F0B0FBF7F307FB13006D
:10624000303020722868FCF70FF980B2B0FBF7F00D
:10625000B0FBF7F307FB1300303060722868FCF7DF
:1062600003F980B2B0FBF7F307FB13003030A072E4
:1062700022460B2189E7A378303BDBB2092BA1D85A
:10628000574C584A23702378DBB25372514A592332
:1062900013704D2353702378032130330120937002
:1062A000FFF79EFBFFF7E2FB2378002B8AD013B0A9
:1062B000BDE8F040FDF792B9A578482D29D1454CAD
:1062C0005623182201252370002607236271684691
:1062D0000622A370A271E3716670E57025710EF05D
:1062E000EBFE009802A912380EF06EFF079B267293
:1062F0006C336372069B2B44A372059BE372049B71
:106300002373039B6373029BA37322460F212846CA
:1063100056E7432D7FF456AF00213C2203A82D4CB5
:10632000029128F07BFB02A8FFF73AFC9DF80830A9
:1063300063709DF80930A3709DF80A30E3709DF8F2
:106340000B3023719DF80C3063719DF80D30A371F3
:106350009DF80E30E3719DF80F30257023729DF883
:1063600013509DF8103063729DF81130A3722A46C5
:106370009DF81230E37205A904F10D00257328F091
:10638000E3FB05F10D012246C9B2012018E7A07810
:10639000392800F28E813038C0B2FEF7EFFF0D4A87
:1063A0002378137063785370A37893700321ECE61D
:1063B000A078392800F27D813038C0B2FEF7E3FFC3
:1063C000EDE7A078392800F274813038C0B2FEF7CA
:1063D000DFFFE4E7B01E00202B620308741C0020DE
:1063E000DC1C0020B5000020A378303BDAB2092A7B
:1063F00000F25F81E0783038C2B2092A00F2598198
:106400002179A1F14802D2B20B2A00F25281AB4DA0
:1064100045FA02F2D50700F14C810A224D2902FB10
:1064200003003AD13C2358434FF47A735843A44BAA
:106430001860A44B1860FFF735F8A34A237813704F
:1064400063785370A3789370E378D3700521237930
:1064500013710120FFF7C4FA9C4B00221A70072227
:106460005A7001229A70DA70A278303A02EB8201F7
:10647000E278303A02EB4102D2B21A7122795A71B3
:10648000934A1278D2B21A72924A1278D2B25A72DF
:1064900013B0BDE8F040FFF7E9BA4829C4D14FF482
:1064A0006163C0E7A278303AD3B2092B00F20181D0
:1064B000E378303BD9B2092900F2FB802079A0F1C2
:1064C0004801C9B20B2900F2F4807C4D45FA01F174
:1064D000C90700F1EE800A214D2801FB02332DD1BE
:1064E0003C2253434FF47A7253437B4A1360106843
:1064F000FEF7F2FF744A2378137063785370A37821
:106500009370E378D3700521237913710120FFF78D
:1065100067FA6E4B00221A7007225A7001229A7095
:10652000DA70A278303A02EB8201E278303A02EB7C
:106530004102D2B29A712279DA71A1E74828D1D109
:106540004FF46162CDE7502B40F08481022D7FF63D
:1065500039AE6178A1F13003012B3FF633AEA37859
:10656000312B7FF42FAE052D2DD1E378302B40F069
:10657000A080574A59480023137013781BB9237918
:10658000303BDBB20370534900230B70037854484F
:10659000DBB2037013784D4ADBB213720B78DBB2B7
:1065A0005372FFF763FA484B22781A7062785A7078
:1065B000A2789A70E278DA7022791A71FDF7C0F841
:1065C0000521414AE1E5082D67D1E378462B40F0EB
:1065D000FF802179A1F13000C0B2092800F2388192
:1065E0006279A2F13003092B00F23281A679A6F17B
:1065F0003003092B00F22C81E379A3F13005092D3A
:1066000000F2268101EB81014900364D203102EB79
:106610008202C9B25200297020323349D2B22F3ED1
:106620000A70F6B2314A03EB8303F6015B00168071
:1066300020332F4ADBB21370244A82F82800637992
:10664000303BDBB282F82930A3792F3BDBB282F8F2
:106650002A30E379303BDBB282F82B302B782BB930
:106660000B7803F0FF020BB9224B1A70FFF7FEF90B
:10667000154B22781A7062785A70A2789A70E27874
:10668000DA7022791A7162795A71A2799A71E27973
:10669000DA71FDF755F8082193E7042D54D1E2781B
:1066A000A2F13003DBB2092B29D9A2F14103192B46
:1066B00022D913B0BDE8F040FFF7CAB9DEF7FFFFFB
:1066C0004C000020F8000020B01E0020B500002083
:1066D0003E000020DC1C0020FC0000200400002004
:1066E0000600002003010020020100203C000020E1
:1066F0000101002000010020A2F13703DBB2734842
:106700000370734B20785970312199706F4918705C
:10671000DA700B786F4ADBB213720B78052B6E4B75
:106720000CBF0121002119706C4B1B78DBB2537236
:10673000FFF79CF9FDF704F84FF4FA60FDF728FA2B
:10674000FFF7B6F804213CE71D2D3ED9A51C002219
:10675000604E2846114610F8013F303BDBB2092B52
:1067600098BFB71802F1010294BF3B7301211E2AA2
:10677000F1D100299DD1FEF75DFC554B50221A70D6
:1067800000225A7007229A700122DA7003F8042F4F
:10679000203415F8012F03F8012FAC42F9D14D4BED
:1067A00000221A7007225A7001229A70DA70474A42
:1067B0001278D2B21A72494A1278D2B25A721E2292
:1067C000DA72FFF753F92321FBE6072D7FF671AF4D
:1067D000002240480234114614F8013F303BDBB23E
:1067E000092B98BF851802F1010294BF2B73012178
:1067F000082AF1D100297FF45CAFFEF78DFC344B01
:1068000050221A7007229A7000210122DA70597002
:1068100003F8042F2F4A50180131007B082900F19A
:10682000300003F8010FF6D10023137007235370D3
:1068300001239370D370254B1B78DBB21372274B67
:106840001B78DBB25372D172FFF710F90D21B8E655
:106850000021B6E6412B7FF4B5AC6378432B7FF47F
:10686000B1AC162D7FF4AEAC1D4D621C002312F8A6
:10687000011FE9540133142BF9D1FEF70BFB194B1F
:106880005B7D012B1DD113490023EA5CC81801333D
:10689000D2B2142B80F82C20F7D1104B00221A70A2
:1068A0001B78DBB24B72FFF7E1F8094A631E15341F
:1068B00013F8011F02F8011BA342F9D1044A162163
:1068C00063E4064B02221A70EFE700BF3E0000208F
:1068D000B01E0020B500002000010020DC1C0020BC
:1068E000361F00208407002037B504460D460029D6
:1068F00039D022480EF0B2FD2B78A3B39CB3606868
:10690000237880B3032B0DD0112B2ED0022B2AD14C
:106910006178012927D00B0625D403B0BDE83040AB
:10692000FFF7E8BB6378012B07D10078012802D07C
:10693000022800D008B905F0D7F800240DF10700AF
:106940008DF8074005F016F90D4A4C231370072304
:1069500093709DF807305470012041330521D070A9
:106960001371FFF73DF803B030BD6378012BFAD106
:106970000378044A03F001031370F4E75C1D002060
:10698000B01E00208C1D0020034B0022C3E9022210
:106990000122C3E9002270474C1F002000487047C5
:1069A0004C1F00204FF0B04382B0DA6C0243DA642F
:1069B000DB6C03400193019B02B070472DE9F0416D
:1069C00086B000240220154D0594FFF7EBFF04204C
:1069D000FFF7E8FF124F03944FF4807601230DEB8D
:1069E0000001CDE901632846032304934FF40058C6
:1069F00001F04AF801A93846CDF8048001F044F8C6
:106A000022464146384601F065F92846224631467D
:106A100001F060F9204606B0BDE8F08100040048AE
:106A200000080048032810B50ED8012810D868B90E
:106A300002460B484FF4807101F04CF900220948DE
:106A40004FF4005101F046F9002010BD0122F0E79B
:106A5000002203484FF4807101F03CF90122EEE777
:106A600000040048000800480220704700207047DA
:106A700001207047002814BF16200F207047000027
:106A80000D48854600F025F80C480D490D4A0023B5
:106A900002E0D458C4500433C4188C42F9D30A4AD3
:106AA0000A4C002301E013600432A242FBD328F019
:106AB0001DF8FCF725FBFEE7000001200000002088
:106AC000A005002090C80308A0050020783F002002
:106AD000FEE7704710B5032000F06EFC01F07CFA71
:106AE000064B18600F20FDF749F8044618B9FCF76B
:106AF0007DFC204610BD0124FBE700BF04010020FF
:106B00004FF0E022136923F00203136170474FF046
:106B1000E022136943F0020313617047014BD3F87D
:106B2000900570470070FF1F014BD3F89405704724
:106B30000070FF1F014BD3F8980570470070FF1FCE
:106B4000024A536823F0010353607047002004E0B9
:106B5000024A536823F0020353607047002004E0A8
:106B6000024A536823F0040353607047002004E096
:106B70008068C0F380007047F7B500230193044696
:106B8000002800F0E980856D25B9FBF743FFE56536
:106B900084F8545023689A68D00040F1A1809A6824
:106BA000D10000F1B480A26D42F01002A265E26D46
:106BB00042F00102E26501251846FFF7D9FFA26DF8
:106BC00002F01002024340F0C980A26D206922F455
:106BD000817242F00202A2659A68D2075DD4226BEC
:106BE000A67E94F82CC0003A18BF01221703D4E9FE
:106BF00002120A43217E42EA8132617E42EAC132B8
:106C000042EA4632002842EA4C02B4BF20F000417A
:106C10004FF400113A430A4394F82010012903D19C
:106C2000002E76D142F48032616A21B1A66A01F465
:106C3000E07131430A43D968E66C21F4FE3121F456
:106C4000FF711143D96094F83C206168012A01F07A
:106C5000404C4CEA060609D1D4E910273A433243A6
:106C6000A66C324342EA0C0242F001061F693E4A1A
:106C70003A4032431A6121F00042B2F1804F0CD009
:106C8000B1F1004F09D0394ED6F8082701F4701140
:106C900022F470120A43C6F808275A69666BA16B82
:106CA00022F0070232435A615A6922F0700242EA26
:106CB00001125A61002835D19A6A62F00F029A6275
:106CC0005B6903F007039E423CD10023E365A36D9B
:106CD00023F0030343F00103A365284603B0F0BD8E
:106CE0009A68234922F0104222F0170242F08052A3
:106CF0009A60204A1268B2FBF1F20132520001920E
:106D0000019A002A3FF44BAF019A013AF7E70025B8
:106D100052E7A16D41F02001A165E16D41F0010153
:106D2000E16581E7B0F5001FCAD19A6AE269013ACC
:106D300092006FF00F0102F01C0201FA02F2216EC4
:106D40000A43BCE7A36D23F0120343F01003A365CD
:106D5000E36D43F00103E3650125BEE7A36D43F056
:106D60001003A365F8E700BF02FCFF1F00200140ED
:106D7000400D030004010020F8B54569082D0446C4
:106D80000E460AD00368DB68D80705D5A36D43F02B
:106D90002003A3650120F8BD0425FCF7F1FE07469A
:106DA00023681A682A4220D0A26D42F40072A265BC
:106DB000DA6812F4406F14D1A27E92B91A681207F1
:106DC0000FD51846FFF7D4FE20BB5A6822F00C02FC
:106DD0005A60A26D22F4807222F0010242F0010298
:106DE000A265227EFAB10020D5E7711CD9D0FCF74C
:106DF000C7FEC01BB04201D8002ED1D123681B684A
:106E00002B40CDD1A26D84F8543042F00402A2652B
:106E10000320C0E7A26D42F02002A265E26D42F0BD
:106E20000102E265DDE70C221A60DCE70368186CFA
:106E300070470000F7B50023019390F85430012B00
:106E4000044600F0C08005680269012380F85430D0
:106E50002846FFF78DFE002840F0AF80D1E90030D2
:106E6000022822F004027ED0B2F1004FC3F3110ECB
:106E700035D1AA6A42EA0E02AA628A68686902EA01
:106E8000032222F07C4222F0FF0220EA03210A437F
:106E9000002B6A611DDA4D4A4D4DD2F80817AB42FE
:106EA00001F0E07043D10D0213D4D2F8083723F07B
:106EB000E073034343F40003C2F80837454B1A68F4
:106EC000454BB2FBF3F20C2302FB03330193019B0E
:106ED00053BB0020002384F8543003B0F0BD226E71
:106EE00000F01F074FF00F0C0CFA07FC6FEA0C06BE
:106EF00022EA0C0CBEF1000F11D1C3F38462BA4038
:106F000042EA0C0222668008E26901309042B4D85D
:106F1000A86AC3F38362BA4006403243ACE793FAEF
:106F2000A3F2B2FA82F2EAE7019B013BCEE72B4DD6
:106F3000AB420BD1C901CCD4D2F8083723F0E073AF
:106F4000034343F08073C2F80837C2E7244DAB42D5
:106F5000BFD14B02BDD4D2F8083723F0E07303430E
:106F600043F48003EFE7B2F1004F01BFAA6AC3F315
:106F700011018A43AA62002BABDA154813498342F8
:106F8000D1F8082709D1D1F8083702F0A07223F010
:106F9000E0731A43C1F808279BE71048834204D1E5
:106FA000D1F8083702F44002F1E70D48834290D14E
:106FB000D1F8083702F0C072E9E7A26D42F0200272
:106FC000A265184686E7022087E700BF002001403F
:106FD000001000B004010020400D0300004000B884
:106FE000002000B4026838B504461046FFF7C0FD23
:106FF00008B9002038BD9368990707D4936823F037
:10700000004323F0170343F010039360FCF7B8FD2F
:10701000054623689B685B07EBD5FCF7B1FD401B79
:107020000228F6D923689B685A07F2D5A36D43F06E
:107030001003A365E36D43F00103E3650120D9E785
:1070400073B50023026801939368DD07044602D5F7
:10705000002002B070BD9168214B194209D0A36D88
:1070600043F01003A365E36D43F00103E3650120E2
:10707000EFE7936823F0004323F0170343F0010385
:107080009360184BD3F8083718021CD4637E012B89
:10709000DED0FCF775FD144E054622681368DB0749
:1070A000D6D49368D9075FBF9368334043F0010398
:1070B0009360FCF765FD401B0228EED923681B682E
:1070C000DA07EAD4CBE7094B094A1B68B3FBF2F3B2
:1070D00001330193019B002BD8D0019B013BF8E7C2
:1070E0001700008000200140E8FFFF7F040100201E
:1070F000400D030038B504460068FFF739FD05462A
:1071000020BB94F85430012B20D0012384F8543054
:107110002046FFF795FFB0B9A36D226823F4706392
:1071200023F0010343F48073A3651C23E06513601F
:1071300084F85400936823F0004323F0170343F0CE
:107140000403936038BD84F85450FBE70220F9E74C
:10715000026838B5936891680446C80701D40020D6
:1071600038BD9907FBD4936803F00503012B19D1AF
:10717000936823F0004323F0170343F00203936066
:1071800003231360FCF7FCFC054623689B68DB07C0
:10719000E5D5FCF7F5FC401B0228F6D923689B686F
:1071A000DA07F2D5A36D43F01003A365E36D43F056
:1071B0000103E3650120D3E770B5044600284BD0F6
:1071C000836D43F002038365FFF70CFF054668B942
:1071D0002046FFF7BDFF054608B90123A3652268D5
:1071E000936823F0104323F01703936023685A68D1
:1071F00022F4677222F003025A6040F29F321A6052
:10720000D968164A0A40DA601A6922F040421A61C7
:107210005A6922F007025A611A6A02F0F0221A62D1
:107220005A6A02F0F0225A62DA6A02F0F022DA6256
:107230009A6A0B4A00269E62D2F8083723F0FE7342
:10724000C2F808372046FBF7F9FBE6652666A66517
:1072500084F85460284670BD0125FBE700023E8398
:107260000020014010B590F85430012B044615D091
:10727000012380F85430FFF7B5FE58B92046FFF7D8
:1072800067FF38B9A36D23F4807323F0010343F043
:107290000103A365002384F8543010BD0220FCE7ED
:1072A000F7B50023019390F85430012B04467FD0AA
:1072B000012380F85430FFF74BFF23689A6812F0DF
:1072C0000102054607D0A36D43F01003A365002318
:1072D00084F854302DE0A16D364F21F4817141F0D6
:1072E0000201A165DE68D96826F4FF4626F07C0617
:1072F00021F40041360421F00301360CD960082046
:107300009968394041F0004199609968002913DA81
:107310000199013101910199B1F52E3FF5D3A36D8A
:1073200023F0120343F01003A365002384F85430C4
:107330000125284603B0F0BDD3F8B410013801F0A0
:107340007F010A44DCD199681A48014041F00101EB
:107350009960D3F8B41021F07F0141EAD202C3F85A
:10736000B4209A68024042F002029A60FCF708FCDE
:10737000074623689A68D20708D4DA683243DA608D
:10738000A36D23F0030343F001039FE7FCF7F8FB31
:10739000C01B0228EDD923689B68D907E9D5A36DE6
:1073A00043F01003A365E36D43F00103E365BFE71A
:1073B0000225BEE7E8FFFF7F0749CA6822F4E062C2
:1073C0000302120403F4E063120C134343F0BF639F
:1073D00043F40033CB60704700ED00E0164B30B54E
:1073E000DC68C4F30224C4F10703251D042B28BF65
:1073F0000423062D4FF0FF358CBF033C002405FA13
:1074000003F321EA0303A54022EA0502A340002872
:1074100043EA0203ACBF00F16040084A4FEA03139D
:10742000B8BF00F00F00DBB2AABF00F561401354F3
:1074300080F8003330BD00BF00ED00E014ED00E047
:10744000002807DB044A4109012300F01F008340A4
:1074500042F82130704700BF00E100E000280CDB5B
:107460004309064900F01F0020330122824041F801
:107470002320BFF34F8FBFF36F8F704700E100E011
:1074800070B5D0E913456560446D14B1D0E9164577
:107490006560D0E9105404F01C060124B4406C600F
:1074A000046863608368102B0BBFA260A160E16079
:1074B000E26070BD0268416CD3B210B5083B142481
:1074C000B3FBF4F30B4CA24288BF0B4A21F003013B
:1074D00099BF01F1804202F50232521807338264EB
:1074E000064AC26403F01F03012202FA03F3036594
:1074F00010BD00BF070402401C0802408008024083
:1075000038B500285CD002682E4B9A424FF0140127
:107510004AD82D4B1344B3FBF1F32C499B00C0E92F
:107520001013022380F825301368056923F4FF4304
:1075300023F070031360D0E9024323432B434569D2
:1075400011682B4385692B43C5692B43056A2B437F
:107550000B431360FFF7AEFFB4F5804F04BF002369
:1075600043604368816C03F07F020A60D0E9131422
:10757000013B032B4C601ED8154B16498165134403
:107580009B000121013A01FA02F200214365C26524
:107590001960114B5A6400230122C36380F8243020
:1075A00080F82520184638BD0C4B1344B3FBF1F38B
:1075B0000B499B00B3E70023C0E91533C365EAE735
:1075C0000120F0E707040240F8FFFDBF0000024081
:1075D0003F8200104009024000090240F8FBFDBF55
:1075E0000004024038B5002841D00268136823F037
:1075F000010313601F4B9A424FF0140130D81E4B09
:107600001344B3FBF1F31D499B00C0E9101301249F
:1076100003F01C0304FA03F3002515604B60FFF729
:1076200049FF836C41681D60D0E913325A604A1EDD
:10763000032A06D8124B0B449B0094401D60114B4B
:107640005C640023C363C0E91533C0E90B33C0E9B0
:107650000D33C36580F8253080F82430184638BDD6
:10766000094B1344B3FBF1F308499B00CDE701201C
:10767000F5E700BF07040240F8FFFDBF000002402D
:107680003F82001000090240F8FBFDBF00040240E9
:1076900070B590F82450012D04463BD090F8256039
:1076A0000125AE4280F824504FF000062CD102256F
:1076B00080F825500568C6632E6826F001062E6006
:1076C000FFF7DEFE036BBBB12B6843F00E032B60AC
:1076D000A36C1A68D20342BF1A6842F480721A601F
:1076E000636D1BB11A6842F480721A602B6843F014
:1076F00001032B60002070BD2B6823F004032B6076
:107700002B6843F00A03E2E78023C36380F8246018
:107710002846F0E70220EEE7034640B190F8252026
:10772000022A06D00422C263002280F8242001200D
:1077300070470268806C116821F00E0111600168C9
:1077400021F480710160116821F001011160D3E919
:10775000100202F01C0101228A404260D3E9132189
:1077600051605A6D32B1116821F480711160D3E912
:10777000162151600122002083F8252083F824007F
:10778000704708B590F82530022B03D00423C3635B
:10779000012008BD03681A6822F00E021A601A68F8
:1077A00022F001021A60826C136823F48073136064
:1077B000D0E9101303F01C02012393404B60D0E981
:1077C00013325A60436D33B11A6822F480721A6022
:1077D000D0E916325A60012380F82530002380F862
:1077E0002430836B03B198470020D2E770B4426C19
:1077F000046C036826681D6802F01C020421914095
:1078000031420FD015F0040F0CD01A6892065EBFFB
:107810001A6822F004021A60036B6160002B33D0F7
:1078200070BC184702219140314217D015F0020F69
:1078300014D01A68940606D41A6822F00A021A6054
:10784000012280F82520114A93428CBF104B114B26
:107850005960002380F82430C36ADFE70821914093
:10786000314211D029070FD5196821F00E01196096
:10787000012303FA02F26260C36380F8253000231B
:1078800080F82430436BC9E770BC70478000024029
:1078900000040240000002400A4A536943F4802376
:1078A00030B55361EFF3108472B60023CD58C55044
:1078B0000433B3F5807FF9D11369DB03FCD484F37F
:1078C000108830BD00400058064B5A69002ABFBFDF
:1078D000054A9A6002F188329A60BABF5869C00FAF
:1078E000002070470040005823016745044B5A6947
:1078F00042F000425A615869C043C00F704700BF50
:107900000040005870B50546FCF73AF9124E04469F
:107910003369D90313D43369DA0744BF01223261D2
:107920004CF2FA32134011D10B4E306910F4802022
:107930000BD0FCF725F9001BA842F6D304E0FCF7B6
:107940001FF9001BA842E3D3032070BD024A136154
:10795000024A01205360F8E7004000585C1F0020F5
:107960002DE9F041184D98462B78012B06460C4620
:10797000174626D001232B704FF47A7000236B60DA
:10798000FFF7C0FFA0B9012E16D1104A536943F08A
:10799000010353612760BFF36F8FC4F804804FF475
:1079A0007A70FFF7AFFF094A536923EA0603536170
:1079B00000232B70BDE8F08139462046FFF76CFFAD
:1079C000EDE70220F6E700BF5C1F002000400058F2
:1079D000054A536923F47E7343EAC00040F48030C3
:1079E00040F0020050617047004000582DE9F0411E
:1079F000234F3B78012B054688463FD001233B703F
:107A00004FF47A7000237B60FFF77CFF044688B94F
:107A10002B68042B13D11B4A536943F4803343F082
:107A2000040353614FF47A70FFF76CFF0446154B63
:107A30001A681B6800233B702046BDE8F0814FF0B8
:107A4000FF33C8F800306E68D5E901321344B34201
:107A50000AD93046FFF7BCFF4FF47A70FFF752FFA8
:107A600050B1C8F800600446064A536923F47E7397
:107A700023F002035361DAE70136E5E70224DBE78E
:107A80005C1F0020004000582DE9F04F524C0023AD
:107A90004FF00F090A6832FA03F501D1BDE8F08F03
:107AA000012505FA03F818EA020200F08E804E68FC
:107AB000032706F003054FEA430E07FA0EFC6F1E7C
:107AC000012F6FEA0C0C32D8876807EA0C0ACF68DE
:107AD00007FA0EF747EA0A078760476827EA0808A7
:107AE000C6F300179F4047EA08074760C76807EAE0
:107AF0000C088F6807FA0EF747EA0807022DC760DF
:107B000017D14FEAD30800EB880803F0070AD8F82A
:107B100020704FEA8A0A09FA0AFB27EA0B0B0F6961
:107B200007FA0AF747EA0B07C8F8207001E0032DAF
:107B3000DCD1076805FA0EF507EA0C073D4316F499
:107B4000403F056041D023F0030707F1804707F568
:107B5000803703F0030CBD684FEA8C0C4FF0070E22
:107B60000EFA0CFEB0F1904F25EA0E0E2FD01B4DF1
:107B7000A8422ED005F58065A84214BF072502252E
:107B800005FA0CF545EA0E05BD602568D74316F4E5
:107B9000801F0CBF3D4015432560656816F4001F2B
:107BA0000CBF3D4015436560D4F8805016F4803F0B
:107BB0000CBF3D401543C4F88050D4F88450B60340
:107BC00054BF3D401543C4F88450013362E700259B
:107BD000D6E70125D4E700BF00080058000400489C
:107BE000374A2DE9F04F00234FF0010A4FF0070B01
:107BF0004FF00F0931FA03F401D1BDE8F08F0AFA12
:107C000003FC1CEA010654D023F0030404F1804471
:107C100004F5803403F00307A568BF000BFA07F8EA
:107C2000B0F1904F08EA050E45D0264DA84244D049
:107C300005F58065A8420CBF02250725BD407545A6
:107C400017D1D2F8805025EA0605C2F88050D2F844
:107C5000845025EA0605C2F88450156825EA060511
:107C60001560556825EA06055560A56825EA0805EA
:107C7000A560056803265C0006FA04F423FA06F6FC
:107C8000254300EB8606056003F00705376AAD0063
:107C900009FA05F527EA05073762856825EA04052C
:107CA0008560456825EA0C054560C56825EA040439
:107CB000C46001339EE70025C0E70125BEE700BF91
:107CC00000080058000400480369194214BF01204D
:107CD000002070470AB18161704781627047436933
:107CE00001EA030221EA030141EA0241816170478E
:107CF000044AD168014208B502D0D060FDF732FED7
:107D000008BD00BF00080058024A136843F480739E
:107D100013607047000400580D4B10B55B690C46AA
:107D200028B99A0507D500F027F820B110BD9B05AA
:107D300001D400F019F8074A1369012C23F0040359
:107D4000136101D130BFF1E740BF20BF20BFEDE795
:107D50000004005800ED00E0024B186800F4C06019
:107D6000704700BF00040058024A136843F4804380
:107D700013607047000400580C4A136823F48043D2
:107D800013600B4B1B6832214B430A49B3FBF1F3E1
:107D90005169890500D533B9536913F4007F14BFC5
:107DA000032000207047013BF2E700BF00040058A9
:107DB0000401002040420F000B4A136823F0070320
:107DC00043F002031360094B1A69012842F00402D0
:107DD0001A6105D130BF1A6922F004021A61704796
:107DE00040BF20BF20BFF6E70004005800ED00E0D0
:107DF0004FF0B0431868C0F3404070474FF0B043B5
:107E00001868C0F3400070474FF0B042536823F445
:107E10007F4343EA0023536070474FF0B043186834
:107E2000C0F34060704700007FB54FF0B0432C4A6C
:107E3000D3F80831C0F3031003F00F0352F82040C9
:107E4000284A52F82330B4FBF3F4FFF785FF264BA2
:107E5000054693E80700B5F5007F04AB03E907008A
:107E600010D0224B9C4218D303F5B70303F67F537F
:107E70009C4229D903F5741303F510639C4225D85D
:107E800002230BE01A4B9C4207D91A4B9C421BD988
:107E900003F5370303F5D853F0E7002304AA02EBF8
:107EA000830353F80C4C144D2B6823F00703234332
:107EB0002B60FBF765FE06462B6803F007039C4228
:107EC00006D1002004B070BD0123E7E70024EAE7F3
:107ED000FBF756FE801B0228EED90320F2E700BF15
:107EE00040620308A062030808200308C0CF6A00AC
:107EF000BFEA21013F933402004000584FF0B043E5
:107F000010B59A68D96812F00C0205D00C2A4AD133
:107F100001F00303012B51D14FF0B0412B480B6806
:107F200013F0080306D00B6813F0080337D1D1F81B
:107F3000941007E00C68240756BFD1F89430096804
:107F4000C3F3032350F82330002A0CBF1846002047
:107F50004FF0B0418A6802F00C020C2A1ED1CA68A8
:107F600002F00302022A2ED0032A06D10B68184A17
:107F700013F4801F174B18BF13464FF0B042D06860
:107F8000D168D268C0F306205843C1F3021301330D
:107F9000B0FBF3F0530F0133B0FBF3F010BD0B68EF
:107FA000C3F30313CEE7042A05D0082A06D11B68C1
:107FB00013F4801305D006480023C9E700231846B0
:107FC000C6E70448C4E7024BD7E700BF4062030896
:107FD0000024F4000048E80108B5FFF78FFF4FF0D8
:107FE000B043044A9B68C3F3031352F82330B0FB39
:107FF000F3F008BDA06203082DE9F0410446002813
:1080000053D04FF0B0439D68DE6803689B0605F0CF
:108010000C0506F0030668D5026A1DB10C2D46D189
:10802000012E44D1002A40D04FF0B043A16A1A6813
:10803000170756BFD3F894301B681B0903F0F003F1
:1080400099421FD90846FFF7EFFE00282DD14FF0C7
:10805000B042136843F0080313601368A16A23F069
:10806000F0030B431360606AFFF7CEFEFFF7B4FF27
:10807000AB4B1860AB4B1868FBF780FD002834D081
:10808000BDE8F0814FF0B042136843F0080313607D
:10809000136823F0F0030B431360606AFFF7B4FE2C
:1080A0000846FFF7C1FE0028E0D00120E8E74FF0C6
:1080B000B043002A54D01A6842F001021A60FBF75C
:1080C0005FFD0746FFF79AFE002842D04FF0B0420E
:1080D000136843F0080313601368A16A23F0F003E8
:1080E0000B431360606AFFF78FFE2368D80748D4FC
:1080F0002368990700F18C8023681E0740F1FA80FD
:10810000A3694FF0B046002B00F0E180D6F8943020
:10811000E16903F01002914200F0C48003F0030211
:10812000022AC2D0D80740F1B380D6F8943023F0A9
:108130000103C6F89430FBF723FD0746D6F89430C8
:10814000990740F1A580FBF71BFDC31B112BF5D947
:1081500004E0FBF715FDC01B0228B3D903208FE70D
:108160001A6822F001021A60FBF70AFD0746FFF7C2
:1081700045FE0028B9D0FBF703FDC01B0228F6D945
:10818000ECE7082D03D00C2D05D1032E03D1636835
:10819000002BADD189E74FF0B043A1681A6822F4F3
:1081A00080120A431A606268B2F5803F10D11A68E3
:1081B00042F480321A60FBF7E3FC0746FFF718FE33
:1081C000002895D1FBF7DCFCC01B6428F6D9C5E775
:1081D000B2F5041F04D11A6842F400121A60E6E7EF
:1081E000196821F480311960196821F400111960AF
:1081F000002AE0D1FBF7C4FC0746FFF7F9FD002891
:108200003FF476AFFBF7BCFCC01B6428F5D9A5E7AB
:10821000042D236903D00C2D0ED1022E0CD1002B7E
:108220003FF443AF4FF0B0426169536823F0FE431F
:1082300043EA016353605FE74FF0B046BBB1336878
:1082400043F480733360FBF79BFC074633685A05A1
:1082500005D4FBF795FCC31B022BF7D97EE77368A7
:10826000626923F0FE4343EA0263736044E73368C4
:1082700023F480733360FBF783FC074633685B05A8
:108280007FF53AAFFBF77CFCC31B022BF6D965E701
:108290004FF0B042E169D2F8943023F010030B4361
:1082A000C2F894304FF0B047D7F8943043F0010350
:1082B000C7F89430FBF764FC0646D7F894309A0769
:1082C00018D4FBF75DFC831B112BF6D946E7D6F8D3
:1082D000943023F00103C6F89430FBF751FC0746B5
:1082E000D6F894309B0705D5FBF74AFCC31B112B2E
:1082F000F6D933E72368580754D50B4F3B68D905A7
:1083000014D4FFF701FDFBF73BFC06463B68DA059A
:108310000CD4FBF735FC831B022BF7D91EE700BFFB
:10832000040100200801002000040058E3684FF019
:10833000B046002B58D023F08003052B02BFD6F89F
:10834000903043F00403C6F890304FF0B046FBF78E
:1083500017FCD6F8903043F001030746C6F890307A
:1083600041F28838D6F890309B0705D4FBF708FC1B
:10837000C31B4345F6D9F1E6E36823F00403812BE0
:108380001BD1FBF7FDFBD6F8903043F08003C6F815
:10839000903007464FF0B04641F28838D6F890301A
:1083A000180504D5E36A002B4AD1002068E6FBF7E4
:1083B000E7FBC01B4045F1D9D0E6FBF7E1FBD6F85F
:1083C000903023F08003C6F8903007464FF0B04657
:1083D00041F28838D6F890301905E3D5FBF7D0FB89
:1083E000C01B4045F6D9B9E6FBF7CAFBD6F890307A
:1083F00023F080030746C6F8903041F28838D6F85B
:1084000090301A0516D4FBF7BBFBD6F8903023F05A
:108410000103C6F8903007464FF0B04841F2883665
:10842000D8F890309B07BDD5FBF7AAFBC31BB3421E
:10843000F6D993E6FBF7A4FBC01B4045DFD98DE6D8
:108440000C2D4ED0022B4FF0B0431A6822F08072F0
:108450001A6033D1FBF794FB0546FFF7DEFC38BB0F
:10846000D4E90C314FF0B0420B43D0682D490140A4
:108470000B43E16B0B43216C0B43616C0B43A16B12
:1084800043EA0123D360136843F080731360D36819
:1084900043F08053D360FBF773FB0446FFF7BDFC4A
:1084A000002882D1FBF76CFB001B0A28F6D955E6A1
:1084B000FBF766FB401B0A28CFD94FE6FBF760FBB2
:1084C0000446FFF7AAFC30B94FF0B042164BD16812
:1084D0000B40D36069E7FBF753FB001B0A28F0D978
:1084E0003CE6012B3FF4E1AD4FF0B043D868236B7D
:1084F00000F003029A427FF4D8AD626B00F0700383
:1085000093427FF4D2ADA26B00F4FE43B3EB022F93
:108510007FF4CBAD636C00F06040C01A18BF01203F
:10852000AEE500BF8C80C111FCFFFEEE2DE9F041ED
:108530000D46044610B90120BDE8F081684E33684D
:1085400003F007038B4216D323689A0727D54FF011
:10855000B047A268BB6823F0F0031343BB60FBF78E
:108560000FFB0646BB68DB0319D4FBF709FB831B33
:10857000022BF7D911E0336823F007030B43336074
:10858000FBF7FEFA0746336803F00703AB42DBD084
:10859000FBF7F6FAC01B0228F5D90320CCE72368C5
:1085A000580617D54FF0B0476269D7F8083123F065
:1085B0000F0343EA1213C7F80831FBF7E1FA064646
:1085C000D7F80831D90305D4FBF7DAFA831B022B5D
:1085D000F6D9E2E723685A0713D54FF0B047E268AF
:1085E000BB6823F4E0631343BB60FBF7C9FA06469C
:1085F000BB689B0305D4FBF7C3FA831B022BF7D997
:10860000CBE72368180714D54FF0B0472269BB6841
:1086100023F4605343EAC203BB60FBF7B1FA06469A
:10862000BB68590305D4FBF7ABFA831B022BF7D9C0
:10863000B3E72368DA070FD4294C236803F0070354
:10864000AB4239D8FFF7C8FC264B1860264BBDE873
:10865000F0411868FBF792BA6268022A1DD1FFF751
:10866000C7FB00283FF467AF4FF0B04641F28838AF
:10867000B36823F003031343B360FBF781FA0746A3
:10868000B368626803F00C03B3EB820FD4D0FBF73E
:1086900077FAC01B4045F3D97FE7032A02D1FFF7E1
:1086A000BCFBDEE712B9FFF7A9FBDAE74FF0B043F6
:1086B0001B685B05D8D43EE7236823F007032B43F0
:1086C0002360FBF75DFA0646236803F00703AB421D
:1086D000B8D0FBF755FA801B0228F5D95DE700BF3B
:1086E00000400058040100200801002008B5FFF7F1
:1086F00073FC4FF0B043044A9B68C3F3022352F863
:108700002330D84008BD00BF8062030808B5FFF7DA
:1087100063FC4FF0B043044A9B68C3F3C22352F892
:108720002330D84008BD00BF806203084FF0B0433B
:10873000D3F89000C0F3400070474FF0B0410209F9
:10874000D1F8883002F47F22000123EA020300F40A
:108750007F200343C1F8883070474FF0B041020CCE
:10876000D1F88830120423EA020343EA0040C1F83A
:10877000880070470368DA0370B5044639D5FFF7FF
:10878000C3FAFBF7FDF9614E05463368DB0532D5C8
:108790004FF0B043616BD3F8902002F440729142E5
:1087A0001DD0D3F89010D3F8902042F48032C3F853
:1087B0009020D3F8902021F4407022F480328D076D
:1087C000C3F89020C3F8900009D5FBF7D9F941F21E
:1087D00088360546FFF7AAFF012840F090804FF049
:1087E000B042616BD2F8903023F440730B43C2F86F
:1087F0009030002605E0FBF7C3F9401B0228C4D9DE
:1088000003262568E8070AD54FF0B0416268D1F821
:10881000883023EA124392B21343C1F88830A90783
:108820000AD54FF0B041A268D1F8883023EA12434C
:1088300092B21343C1F88830AA0609D54FF0B0426E
:108840002169D2F8883023F440630B43C2F88830A2
:10885000AB0502D5206AFFF780FF680502D5606A84
:10886000FFF77BFF290502D5A06AFFF776FF6A06AE
:1088700002D56069FFF761FF2B0602D5A069FFF7FB
:108880005CFFE80502D5E069FFF757FFE90610D560
:108890004FF0B042E168D2F8883023F440730B43C4
:1088A000C2F88830B1F5807F02BFD36843F080738F
:1088B000D3602A040ED54FF0B042216BD2F8883035
:1088C00023F040430B43C2F8883019B9D36843F012
:1088D0008073D3606B0410D54FF0B042E16AD2F8D8
:1088E000883023F040530B43B1F1005FC2F8883069
:1088F00003D1D36843F48033D360304670BDFBF7B7
:108900003FF9401BB0427FF665AF79E7000400589D
:1089100030B590F82C30012B02464FF0020022D0E7
:10892000174B82F82D00CA24012582F82C505C6276
:1089300053245C62B1F5807F146B996914D121F4E2
:1089400088519961596C24F0010421F00041596467
:108950001463DD650A4BFF2159620020012382F870
:108960002D3082F82C0030BD21F408519961D96C6A
:1089700024F0020421F00041D9641463D865E9E7CA
:108980000028004070B50B4E036B756D1D40EA0763
:10899000044603D50123F365FBF77BFBAB0704D546
:1089A0000223F365204600F0C9F9012384F82D3035
:1089B00070BD00BF0028004038B50A4CE36823F0C2
:1089C0002003E360FBF7DCF80546E3689B0601D56E
:1089D000002038BDFBF7D4F8401BB0F57A7FF4D9FE
:1089E0000320F6E700280040F8B5114DEC6814F0BC
:1089F000400406461AD1EB6843F08003EB60FBF7B6
:108A0000BFF823460746EC6814F0400401D1032B5D
:108A100001D11846F8BDFBF7B3F8C01BB0F57A7F5B
:108A2000234684BF032386F82D30ECE70023F0E7CC
:108A30000028004038B50F4CE36823F08003E36062
:108A4000A3699B06054606D4FFF7B6FF10B10320C5
:108A500085F82D0038BDA36923F02003A361FFF73B
:108A6000ABFF10B1032085F82D00A36943F020036C
:108A7000A361EFE70028004038B5044600284BD03A
:108A800090F82D3003F0FF021BB980F82C20FAF784
:108A900091FB0223214D84F82D30EB68DB0636D4A0
:108AA000CA236B6253236B622046FFF79DFF10B110
:108AB000FF236B6238BDAB6923F08E6323F0400364
:108AC000AB6121696368AA690B431343A26913432D
:108AD000AB61D4E9022343EA02432B61D4E90931B3
:108AE000EA680B4322F4F8521343EB602046FFF789
:108AF000A1FF0028DCD1D4E90713AA690B4322F0B7
:108B00006042134362691343AB61FF236B6201232D
:108B100084F82D300020CDE70120CBE7002800406D
:108B20000023092803D840EA0310C0B270470A386E
:108B30000133C0B2F5E700002DE9F04790F82C3082
:108B4000012B05464FF0020069D0012385F82C3037
:108B50004E4B85F82D00DE6806F44076B6F5807F32
:108B600078D04C69087891F8019091F802A091F8BA
:108B70002470002A55D19B6913F0400308BFCB70C5
:108B8000FFF7CEFF80464846FFF7CAFF0246504631
:108B9000FFF7C6FF81463846FFF7C2FF0B6ACF7862
:108BA000234343EA875343EA090343EA084343EA7A
:108BB000022343EA0063354ACA20506253205062C0
:108BC0008C6A8869B4F5807F946945D124F488540F
:108BD00094610124D465B6F5807F09BFCB69136425
:108BE0000343536418BF5064284B4A681A672A6BC2
:108BF00042F001022A639A6942F488529A61244A37
:108C0000D2F8803043F40033C2F880301F4BFF228B
:108C10005A620020012385F82D3085F82C00BDE82C
:108C2000F087B4F1803F07D0B4F5000F04D09B6902
:108C300013F0400308BFCB700B6ACA781C4344EAA8
:108C40000A0444EA004343EA092343EA825343EA1D
:108C50000763B0E70023AEE724F4085494610224CC
:108C6000D465B6F5807F09BFCB6993640343D364B1
:108C700018BFD064054B4A685A672A6B42F002025B
:108C80002A639A6942F40852B8E700BF00280040FE
:108C90000008005890F82C20012A03464FF00200EB
:108CA00012D00A4A83F82D00CA2151625321516221
:108CB000916941F020019161FF2151620020012260
:108CC00083F82D2083F82C00704700BF0028004057
:108CD00090F82C20012A03464FF0020019D00D4ACB
:108CE00083F82D00CA2151625321516291690A48CB
:108CF00041F080019161D0F8801041F48021C0F8EA
:108D00008010FF2151620020012283F82D2083F87A
:108D10002C0070470028004000080058064B5A6D90
:108D2000520610B5044603D54022DA65FBF7B4F9C4
:108D3000012384F82D3010BD0028004070478900C1
:108D400001F1804101F531410A607047890001F16C
:108D5000804101F531410868704700002DE9F34773
:108D60001F46894690460446FAF70AFF0A9D3D448D
:108D70002D1AFAF705FF264B1E68C6F3CB366E4355
:108D8000824601962268936839EA03030CBF0123E7
:108D90000023434501D100202EE07B1CF3D0FAF7DD
:108DA000EFFEA0EB0A00A84229D323685A6822F0FC
:108DB000E0025A606268B2F5827F0AD1A268B2F519
:108DC000004F02D0B2F5806F03D11A6822F0400242
:108DD0001A60A26AB2F5005F07D11A6822F4005245
:108DE0001A601A6842F400521A60012384F85D3058
:108DF000002384F85C30032002B0BDE8F087019ABC
:108E0000019B002A03F1FF33019308BF1546B9E720
:108E1000040100202DE9F74F994600238DF8033017
:108E2000044688461746FAF7ABFE0C9D4D442D1AB2
:108E3000FAF7A6FE2C4BD4F800B01E6823235E433D
:108E4000360D6E43824601962268936803EA080352
:108E5000BB4201D100203AE0B8F5C06F07D137B965
:108E60009BF80C30DBB28DF803309DF80330B9F17C
:108E7000FF3FEAD0FAF784FEA0EB0A00A84229D30C
:108E800023685A6822F0E0025A606268B2F5827F75
:108E90000AD1A268B2F5004F02D0B2F5806F03D1BB
:108EA0001A6822F040021A60A26AB2F5005F07D188
:108EB0001A6822F400521A601A6842F400521A60CA
:108EC000012384F85D30002384F85C30032003B074
:108ED000BDE8F08F019A019B002A03F1FF33019353
:108EE00008BF1546B0E700BF0401002073B50B466C
:108EF00000920D4616464FF4C05100220446FFF77B
:108F000089FF024630B1236E43F02003236603201D
:108F100002B070BD00962B4680212046FFF71EFF51
:108F200002460028EFD100962B464FF4C061204640
:108F3000FFF770FF0028EBD0E5E74368B3F5827FC9
:108F4000F7B504460E4617460BD18368B3F5004FBC
:108F500002D0B3F5806F04D12268136823F0400378
:108F6000136000973346002280212046FFF7F6FE6B
:108F7000054628B1236E43F020032366032514E041
:108F80006368B3F5827F10D1A368B3F5004F02D0B8
:108F9000B3F5806F09D10097334600224FF4C061CA
:108FA0002046FFF737FF0028E4D1284603B0F0BD84
:108FB000F8B5044600287ED0436A002B50D14268A1
:108FC000B2F5827F00D0C36194F85D3003F0FF02F8
:108FD00023B984F85C202046FAF752F92268E06849
:108FE000022384F85D301368B0F5E06F23F040038E
:108FF00013604FF0000337D91D46B0F5706F18BFEE
:10900000A362A7686368A169A66A07F4044703F42A
:1090100082733B43276907F002073B43676907F008
:1090200001073B4301F400773B43E76907F038074A
:109030003B43276A07F080073B4306F400573B4356
:10904000B6F5005F136014D1236B8BBBB0F5E06FF6
:109050000DD902232363136843F40063136008E00F
:109060000023C0E90433AFE74FF48055C7E701237D
:109070002363636A676B03F0100307F0080700F4CB
:1090800070603B43090C034301F004010B432B4385
:10909000B6F5005F536004BFA38D1361D36923F459
:1090A0000063D36100200123206684F85D30F8BDA1
:1090B000022BDED1CFE70120F9E7000070B50446AE
:1090C00090F85C00012800F0CF80012084F85C005B
:1090D00094F85D0066680128C5B20AD0B6F5827FB3
:1090E00040F0C080A068002840F0BC80042D40F013
:1090F000B980002951D0002A4FD0002B4DD094F8D0
:109100005D00A16304281CBF052084F85D000020D9
:109110002066C4E91300A06AE387B0F5005F216808
:10912000A3872264A4F84430A4F8463007D1086825
:1091300020F400500860086840F400500860486857
:1091400020F4C0404860E068B0F5E06FA06D29D918
:109150004B6823F480534B6094F85D30434E444D8C
:10916000042B444B18BF1D46434B18BF3346C0E980
:109170000B35424B436300238363B4F846300C3114
:109180009BB2FEF785FA0346002848D0236E43F0D1
:1091900010032366012384F85D300120002384F846
:1091A0005C3070BD4D6845F480554D60656DAD69AE
:1091B000B5F5806F0AD113F0010F4B681ED123F46F
:1091C00080434B60E38FC3F34E03E3878369B3F5BA
:1091D000806FC1D14B6823F480534B60B4F84630A4
:1091E00013F0010F4B6811D123F400534B60B4F816
:1091F0004630C3F34E03A4F84630ADE743F4804352
:109200004B60E38FC3F34E030133DEE743F40053B7
:109210004B60B4F84630C3F34E030133EBE72268EA
:10922000606D516841F001015160C0E90B33C0E944
:109230000D33E38FA16B9BB20C32FEF729FA0028A5
:10924000A4D123681A6852065EBF1A6842F0400231
:109250001A605A6842F020025A605A6842F00202CC
:109260005A609BE7022099E702209AE7B59300082D
:109270008592000891920008BF9200089D92000814
:109280007047704708B5806AFFF7FBFF08BD70475D
:1092900008B5806AFFF7FBFF08BD7047806A026867
:1092A00008B5536823F003035360036E43F01003C3
:1092B0000366012380F85D30FFF7EFFF08BD7FB53F
:1092C000064600230393846A8DF80B30FAF758FCA6
:1092D00033681B689A06054668D42268536823F0F1
:1092E00020035360A36AB3F5005F13D101220090FD
:1092F000642311462046FFF731FD18B1236E43F079
:1093000002032366E3682668B3F5E06F2ED9F3689D
:109310000393039BA2682368002A43D16268B2F5D5
:10932000827F3FD15A6822F003025A6064212A46A4
:109330002046FFF702FE08B1202323660023A4F88D
:1093400046302268012384F85D309368DB0606D539
:10935000236E43F0020323664FF6EF739360236E90
:1093600023B32046FFF799FF04B070BD337BDBB217
:109370008DF80B309DF80B30236B022BCAD10122E4
:109380000095642311462046FFF7E8FC18B1236ED0
:1093900043F002032366337BDBB28DF80B309DF87C
:1093A0000B30B7E75A6822F00102BEE72046FFF70C
:1093B00067FFD9E77FB5064600230393846A8DF8DB
:1093C0000B30FAF7DDFB33681B68990605465ED45F
:1093D0002268536823F020035360A36AB3F5005F4B
:1093E0001BD1E368B3F5E06F3ED1236B012B3BD17A
:1093F000009064234FF400724FF4C0612046FFF7E1
:1094000009FD18B1236E43F00203236623681B7B1A
:10941000DBB28DF80B309DF80B302A4664212046D4
:10942000FFF764FD18B1236E43F020032366236821
:109430005A6822F003025A600022E287A4F846200C
:10944000012284F85D209A68D20606D5226E42F089
:10945000020222664FF6EF729A60236EBBB120467D
:10946000FFF71BFF04B070BD009564234FF48062CA
:109470004FF4C0612046FFF7CDFC18B1236E43F0D6
:10948000020323662368DB680393039BC5E720463A
:10949000F9F712FAE6E70000036830B559689A68F0
:1094A00002F04105012D85B0044606D14D0604D5D4
:1094B000C36C05B0BDE830401847950704D50806D1
:1094C00002D5236D2046F4E712F4B07F59D08D0603
:1094D00057D550060FD594F85D0003284FF00005CE
:1094E00049D0206E40F0040020660095D8680090B6
:1094F00098680090009895060CD5206E40F0010009
:1095000020660020029098680290186820F04000C1
:1095100018600298D00508D5226E42F00802226633
:10952000002203929A680392039A226E4AB35A6801
:1095300022F0E0025A60012284F85D208A0722D0DE
:109540005A68A06D22F003025A6040B1104B836349
:10955000FEF717F918B1236E43F040032366606DE0
:1095600078B10B4B8363FEF70CF950B1236E43F0D7
:109570004003236605E00195DA6801929B68019338
:10958000019B05B030BD2046FFF787FEF9E700BF1D
:109590009595000808B5806A0023A0F84630C38777
:1095A000FFF77BFE08BD0000034AD2F8903043F479
:1095B0000043C2F89030704700040058034AD2F8C4
:1095C000903023F40043C2F89030704700040058F4
:1095D000074B1A6822F040021A6040F441704FF4C1
:1095E000B85218605A601A6842F040021A60704718
:1095F0000000015837B5054600284ED0837903F0A6
:10960000FF046BB1032C0BD0254B4FF400629A6121
:109610002868FFF7DDFF002401232B71AC602FE0E9
:1096200000236B712846FAF7BFF91E4AD2F8903032
:1096300043F48053C2F89030002CE5D102234FF060
:10964000B042AB71D2F8943023F40043C2F89430A6
:10965000154B1B681C214B43DB0C64214B430193CE
:10966000019B93B90124AC60FFF79EFF0C4B9A68F5
:1096700042F400629A604FF400629A61002CC7D0F5
:109680000123AB71204603B030BD019B013B019328
:10969000D2F894305B04E3D4E6E70124F2E700BF9C
:1096A00000040058000800580401002037B5174D89
:1096B0002B6802461C204343DB0C642043431448C0
:1096C0000193019B93B901209060114C21732B6889
:1096D0001C214B43DB0C64214B430193019B6BB971
:1096E000012090600A4BDB6803B030BD019B013B59
:1096F000019383689C07E4D50020E6E7019B013BCA
:109700000193A368DB07E9D5ECE700BF0401002063
:109710000000015837B5184D2B6802461C20434302
:10972000DB0C6420434315480193019BA3B901203E
:109730009060124CFF2323732B681C256B43DB0CBA
:1097400064256B430193019B73B9012090600B4B1F
:10975000DB680B7003B030BD019B013B0193836854
:109760009C07E2D50020E4E7019B013B0193A3683D
:10977000DB07E8D5EBE700BF04010020000001583B
:109780000E4B0F491B681822534382B01B0D6422F5
:10979000534301934B69019AC3F3800322B9022317
:1097A0008360012002B07047019A013A01924A6930
:1097B000920701D5002BEDD10020F3E70401002032
:1097C0000004005807B50379012B0FD10A4B1B6821
:1097D000182253431B0C0193FFF7F0FE019B013B42
:1097E0000193019B002BF9D1FFF7DEFE03B05DF87A
:1097F00004EBFFF7C5BF00BF04010020F8B51E460B
:109800008379012B154604460F46DAB22DD14379F0
:10981000012B2AD0022342718371FFF7D3FF0D2160
:109820002046FFF7CBFEFFF741FF390A2046FFF73E
:109830003DFFF9B22046FFF739FF2E44B5420ED165
:109840002046FFF7B1FEFFF79BFFA0680123003819
:10985000A3714FF0000318BF01206371F8BD15F824
:10986000011B2046FFF722FFE8E70220F6E7F8B5E4
:109870001E468379012B154604460F46DAB22FD1D6
:109880004379012B2CD04271FFF79CFF1D2120460C
:10989000FFF794FEFFF70AFF390A2046FFF706FF9D
:1098A000F9B22046FFF702FF00212046FFF7FEFE37
:1098B0002E44B5420ED12046FFF776FEFFF760FF3B
:1098C000A06801230038A3714FF0000318BF0120E6
:1098D0006371F8BD29462046FFF71CFF0135E8E714
:1098E0000220F6E7F8B51F468379012B154604469A
:1098F0000E46DAB22CD14379012B29D04271FFF701
:1099000061FF06F0EF03A3F1840253425341237138
:1099100031462046FFF752FEFFF7C8FE2F44AF4204
:1099200010D1FFF741FE842E02D02046FFF728FF1A
:10993000A06801230038A3714FF0000318BF012075
:109940006371F8BD15F8011B2046FFF7AFFEE6E78F
:109950000220F6E7F8B51E468379012B154604462A
:109960000F46DAB227D14379012B24D04271FFF799
:1099700029FF39462046FFF721FEFFF797FE002119
:109980002046FFF793FE2E44B5420ED12046FFF746
:109990000BFEFFF7F5FEA06801230038A3714FF01E
:1099A000000318BF01206371F8BD29462046FFF768
:1099B000B1FE0135E8E70220F6E737B50023ADF840
:1099C000043001AA022312210546FFF7C3FFBDF8A8
:1099D0000440022364BA01AAA4B219462846FFF73C
:1099E00081FFE20702D528460AF094FFA30702D5BB
:1099F00028460AF095FF600702D528460AF0BAFF0C
:109A0000210702D528460AF0BBFFE20602D5284608
:109A10000AF0BCFFA30602D528460AF0A5FF60069F
:109A200002D528460AF082FF210606D514F480717B
:109A300018BF012128460AF07FFFA20502D528465B
:109A40000AF08AFF630402D528460AF0A5FF03B096
:109A500030BDF8B51E468379012B154604460F46E6
:109A6000DAB227D14379012B24D04271FFF7AAFE45
:109A70000E212046FFF7A2FDFFF718FE39462046CB
:109A8000FFF714FE2E44B5420ED12046FFF78CFDA1
:109A9000FFF776FEA06801230038A3714FF00003A2
:109AA00018BF01206371F8BD15F8011B2046FFF7B0
:109AB000FDFDE8E70220F6E7F8B51E468379012BA5
:109AC000154604460F46DAB22BD14379012B28D034
:109AD0004271FFF777FE1E212046FFF76FFDFFF76B
:109AE000E5FD39462046FFF7E1FD00212046FFF75E
:109AF000DDFD2E44B5420ED12046FFF755FDFFF7A0
:109B00003FFEA06801230038A3714FF0000318BF87
:109B100001206371F8BD29462046FFF7FBFD0135A2
:109B2000E8E70220F6E70000036A23F0010303627E
:109B3000036A70B5446882690D6822F4803222F0AD
:109B400073022A438D6823F002032B43124DA8426F
:109B500006D0124EB04203D0A6F58066B04214D1B2
:109B6000CE6823F008033343A84223F0040306D051
:109B70000B4DA84203D005F58065A84205D124F419
:109B80004075D1E9054634432C43446082614A68FC
:109B90004263036270BD00BF002C014000480140D9
:109BA00000440140036A23F480730362036A42683D
:109BB00070B5C4690D6824F4803424F073042C4318
:109BC0008D6823F4007343EA05230F4DA8420ED19C
:109BD000CD6823F4006343EA052323F48063D1E9CD
:109BE000055622F44052354342EA051206E0074D7D
:109BF000A842F4D005F58065A842F0D042604A68DA
:109C0000C461C263036270BD002C01400044014086
:109C1000036A23F480530362026A30B54468C3695F
:109C20000D6823F0807323F4E64343EA05238D682F
:109C300022F4005242EA05320A4DA84207D005F547
:109C4000C055A84203D005F58065A84204D14D69EE
:109C500024F4804444EA85144460C3614B6803647F
:109C6000026230BD002C0140036A23F4803303629A
:109C7000026A30B54468436D0D6823F4803323F0E5
:109C800070032B438D6822F4003242EA05420B4DEB
:109C9000A84207D005F5C055A84203D005F5806558
:109CA000A84204D14D6924F4803444EA0524446078
:109CB00043654B688365026230BD00BF002C0140E4
:109CC000036A23F480130362026A30B54468436D6B
:109CD0000D6823F0807323F4E04343EA05238D6885
:109CE00022F4001242EA05520A4DA84207D005F5B7
:109CF000C055A84203D005F58065A84204D14D693E
:109D000024F4802444EA8524446043654B68C36599
:109D1000026230BD002C0140704710B5846A626A4F
:109D200082420BD101232377D2690AB984F83E30ED
:109D30002046F9F70DFE0023237710BDA36A834266
:109D400008D102222277DB69002BF1D1012384F8AC
:109D50003F30EDE7E36A834208D104222277DB69D2
:109D6000002BE5D1012384F84030E1E7236B8342E7
:109D7000DED108222277DB69002BD9D1012384F8B8
:109D80004130D5E7704710B5846A636A834207D1D2
:109D9000012323772046FFF7F5FF0023237710BD2B
:109DA000A36A834201D10223F3E7E36A834201D12C
:109DB0000423EEE7236B8342ECD10823E9E77047E5
:109DC00010B5846A636A834209D10123237784F83A
:109DD0003E302046FFF7F3FF0023237710BDA36A30
:109DE000834205D102232377012384F83F30F0E733
:109DF000E36A83424FF0010304D10422227784F8FE
:109E00004030E6E7226B824203BF0822227784F8C3
:109E1000413084F83D30DCE71A4A0368904210B5BF
:109E200002D0B0F1804F09D14C6823F0700390420A
:109E300043EA040309D0B0F1804F06D0124A9042A1
:109E400003D002F58062904203D1CA6823F44073C4
:109E500013434A6923F08003134303608B68C36292
:109E60000B688362074B984207D003F5C0539842B2
:109E700003D003F58063984201D10B69036301238A
:109E8000436110BD002C01400044014010B5044660
:109E900050B390F83D3003F0FF021BB980F83C202E
:109EA000F9F73CFF0223206884F83D30211DFFF7BD
:109EB000B3FF012384F84830002084F83E3084F852
:109EC0003F3084F8403084F8413084F8423084F8E0
:109ED000433084F8443084F8453084F8463084F8C0
:109EE000473084F83D3010BD0120FCE710B5044632
:109EF00050B390F83D3003F0FF021BB980F83C20CE
:109F0000FFF70AFF0223206884F83D30211DFFF788
:109F100083FF012384F84830002084F83E3084F821
:109F20003F3084F8403084F8413084F8423084F87F
:109F3000433084F8443084F8453084F8463084F85F
:109F4000473084F83D3010BD0120FCE7036A23F060
:109F500010030362036A426870B584690D6824F0D7
:109F6000807424F4E64444EA05248D6823F0200339
:109F700043EA05130F4DA8420ED1CD6823F08003AC
:109F800043EA051323F04003D1E9055622F4406269
:109F9000354342EA850206E0074DA842F4D005F5B4
:109FA0008065A842F0D042604A688461826303629F
:109FB00070BD00BF002C01400044014038B590F84E
:109FC0003C30012B044673D001200C2A84F83C005D
:109FD0004ED008D8042A2BD0082A39D0BAB1002391
:109FE00084F83C3038BD102A52D0142AF7D12068AA
:109FF000FFF766FE436D0A6943F400634365436DF2
:10A0000023F480634365436D43EA02234EE02068F6
:10A01000FFF78AFD83690A6943F008038361836956
:10A0200023F0040383618369134383610020D6E72F
:10A030002068FFF78BFF83690A6943F4006383613B
:10A04000836923F480638361836943EA0223ECE735
:10A050002068FFF7A7FDC3690A6943F00803C361DD
:10A06000C36923F00403C361C3691343C361DDE71C
:10A070002068FFF7CDFDC3690A6943F40063C3613B
:10A08000C36923F48063C361C36943EA0223EDE734
:10A090002068FFF7E9FD436D0A6943F00803436553
:10A0A000436D23F004034365436D13434365BDE7EC
:10A0B000022097E710B584680A4324F47F4442EAFB
:10A0C00003222243826010BD38B590F83C30012B4A
:10A0D00004464FF0020000F0958084F83D00012214
:10A0E000206884F83C208568474B2B4083600B68D0
:10A0F000602B54D037D8402B6BD019D8202B0DD0E3
:10A100000AD833F0100109D0012384F83D30002330
:10A1100084F83C30104638BD302BF5D1826822F4EB
:10A12000401222F070021A4342F0070282602BE0D4
:10A13000502BE9D14A68CD68016A036A23F0010314
:10A140000362836921F00A0123F0F00343EA051357
:10A150000A4383610262836823F4401323F070038F
:10A1600043F057030FE0B3F5805F0DD0B3F5005F08
:10A170000CD0702BC8D1CB68D1E90121FFF79AFF31
:10A18000836843F0770383600022BDE7CB68D1E9A1
:10A190000121FFF78FFF836843F48043F3E7036AED
:10A1A0004D68C96823F0100303628269036A22F4D0
:10A1B000704223F0A00343EA051342EA01328261B0
:10A1C0000362836823F4401323F0700343F06703B2
:10A1D000D9E74A68CD68016A036A23F00103036284
:10A1E000836921F00A0123F0F00343EA05130A43CF
:10A1F00083610262836823F4401323F0700343F009
:10A200004703C0E7024685E78800CEFF036A01F0F6
:10A210001F0110B501248C4023EA04030362036A82
:10A220008A401A43026210BD38B50D46082D044617
:10A2300011461BD005D85DB1042D14D094F843000D
:10A2400008E00C2D15D0102DF8D190F8420001E057
:10A2500090F83E00A0F1020CDCF1000040EB0C0095
:10A2600050B1022076E090F83F00F3E790F840000C
:10A27000F0E790F84100EDE7082D1AD007D86DB14E
:10A28000042D13D094F84320012A19D00CE00C2D92
:10A2900027D0102DF6D194F842000CE094F83E201F
:10A2A000501E424242415AB9012053E094F83F20E7
:10A2B000F6E794F84000421E504250410028F3D087
:10A2C0000029F1D0002BEFD0082D4FF0020256D01C
:10A2D0000AD885B1042D3ED0042D84F84320E3D163
:10A2E0003BE094F84100E6E70C2D5CD0102DF3D153
:10A2F00084F84220D8E7606A84F83E203A4AC26275
:10A300003A4A02633A4A426322683432FDF7C0F99E
:10A310000028C9D12268D36843F400732068D36051
:10A3200029460122FFF772FF324A904250D0324B49
:10A3300098424DD003F58063984249D0B0F1804FE8
:10A340004DD182682D4B1340062B02D0B3F5803FD0
:10A3500045D1002038BD84F83F20A06A224AC2625D
:10A36000224A0263224A426322683832FDF790F99A
:10A37000002899D12268D36843F48063CEE7E06A6D
:10A3800084F84020184AC262184A0263184A42639D
:10A3900022683C32FDF77CF9002885D12268D36819
:10A3A00043F40063BAE7206B84F841200E4AC2628E
:10A3B0000E4A02630E4A426322684032FDF768F992
:10A3C00000287FF471AF2268D36843F48053A5E777
:10A3D000436C904243F400434364B2D0AEE7036859
:10A3E00043F001030360B4E71B9D0008879D00084C
:10A3F000C19D0008002C01400044014007000100FD
:10A40000FFF712BF082938B504460D464FD004D8CF
:10A4100061B1042944D0012038BD0C29FBD1026868
:10A42000006BD36823F48053D36005E00268406A70
:10A43000D36823F40073D360FDF7A3F920680022EA
:10A440002946FFF7E3FE2A4B984207D003F5C05395
:10A45000984203D003F5806398420DD1026A41F21D
:10A4600011131A4208D1026A40F244431A4202BF51
:10A47000436C23F400434364026A41F211131A420D
:10A4800008D1026A40F244431A4202BF036823F033
:10A490000103036001238DB984F83E300020BBE73F
:10A4A0000268806AD36823F48063D360C4E70268DB
:10A4B000C06AD36823F40063D360BDE70C2D13D0CA
:10A4C00007D8042D0AD0082D0BD0012384F843307F
:10A4D000E4E7102DF9D184F84230DFE784F83F300B
:10A4E000DCE784F84030D9E784F84130D6E700BF94
:10A4F000002C0140FFF786BF70B590F83C30012B6F
:10A5000002464FF0020020D082F83D000F4D106847
:10A5100043688468A84202BF4E6823F47003334343
:10A520000E6823F070033343A842436002D0B0F1B9
:10A53000804F04D1896824F080030B43836001239A
:10A54000002082F83D3082F83C0070BD002C0140B4
:10A5500010B590F83C30012B02463BD0CB688868A0
:10A560001D4C23F440730343486823F48063034382
:10A57000086823F400630343086923F4805303430A
:10A58000486923F400530343086B23F480430343D7
:10A59000886923F4702343EA00431068A04214D171
:10A5A000CC6923F0805323438C6A23F4700343EA7D
:10A5B00004530C6A23F0807323434C6AC96A23F066
:10A5C0000073234323F000530B434364002082F8BD
:10A5D0003C0010BD0220FCE7002C0140026852E85C
:10A5E000003F23F0C00342E8003102680029F5D1A2
:10A5F00002F1080353E8003F23F4000302F1080CC2
:10A600004CE800310029F3D12023C0F8883070478E
:10A6100010B5026852E8003F23F4907342E800311D
:10A6200002680029F5D10F4C02F1080353E8003FFE
:10A63000234002F1080C4CE800310029F4D1C36E2C
:10A64000012B07D152E8003F23F0100342E800310C
:10A650000029F7D12023C0F88C300023C36643675C
:10A6600010BD00BFFEFFFFEFF8B504461346D4F857
:10A670008850202D32D1F1B1EAB1E06FA4F8562014
:10A68000A4F8542000262122C4F890602165C4F863
:10A690008820226888B1124FC762124F0763124F99
:10A6A0002832C0E90D76FCF7F3FF30B11023C4F86F
:10A6B0009030C4F888500120F8BD236840221A6207
:10A6C000226802F1080353E8003F43F0800302F1DF
:10A6D000080141E800300028F3D1EDE70220EBE764
:10A6E000EDA6000835A7000841A7000808B50346F5
:10A6F000806A1B681B6813F0200317D1A0F856303E
:10A70000026802F1080353E8003F23F08003083297
:10A7100042E8003102680029F2D152E8003F43F0DC
:10A72000400342E800310029F7D108BDF9F7E8FD00
:10A73000FBE7704708B5806AFFF7FBFF08BD70476D
:10A74000806A38B50468D0F88830D0F88C50A26898
:10A75000120606D5212B04D10023A0F85630FFF7AE
:10A760003DFFA3685B0606D5222D04D10023A0F887
:10A770005E30FFF74DFFD0F8903043F01003C0F883
:10A780009030FFF7DCFF38BD08B5806A0023A0F8E1
:10A790005E30A0F85630FFF7D2FF08BD70470000CA
:10A7A0000368D9691A682DE9F04140F60F06314275
:10A7B0009D68044610D18E0640F1978002F0200675
:10A7C00005F080573E4300F09080436F002B00F06F
:10A7D0008580BDE8F0411847AB4EAC482E40104094
:10A7E000304300F08280CF0709D5D00507D501207E
:10A7F0001862D4F8900040F00100C4F890008F0770
:10A8000009D5E80707D502201862D4F8900040F077
:10A810000400C4F890004F0709D5E80707D50420C5
:10A820001862D4F8900040F00200C4F890000F07BE
:10A830000BD502F02000304307D008201862D4F86E
:10A84000900040F00800C4F890000E050AD55001B1
:10A8500008D54FF400601862D4F8903043F020031C
:10A86000C4F89030D4F89030002B37D08B0609D53F
:10A8700002F0200205F080552A4303D0636F0BB12C
:10A88000204698472668D4F89020B36802F0280242
:10A8900003F0400353EA0205204621D0FFF7B8FE3B
:10A8A000B3685F0617D5226802F1080353E8003F3A
:10A8B00023F04003083242E800310029F3D1D4F8F4
:10A8C000800040B1724B8363FCF75BFF30B1D4F87A
:10A8D0008000836B7DE72046FFF731FFBDE8F08104
:10A8E000FFF72DFFC4F89050F8E7E06E012840F024
:10A8F0008980CE0640F18680D00640F18380102208
:10A900001A629A6851064BD5D4F8802011684A68BB
:10A9100092B2002AE2D0B4F85C009042DED9A4F8EA
:10A920005E200A6892062FD453E8002F22F480722A
:10A9300043E800210029F7D103F1080252E8002F73
:10A9400022F0010203F1080040E800210029F3D1C0
:10A9500003F1080252E8002F22F0400203F1080040
:10A9600040E800210029F3D12022C4F88C20E166C0
:10A9700053E8002F22F0100243E800210029F7D10C
:10A98000D4F88000FCF7C8FE02232367B4F85E30D9
:10A99000B4F85C10C91A89B22046FFF7FFFE9DE7A4
:10A9A000B4F85E20B4F85E00B4F85C1080B292B2E5
:10A9B000002893D0891A89B200298FD053E8002F3C
:10A9C00022F4907243E800200028F7D1314D03F1C2
:10A9D000080252E8002F2A4003F1080646E800204A
:10A9E0000028F4D12022C4F88C206067E06653E888
:10A9F000002F22F0100243E800200028F7D10223A4
:10AA00002367C9E7CF0209D56E0207D54FF480123C
:10AA100020461A62BDE8F04100F0A0BD08060BD543
:10AA200002F0800005F40005284305D0A36F002B39
:10AA30003FF454AF2046CCE64F0611D556060FD54D
:10AA400053E8002F22F0400243E800210029F7D10B
:10AA50002023C4F88830A1672046F9F751FC3DE770
:10AA60000D0206D5500004D52046BDE8F04100F0A7
:10AA700077BDCB017FF532AF002ABFF62FAF20465E
:10AA8000BDE8F04100F06BBD0100001020010004A2
:10AA900089A70008FEFFFFEFD0F88C20B0F8601007
:10AAA000222A08B5036855D15B6A826D0B4013708A
:10AAB000836D01338365B0F85E30013B9BB2A0F833
:10AAC0005E30B0F85E309BB2002B42D1026852E893
:10AAD000003F23F4907342E8003103680029F5D168
:10AAE00003F1080252E8002F22F0010203F1080CE2
:10AAF0004CE800210029F3D12022C0F88C20184A0C
:10AB000041679342016705D1C26E012A0ED0F9F761
:10AB100005FC1EE05A681102F6D553E8002F22F01A
:10AB2000806243E800210029F7D1EDE70022C266E8
:10AB300053E8002F22F0100243E800210029F7D14A
:10AB4000DA69B0F85C10D20644BF10221A62FFF72F
:10AB500025FE08BD9A6942F008029A61F9E700BF34
:10AB600000800040D0F88C20B0F86010222A08B590
:10AB7000036852D15A6A1140826D22F8021B826525
:10AB8000B0F85E20013A92B2A0F85E20B0F85E20E4
:10AB900092B2002A40D153E8002F22F4907243E889
:10ABA00000210029F7D103F1080252E8002F22F01A
:10ABB000010203F1080C4CE800210029F3D1202206
:10ABC000C0F88C20174A41679342016705D1C26ED5
:10ABD000012A0ED0F9F7A2FB1EE05A681102F6D541
:10ABE00053E8002F22F0806243E800210029F7D1CA
:10ABF000EDE70022C26653E8002F22F0100243E87E
:10AC000000210029F7D1DA69B0F85C10D20644BF00
:10AC100010221A62FFF7C2FD08BD9A6942F00802CD
:10AC20009A61F9E7008000402DE9F84F0368B0F819
:10AC30006060D3F81CB01F689D68D0F88C20222A71
:10AC4000044640F0B980B0F8683043B1DFF8749141
:10AC5000DFF874A14FF000081BF0200F20D1B4F8EA
:10AC60005E309BB2D3B1B4F868209A4216D92268FC
:10AC700002F1080353E8003F23F08053083242E812
:10AC8000003122680029F2D1504B636752E8003F3F
:10AC900043F0200342E800310029F7D1BDE8F88FE6
:10ACA0002368A26D5B6A33401370A36D0133A36503
:10ACB000B4F85E30013B9BB2A4F85E302368D3F851
:10ACC0001CB01BF0070F2ED01BF0010F09D0F905A7
:10ACD00007D501221A62D4F8902042F00102C4F88C
:10ACE00090201BF0020F09D0EA0707D502221A6252
:10ACF000D4F8902042F00402C4F890201BF0040F16
:10AD000009D0E80707D504221A62D4F8903043F03E
:10AD10000203C4F89030D4F8903023B12046FFF7F6
:10AD20000EFDC4F89080B4F85E309BB2002B93D136
:10AD3000226852E8003F23F4807342E80031236820
:10AD40000029F5D103F1080252E8002F02EA0902B6
:10AD500003F1080040E800210029F3D120225345E7
:10AD6000C4F88C20616721670AD05A68110207D5A0
:10AD700053E8002F22F0806243E800210029F7D138
:10AD8000E26E012A14D10022E26653E8002F22F07D
:10AD9000100243E800210029F7D1DA69B4F85C1009
:10ADA000D20644BF10221A622046FFF7F7FC53E791
:10ADB0002046F9F7B3FA4FE79A6942F008029A6120
:10ADC0006CE700BFFEFFFFEF0080004099AA00087B
:10ADD0002DE9F84F0368B0F86060D3F81CB01F6825
:10ADE0009D68D0F88C20222A044640F0B780B0F845
:10ADF000683043B1DFF87091DFF870A14FF00008C0
:10AE00001BF0200F20D1B4F85E309BB2D3B1B4F860
:10AE100068209A4216D9226802F1080353E8003FDD
:10AE200023F08053083242E8003122680029F2D131
:10AE30004F4B636752E8003F43F0200342E8003184
:10AE40000029F7D1BDE8F88F2368A26D596A314017
:10AE500022F8021BA265B4F85E20013A92B2A4F86F
:10AE60005E20D3F81CB01BF0070F2ED01BF0010F93
:10AE700009D0F90507D501221A62D4F8902042F0D2
:10AE80000102C4F890201BF0020F09D0EA0707D591
:10AE900002221A62D4F8902042F00402C4F89020F2
:10AEA0001BF0040F09D0E80707D504221A62D4F872
:10AEB000903043F00203C4F89030D4F8903023B1BE
:10AEC0002046FFF73CFCC4F89080B4F85E309BB29B
:10AED000002B95D1226852E8003F23F4807342E8AA
:10AEE000003123680029F5D103F1080252E8002F50
:10AEF00002EA090203F1080040E800210029F3D129
:10AF000020225345C4F88C20616721670AD05A6813
:10AF1000110207D553E8002F22F0806243E8002198
:10AF20000029F7D1E26E012A14D10022E26653E82B
:10AF3000002F22F0100243E800210029F7D1DA693E
:10AF4000B4F85C10D20644BF10221A622046FFF704
:10AF500025FC55E72046F9F7E1F951E79A6942F0F7
:10AF600008029A616EE700BFFEFFFFEF008000401D
:10AF700065AB000838B5044603682169A2681D68FE
:10AF8000C0690A4361690A437749024329400A4379
:10AF90001A605A68E16822F440520A435A60734AC0
:10AFA000A16993421CBF226A11439A6822F06E4243
:10AFB00022F430620A439A60DA6A616A22F00F0270
:10AFC0000A43DA626A4A934219D14FF0B043694AA0
:10AFD000D3F8883003F0030343F44033934200F086
:10AFE000B480B3F1031F24D0013A934240F0B580FE
:10AFF000B0F5004F40F08F80FCF780FF6EE05E4AB6
:10B0000093421CD14FF0B0435C49D3F8883003F031
:10B010000C0343F440228A4200F0978006D8002BAC
:10B020007CD0574B9A42E3D0012026E0B2F10C1FAE
:10B03000FAD1B0F5004F53D04FF4004075E04B4AC1
:10B040009342F1D14FF0B043D3F8883003F440631A
:10B05000B3F5006F18D006D85BB1B3F5806FE3D1BC
:10B06000FCF74CFF07E0B3F5406FDDD14FF4004033
:10B070000BE0FDF73BFB40B900204FF00113A36646
:10B080000023C4E91D3338BD3E4865683E4B626A03
:10B0900005EB450133F81220B0FBF2F39942C3D817
:10B0A000B3EB053FC0D800231946F7F7FDF90902B5
:10B0B00041EA10616B080002C0182A464FF00003F5
:10B0C00041F10001F7F7F0F9304BA0F540729A42D8
:10B0D000AAD82368D860CFE7FDF708FB0028CBD0BB
:10B0E0006168294B626A33F81220B0FBF2F24B0818
:10B0F00003EB42034FF6EF72B3FBF1F3A3F1100140
:10B10000914291D823F00F02216892B2C3F3420317
:10B110001343CB60B0E7FCF7F1FE04E0B0F5004F5D
:10B12000DAD0FDF7E3FA0028A6D06368616A164A10
:10B1300032F81120B0FBF2F000EB5300B0FBF3F05B
:10B140004FF6EF73A0F11002C1E7B0F5004F0D48C4
:10B15000EBD1C5E7FDF7DAFAC0E7B0F5004FF9D05B
:10B16000FDF7D4FADFE700BFF369FFCF00800040AE
:10B1700000380140020003000044004008000C00B9
:10B1800004000C000024F400E0620308FFFC0F0040
:10B19000836ADA0710B506D50168C46A4A6822F4E2
:10B1A000003222434A609C0706D50168046B4A6856
:10B1B00022F4803222434A60590706D50168446B65
:10B1C0004A6822F4802222434A601A0706D50168A1
:10B1D000846B4A6822F4004222434A60DC0606D5AA
:10B1E0000168C46B8A6822F4805222438A609906FF
:10B1F00006D50168046C8A6822F4005222438A60F2
:10B200005A060FD50168446C4A6822F48012224322
:10B21000B4F5801F4A6005D14A68846C22F4C002EC
:10B2200022434A601B0606D50268C16C536823F4AA
:10B2300000230B43536010BD2DE9F843DDF8209047
:10B2400005460F46164698462A68D36937EA03032F
:10B250000CBF01230023B34201D0002029E0B9F143
:10B26000FF3FF2D0F8F78CFCA0EB080048452C68B3
:10B2700002D8B9F1000F1ED154E8003F23F4D07377
:10B2800044E80032002AF7D104F1080353E8003FF4
:10B2900023F0010304F1080141E80032002AF3D150
:10B2A0002023C5F88830C5F88C30002385F8843019
:10B2B0000320BDE8F88323685A07C5D5E3691B0559
:10B2C000C2D54FF40063236254E8003F23F4D073E7
:10B2D00044E80032002AF7D104F1080353E8003FA4
:10B2E00023F0010304F1080141E80032002AF3D100
:10B2F0002023C5F88830C5F88C30C5F89030D4E7E5
:10B3000073B504460026C0F89060F8F739FC23684E
:10B310001B681A07054619D423681B685B070AD502
:10B320006FF07E43009300222B464FF480012046AD
:10B33000FFF782FFB0B900202023C4F8883084F8DA
:10B340008400C4F88C30E06620670CE06FF07E4328
:10B350000093324603464FF400112046FFF76CFF7E
:10B360000028D9D0032002B070BD10B5044650B3F8
:10B37000D0F888301BB980F88430F8F7CFFE226807
:10B380002423C4F88830136823F001031360204697
:10B39000FFF7F0FD012816D0A36A13B12046FFF78E
:10B3A000F7FE23685A6822F490425A609A6822F0A5
:10B3B0002A029A601A6842F0010220461A60BDE82B
:10B3C0001040FFF79DBF012010BD000030B5816522
:10B3D0008168A0F85C200023B1F5805FA0F85E20B2
:10B3E000436735D10369002B40F2FF1318BFFF23D9
:10B3F000A0F860300023C0F890302223C0F88C30D1
:10B40000016801F1080353E8003F43F001030831EC
:10B4100041E800340368002CF2D1456E846801696C
:10B42000B5F1005F32D1B0F8685095422ED8B4F52E
:10B43000805F244A03D1244C002908BF224642677A
:10B44000B1B153E8002F42F4807243E80021F7E7DE
:10B4500029B90369002B14BF7F23FF23C8E7B1F18B
:10B46000805FC5D10369002B14BF3F237F23BFE753
:10B4700003F1080252E8002F42F0805203F1080065
:10B4800040E800210029F3D1002030BDB4F5805FF1
:10B490000E4A03D10E4C002908BF2246426741B133
:10B4A00053E8002F42F4907243E800210029F7D1BD
:10B4B000EAE753E8002F42F0200243E80021002988
:10B4C000F7D1E1E729AC0008D1AD000899AA00083E
:10B4D00065AB0008D0F88C30202B30B415D1B9B151
:10B4E000B2B100230468C3660A4B9C420AD0636869
:10B4F0001B0207D554E8003F43F0806344E8003561
:10B50000002DF7D130BCFFF761BF022030BC70477F
:10B510000120FBE700800040436E30B52BB90123CA
:10B52000A0F86A30A0F8683030BD0368094D9A6809
:10B530009968094C490FC2F342626B5C615CDB00A5
:10B54000B3FBF1F3A0F86A30AB5CA25CDB00B3FBA9
:10B55000F2F3E7E700630308F862030870477047F7
:10B5600070471FB504AB03E9060090F88430012B47
:10B5700004463AD0012380F884302423C0F8883070
:10B5800003681A6822F001021A609A6822F44012D5
:10B590000A439A6071B95A68BDF80C009DF80E1004
:10B5A00022F0100202435A605A6822F07F4242EAB7
:10B5B00001625A601A6842F001021A60F8F7E0FA74
:10B5C0006FF07E42034600924FF480010022204635
:10B5D000FFF732FE38B92023C4F88830002384F8FE
:10B5E000843004B010BD0320F8E70220F9E790F89A
:10B5F0008430012B0FD0012380F88430016851E89A
:10B60000002F42F0020241E80023002BF6D180F81F
:10B610008430184670470220704710B590F8843087
:10B62000012B044617D02423C0F8883003681A6819
:10B63000196821F00101196042F000524FF00051E9
:10B6400041661A60FFF768FF2023C0F888300020A9
:10B6500084F8840010BD0220FCE770B590F88430B7
:10B66000012B044617D005682423C0F888302E68C3
:10B670002B6823F001032B60AB6823F06043194370
:10B68000A960FFF749FF20232E60C0F88830002012
:10B6900084F8840070BD0220FCE770B590F8843017
:10B6A000012B044617D005682423C0F888302E6883
:10B6B0002B6823F001032B60AB6823F06063194310
:10B6C000A960FFF729FF20232E60C0F888300020F2
:10B6D00084F8840070BD0220FCE7000038B5084DF6
:10B6E000052455F8043B2BB9013C14F0FF04F8D1B4
:10B6F000204638BDDB6898470028F5D0F9E700BF41
:10B70000B0200020034BD870034B1B681B6C03B1A7
:10B71000184770479820002094200020034B18748D
:10B72000034B1B685B6C03B11847704798200020DF
:10B7300094200020F0B5314D314B95F90420314E65
:10B7400091B00C46012795F905108DF80470022878
:10B750008DF809208DF80A1010D18DF80800D871E5
:10B760001C7203F075FB337803B114B101A804F027
:10B77000A5F8254B059A1A6011B0F0BD59714FF428
:10B7800080711A71D9801C7233788DF8087053BBA0
:10B790001F2306A88DF81C208DF8183003F036FD05
:10B7A00020238DF8183006A82B798DF81C3003F073
:10B7B0002DFD22238DF8183006A86B798DF81C30EA
:10B7C00003F024FD21238DF8183006A86B798DF83D
:10B7D0001C3003F01BFD29238DF8183006A80B4BF5
:10B7E000079303F013FD03F033FB012306A88DF844
:10B7F00018308DF81C3003F009FDB4E798200020C4
:10B800003C010020741F002068200020000400017B
:10B810007FB5092301A88DF8043004F04FF80038F3
:10B82000044B059A1A6018BF0120404207B05DF82A
:10B8300004FB00BF6820002070B504460B46144985
:10B8400062784A700020A2780A7208701A884A72D8
:10B850009A788A72DB780B746368CB600D4B1B6837
:10B86000DA6A2AB1237803F0FB030A2B00D0904751
:10B87000094E002556F8043B1BB15B6A0BB120460C
:10B8800098470135EBB2052B6DB2F3D170BD00BF07
:10B890000C01002094200020B020002070B5044648
:10B8A00011480123037063784370A3788372E368BF
:10B8B000C360E378037623694376237943720B4BA5
:10B8C0001B689B6A03B19847094E002556F8043B54
:10B8D0001BB19B690BB1204698470135EBB2052B94
:10B8E0006DB2F3D170BD00BF200100209420002074
:10B8F000B0200020014B1868704700BF682000206E
:10B9000000B58BB0012368468DF8003003F058FB7A
:10B9100038B99DF80400003818BF01200BB05DF85D
:10B9200004FB0020FAE7000008B502F049FC40B92A
:10B93000FFF7E6FF012806D0054B197AD879FFF703
:10B94000F9FE012008BDBDE80840FFF7C7BE00BFF3
:10B950003C0100202DE9F04186B005460E46174611
:10B9600002F02EFC002873D102F042FC044640B9DC
:10B97000FFF7C6FF01280AD03D4B197AD879FFF7A7
:10B98000D9FE6FF00204204606B0BDE8F081DFF872
:10B99000E48088F80860003E18BF01268DF8046036
:10B9A000354E687833798DF81230694603F0A6FA7F
:10B9B00000283FD08DF804400394ADF810406FF09C
:10B9C000060495E803002D4B83E80300337988F8DB
:10B9D0000A30394601A804F075F8294B059A1A6017
:10B9E00011283FD801A353F820F000BF57BA000830
:10B9F00051BA000865BA000865BA000865BA0008BF
:10BA000065BA000865BA000883B9000865BA00087D
:10BA100065BA000865BA00084BBA000865BA0008A4
:10BA200065BA000851BA000851BA000851BA0008B6
:10BA30006BBA00082B788DF808306B78ADF81030B1
:10BA40006B6803934FF0FF34BBE76FF005049AE790
:10BA50006FF0010497E70B4B00221A70E31D18BF2B
:10BA6000144690E74FF0FF348DE76FF004048AE747
:10BA70003C010020200100209820002030010020FF
:10BA8000682000206720002037B502F0BBFB134D73
:10BA9000052455F8043B4BB11A693AB19B682BB1A8
:10BAA000984718B155F8043C1B699847013C14F0BD
:10BAB000FF04EED1FFF712FE68B9094D2B7853B1A0
:10BAC000084BADF80040D978019422466846FFF74C
:10BAD00041FF00B92C7003B030BD00BFB020002082
:10BAE000672000209820002030B58BB0044602F07B
:10BAF00067FB0546002835D1FFF702FF012834D146
:10BB000068468DF8005003F05BFA40BB9DF80430A6
:10BB1000A34204D0012C22D0022C12D014B1002058
:10BB20000BB030BD002BFAD068468DF8044003F00E
:10BB30006DFBA0B90E4B1B681B6B002BEFD0984719
:10BB4000EDE763B968468DF8044003F05FFB30B958
:10BB5000074B1B681B6B002BE1D02046EFE74FF033
:10BB6000FF30DDE76FF00100DAE76FF00200D7E7A2
:10BB70009420002010B504468AB018B94FF0FF3069
:10BB80000AB010BD002368468DF8003003F018FAA3
:10BB90000028F3D19DF804302370F1E77FB500222F
:10BBA0000B4620498DF8072001220A7042784A701E
:10BBB0000446002A33D102790A721A884A729A78A6
:10BBC0008A72DB780B740369CB60C378164D8DF8ED
:10BBD0000830037B8DF80930836803932B68DB6A98
:10BBE0000BB102A898472B689B6B13B1227E02B160
:10BBF00098470E4E052556F8043B1BB1DB690BB187
:10BC000020469847013D15F0FF05F4D10DF10700DE
:10BC1000FFF7B0FF637913B1054B01221A7004B02E
:10BC200070BD00BF0C01002094200020B020002037
:10BC30006720002010B504468AB018B94FF0FF30D5
:10BC40000AB010BD202368468DF8003003F0B8F923
:10BC50000028F3D1024A9DF9043023701371EFE7F5
:10BC60009820002000B58BB02323019068468DF802
:10BC7000003003F0CBFA003818BF012040420BB06F
:10BC80005DF804FB70B5654C01468EB01822204665
:10BC900006F0BCFF624B00221A70FAF77FFE237891
:10BCA0004068012202FA03F1014004D15D4B0846CD
:10BCB00008F098FFFEE75C495C481A4602F00AFF6C
:10BCC00018B14FF0FF300EB070BD272304A88DF8D7
:10BCD000103003F09BFA564E564D002870D10123C8
:10BCE00033702B68DB690BB100209847272304A829
:10BCF0008DF8103003F064F9059B93F8482022700A
:10BD000093F8182193F81A316270A370464BD3E967
:10BD1000020106F06BFE05460028D2D1464E0623EE
:10BD200004A88DF8103003F04BF9059B736104A84B
:10BD300003F06CFA022304A88DF81030059603F086
:10BD40003FF90836032304A88DF81030059603F058
:10BD500037F90F2606F010FF012304A88DF81430E0
:10BD60008DF8106003F052FA10230DEB03008DF8EC
:10BD700010308DF8145003F049FA04238DF8103078
:10BD800004A8A3788DF8143003F040FA3A238DF814
:10BD9000103004A86369059303F038FA02A92078EB
:10BDA0008DF8086004F0CCFF003818BF0120E07166
:10BDB0001420FFF757FFE07904F046F8284682E7A1
:10BDC00028238DF810302B681B6943B104A803F0B9
:10BDD000F7F82B6805981B6940F2C4519847272350
:10BDE00004A88DF8103003F011FA50B9012304A80B
:10BDF0008DF8103003F0E4F89DF81430002B7FF438
:10BE00006EAF3378002B7FF46CAF052204A88DF859
:10BE10001020059303F0FAF978E700BF982000207E
:10BE200067200020086303086C2000208420002085
:10BE3000741F002094200020D420002037B5002358
:10BE40000D4601930446D0B900F07CFD0190019BA2
:10BE5000D3B10F4A42F824300E4A9A620E4A126851
:10BE6000916B1963916C596392690C49D9625A615B
:10BE700028465B680A49F2229847002006E001A99B
:10BE800000F076FD0028E2D04FF0FF3003B030BD67
:10BE9000B020002035B700089420002011B8000819
:10BEA000751F0020194B07B51860194B194A1A6005
:10BEB000194A5A60194A9A60194ADA60194B02689D
:10BEC0001A6042685A6082689A60C268DA60164AEC
:10BED0001A6182695A61154BC26B5A60144A01910A
:10BEE00019609A601946134ADA600020FFF7A6FF2E
:10BEF00048B901A800F02AFD003818BF01204042CF
:10BF000003B05DF804FB4FF0FF30F9E79420002008
:10BF1000842000209DB800089DBB0008DDBF0008FC
:10BF200039B800086C200020F10C0108C420002062
:10BF300005B700081DB7000849B118B1012804D0A1
:10BF400000207047034B0B60FAE7034BFBE74FF011
:10BF5000FF307047000400010100010208B503F042
:10BF60008FFF002814BF6FF00100002008BD08B546
:10BF700002F096FF002814BF6FF00100002008BDFA
:10BF800020B1044BDB790370002070474FF0FF3085
:10BF9000704700BF9820002008B5034BD87103F00C
:10BFA00053FF002008BD00BF9820002010B50446B4
:10BFB0008AB018B94FF0FF300AB010BD212368468F
:10BFC0008DF8003002F0FCFF0028F3D1024A9DF901
:10BFD000043023705371EFE7982000202DE9F041E1
:10BFE0002F4D304F00232B7043786B703B689B6A5A
:10BFF0008AB004460BB128469847DFF8AC8000268B
:10C0000058F8043B1BB11B6A0BB120469847013618
:10C01000F3B2052B76B2F3D12378052B2FD00B2B5F
:10C0200035D0012B25D1214C062368468DF80030F0
:10C0300002F0C6FF0199E07906F01EFD10B91C4B15
:10C04000019A5A611B48FFF7F5FD1B48FFF7AEFF49
:10C050006B788BB9A371194B5878FFF745FD3B6896
:10C060005B6A0BB1114898476B7813B9E07906F019
:10C0700095FD0AB0BDE8F081FF23A371EFE7104BF7
:10C0800001225A74227A9A74627ADA74F1E7637838
:10C09000002BEED00AB0BDE8F041FFF7B9BB00BFFE
:10C0A0002001002094200020B02000203C0100202E
:10C0B000D4200020400100204101002098200020D1
:10C0C0000C01002030B58BB0FFF751FF0446F0B9EA
:10C0D00004F016FE831C1DD0F8B9134D2B685B6964
:10C0E000DBB1272368468DF8003002F069FF2B682A
:10C0F00001985B694FF4B961984704F013FE78B971
:10C100002CB9094B1B68DB690BB10120984720460D
:10C110000BB030BD6FF00704EFE74FF0FF34ECE7F2
:10C120004FF0FF34F3E700BF94200020014B187854
:10C13000704700BF04210020014B5878704700BFB2
:10C1400004210020064B074810B501225A7309F05C
:10C1500085F9054B5B6913B1BDE81040184710BD68
:10C1600004210020EC2000204801002013B50A4CD7
:10C1700079B1A27001230022616023700748084B47
:10C1800000924FF0FF3109F0BDF80023637002B058
:10C1900010BD2170F9E700BF04210020EC20002031
:10C1A00045C100082DE9FF47C378CA2B804600F03F
:10C1B000BE8004B0BDE8F087D8F808305A5D6E1C28
:10C1C000F6B2032A0FD8DFE802F0022E6CAB7A68D1
:10C1D00000231355611CA31CDBB2C9B201205054CB
:10C1E0000334D054E4B2354698F80C30AB42E3D86F
:10C1F000002CDED0CA238DF80830504B8DF8094052
:10C200005B6803930DF10700FFF7BAFE0020FFF70C
:10C21000C3FE0122002102A8FFF79CFB9DF8070046
:10C22000FFF7BAFEC5E700227A7398F818204AB9DA
:10C230006A1DD2B2397A9A5C01F00F0102F00F0246
:10C24000914202D0AE1DF6B2CDE7AA1CD2B29E5DDD
:10C250009A5C06EB0226EA1CD2B20DF1080A9A5C3F
:10C2600006EB02462A1DD2B250469B5C06EB0366E3
:10C2700008F022FF029B334402939AE8030008F07F
:10C28000F3FE3B7AC3F30302013262F303033B7212
:10C290002B4B1B6B002BD5D00136022ED2D89847E2
:10C2A000D0E7EE1C0235EDB21E215B5D002003F0ED
:10C2B0000F0380259D4006F08DFC7A6802231355FC
:10C2C00004EB030A631CDBB20021D154054402A82D
:10C2D00008F0F2FE029B7A684B4504F1030188BF27
:10C2E000A3EB09035FFA8AFAC9B2180A02F80A3006
:10C2F0005054611D201DC9B2C0B24FEA134C1B0E31
:10C3000002F800C053544FF47A7169430D4809F0A4
:10C31000DFF806340B48F6B2E4B209F09FF862E7A2
:10C320009B5D023503F007037B73EEB25BE70024ED
:10C33000024FDFF81490254656E700BF0421002085
:10C3400048010020EC200020803DD51210B5114C92
:10C35000637A8AB0E3B104238DF800306846A37A8B
:10C360008DF8043002F052FF18238DF80030684633
:10C37000E37A8DF8043002F049FF20238DF8003075
:10C380006846237B8DF8043002F040FF002363727F
:10C390000AB010BD04210020004870474801002069
:10C3A00030B58FB0FFF7C0FA002861D1324C657A02
:10C3B0004DBB042304A88DF8103002F001FE9DF857
:10C3C0001430A37204A88DF8145002F01FFF182334
:10C3D00004A88DF8103002F0F3FD9DF81430E372DC
:10C3E00004A801238DF8143002F010FF202304A8C4
:10C3F0008DF8103002F0E4FD9DF8143023731F4BCC
:10C40000DB6A03B1984702A808F056FE029A1C4B5B
:10C410001C4913448B4288BF1B4B616888BF9B1823
:10C420001A0A4B708A701A0C1B0E0B71237ACA7091
:10C4300001256FF304134B710D7023720DF107008A
:10C4400040F2CA63ADF8103005916572FFF798FDB0
:10C450000020FFF7A1FD2A46002104A8FFF77AFA81
:10C4600004469DF80700FFF797FD20460FB030BD4A
:10C470004FF0FF34F9E700BF0421002048010020FD
:10C4800080C22AED803DD512008555DA10B5054CE5
:10C49000637B2BB1FFF784FF10B9637B013B6373B0
:10C4A00010BD00BF04210020014B1878704700BF69
:10C4B00030210020014B5878704700BF3021002008
:10C4C00070470000044B9A7A0AB101225A70034B5C
:10C4D0005B6903B1184770473021002080010020BC
:10C4E00073B5224C6378002B33D008F025FF6668C3
:10C4F0000546FFF7FFF90644AE4214D2A37A93B182
:10C50000E0228DF800208DF80130217AE368019354
:10C5100001226846FFF71EFA08B1073010D1002348
:10C520006370A372656094F83430EBB1002384F833
:10C5300034300F4B5B6BBBB102B0BDE870401847A5
:10C5400040F2DC510B4808F0C3FF0A4808F086FFB0
:10C55000E8E794F83520002AE5D094F8360084F80E
:10C560003530FFF7C1FADEE702B070BD30210020A0
:10C57000800100201421002037B5104D104CC8B1A7
:10C58000C1B16272012300222860E16023700D486E
:10C590000D4B00924FF0FF3108F0B4FE00250B4820
:10C5A00025822022294606F045FB6570A574A586E4
:10C5B00003B030BD00232B602370EFE72C21002057
:10C5C0003021002014210020C5C40008442100208F
:10C5D0002DE9F0478E4C23788CB0002B56D0C278D2
:10C5E0000AB9837B13B1238A01332382437B002B57
:10C5F0004CD0E02A4AD10023A372876897F80080C4
:10C60000B8F1220F27D8B8F1220F30D8DFE818F0A0
:10C610004100FB0052005A0061006E0075008E0060
:10C620009D00B400C7002F002F002F002F002F0007
:10C630002F002F002F002F002F002F002F002F0082
:10C640002F002F002F002F002F002F002F002F0072
:10C65000C900D000D400B8F17E0F00F0CC80B8F152
:10C660007F0F00F0DF80B8F17D0F00F0AB80A57A7E
:10C67000002D00F05B81674C637A3BB94FF47A710F
:10C68000204608F025FF204608F0E8FE0CB0BDE883
:10C69000F087E36801220021A2721970A37AE16891
:10C6A0009818A0720620C854A37AE1689818A0725E
:10C6B000CA54DCE7584B9B6A002BD8D001210220DA
:10C6C0009847D4E77B7884F83630012384F83530F6
:10C6D000CDE704238DF804307B78003B18BF01239D
:10C6E00001A88DF8083002F091FDC0E77878003895
:10C6F00018BF012003F0A8FBB9E7484E0FCE01ADEB
:10C700000FC50FCE0FC596E8070085E807007B78B8
:10C710000A2BACD8424A12685268002AA7D00CA94A
:10C7200001EB830353F82C0C9047A0E77878431E65
:10C73000012B9CD83A4B01381B6818BF012020728E
:10C740009B68002B93D0984791E7E268012308216A
:10C75000A3721170627A057BA17AAA4228BF2A4689
:10C76000934284D285685A1CEB5CE56801334E1C09
:10C77000A6726B54D3B2EDE7E3680122A2720922DC
:10C780001A70A37AE268218A581CA072D154A27A46
:10C79000238AE1681B0A501CA0728B5467E723822E
:10C7A00065E705238DF8043001A803F087F85EE7FC
:10C7B000194BDB6A98475AE7194B78781B68607504
:10C7C000DB68BEE7037B072B7FF451AF06238DF8B0
:10C7D0000430B7F80130ADF808307B793A791B04A2
:10C7E00043EA0223FA781343642253430393BB7949
:10C7F0008DF81030D8E73B2201A88DF804208DF881
:10C80000083002F003FD012384F834302FE700BF25
:10C810003021002014210020800100201420030872
:10C820002C2100202A2301A88DF8043002F0C8FB37
:10C8300094F80A90E6689DF808009DF809509DF864
:10C840000A709DF80BC09DF80D309DF80E209DF8E4
:10C850000F109DF80CE009F1010A84F80AA006F80F
:10C860000980354E94F80A903668D4F80C8009F1A6
:10C87000010A84F80AA096F803A008F809A094F821
:10C880000A90D4F80C8009F1010A84F80AA096F8FD
:10C8900002A008F809A094F80A90D4F80C8009F1D5
:10C8A000010A84F80AA096F801A008F809A094F8F3
:10C8B0000A9009F1010A84F80AA096F80080E66857
:10C8C00006F8098094F80A80E66808F1010984F8FE
:10C8D0000A9006F808C094F80AC0E6680CF101084E
:10C8E00084F80A8006F80C70A77AE66807F1010C54
:10C8F00084F80AC0F555A57AE6686F1CA7727055D2
:10C90000A07AE568461CA6722954A17AE0684D1CFD
:10C91000A5724254A27AE168501CA0728B54A37A8B
:10C92000E268591CA17202F803E0A0E6034808F08F
:10C9300047FD6570AAE600BF2C21002014210020CD
:10C94000704700000048704780010020002108B5B2
:10C950000120FFF773FA014638B90220FFF76EFA9B
:10C96000003818BF0120404208BD4FF0FF30FBE700
:10C9700010B50C4661B1012803D0022805D0002073
:10C9800010BDFFF709FD2060F9E700F01FFCFAE792
:10C990004FF0FF30F4E70000014B1878704700BFFC
:10C9A000F0010020014B5878704700BFF0010020D3
:10C9B000F7B500208DF80700EFF3108272B62A4F0A
:10C9C000BB78FD7882F31088012B08D0022B04D1AC
:10C9D000264B93F82030012B3CD103B0F0BD234E01
:10C9E0000DF10700FFF7C6F8382303FB056393F842
:10C9F0002C00012806D19DF80730022B08D1002316
:10CA0000BB70EAE7022803D19DF80730012BF5E758
:10CA1000FFF76AF805EB4504E400B0B9144BB870B1
:10CA20001C44382303FB05664FF47A7196F82830CE
:10CA3000994096F82C30012B00D1C901204608F00E
:10CA400047FD204608F00AFDC7E70A4B1C444FF497
:10CA50007A71F3E7FFF748F80028D0D0044C05EBD3
:10CA6000450504EBC504F2E7F00100209821002001
:10CA7000682100208021002037B50F4CD1B100255E
:10CA80000123A160227123702A460C4B0C480095AB
:10CA90004FF0FF3108F036FC0A4B0B4800952A4650
:10CAA0004FF0FF3108F02EFC084A0023637013702A
:10CAB00003B030BD2170F7E7F001002005CB00087E
:10CAC00080210020D1CA0008682100209821002080
:10CAD00010B5084808F074FC074B002283F82020AA
:10CAE000064B02225A80064B5B6913B1BDE8104029
:10CAF000184710BD6821002098210020F001002077
:10CB0000B801002010B5084808F05AFC074A012374
:10CB100082F82030064A5380064B5B6913B1BDE8AA
:10CB20001040184710BD00BF802100209821002030
:10CB3000F0010020B80100202DE9F04FC378C82B88
:10CB40008FB0824600F029830FB0BDE8F08FDAF88D
:10CB50000820D05C591CC9B2052816D8DFE810F0AF
:10CB60000600AA00F000AE01E1018B02BA680023C2
:10CB7000601C1355C0B2A31CDBB24FF0020C02F8CC
:10CB800000C001200334D054E4B20B469AF80C20C4
:10CB90009A42DCD8002CD7D0C8238DF81430B74B7C
:10CBA0008DF815409B6806930DF11300FFF7E8F927
:10CBB0000020FFF7F1F90122002105A8FEF7CAFEC7
:10CBC0009DF81300FFF7E8F9002DBDD1AC4CAD4F37
:10CBD000637803F003032A46294600930220AA4BF8
:10CBE00008F000F82646636800932A462946A74BBA
:10CBF000022007F0F7FF16F8083F00932A4629465F
:10CC0000A34B022007F0EEFF012516F8013F009329
:10CC100000223B4611460220013507F0E3FF102DAC
:10CC2000F3D1002211469B4B022007F0DBFFA369E2
:10CC3000009300221146984B022007F0D3FFE369CE
:10CC4000009300221146954B022007F0CBFF636A48
:10CC5000009300221146924B022007F0C3FF94F884
:10CC600028200123934000221146009302208D4B7F
:10CC700007F0B8FF94F82C300022012B236B0093AF
:10CC80001146894B4FF0020040F08D8207F0AAFF59
:10CC900094F9343000930022844B1146022007F0AF
:10CCA000A1FFE38E0093824B00221146022007F081
:10CCB00099FF49E7BD6812F801C001222A550233E5
:10CCC00000220234DBB2E4B2114696460CF0010CAD
:10CCD00096F80080BEF1000F07D0120102F070023A
:10CCE00011436970054619464FE7B8F1000FF4D0BB
:10CCF000BCF1000F21D005F804E004F1010E5FFA49
:10CD00008EFE716805F80E1004F1020E71685FFA6C
:10CD10008EFE090A05F80E1004F1030E5FFA8EFE6E
:10CD2000B6F8068005F80E80211DC9B296F807E016
:10CD300005F801E00534E4B2614601328646C7E7F2
:10CD4000555C382105F0030501FB056103F1020B79
:10CD50005FFA8BFB4D70002D40F08E80D81C12F8CE
:10CD60000B107160C0B203F1050C105C01EB0021E7
:10CD7000181DC0B27160105C5FFA8CFC01EB0041C1
:10CD8000716012F80CC0981D01EB0C6903F11601DB
:10CD9000DFF820C1C6F80490C0B2C9B2864601309F
:10CDA000C0B212F80EE00CF801EF8842F6D1115C27
:10CDB000B16103F11700C0B203F11E0B105C01EB6F
:10CDC000002103F11800C0B2B161105C01EB004119
:10CDD00003F11900C0B2B161105C01EB006803F10E
:10CDE0001A01C9B2C6F8188003F11B00515CF16149
:10CDF000C0B25FFA8BFB105C01EB002103F11C0059
:10CE0000C0B2F161105C1D3301EB0041DBB2F16196
:10CE1000D35C0DF1170001EB036321220021F361C4
:10CE2000039321F0FBFD40F20112ADF8142072785B
:10CE3000039B0A93C2F301028DF8162005A81E4A2F
:10CE4000CDF818900792CDF8248002F065FC0123FC
:10CE500090B93370B96802230B55621C1C44382307
:10CE600003FB0563D2B25B78C3F3010343EA80009E
:10CE70008854E4B2594688E60120EBE7F00100202F
:10CE800098210020A76303086C6303087F630308ED
:10CE900094630308096B0308AD630308C0630308C8
:10CEA000D3630308E6630308FB6303080E64030807
:10CEB000246403089F210020A0210020555C382015
:10CEC00005F00305023300FB05FB5FFA83F906EB6F
:10CED0000B034FF00008184610224146083083F833
:10CEE0000180C3F80480039305F0A4FE039BC3E90B
:10CEF0000688BB68032204F101081A5528465FFA28
:10CF000088F802F051FC40B145F00403BA680234DD
:10CF100002F80830E4B2494637E606F80B002B4623
:10CF2000F4E74FF0000B8DF813B0555C03F10208E5
:10CF300015F003055FFA88F840F09680DFF874B2C8
:10CF40004FF002098BF82C90D81C12F80810CBF87F
:10CF50002410C0B203F10B08105C01EB0021181D76
:10CF6000C0B2CBF82410105C01EB0041581DC0B2D8
:10CF7000CBF82410105C01EB00618F480844991D28
:10CF8000C9B2CBF82400515C01F00F018BF82810D6
:10CF9000D91DC9B203F10800515CCBF83010C0B202
:10CFA0005FFA88F8105C41EA002103F10900C0B281
:10CFB000CBF83010105C0A3341EA00416420414351
:10CFC000DBB2CBF83010D35C8BF834300DF11302A8
:10CFD0000BF12C01284602F013FC002849D105A8CA
:10CFE00008F06AF8DBF82420059BA2EB030BBBF1E9
:10CFF000000F31DD4FF47A7101FB0BF16F480391A3
:10D0000008F066FA6D4808F029FA039900916C4B14
:10D0100029462A46484607F0E5FD0121BA6804235F
:10D020001355601CC0B29DF813C002F800C0A31CC9
:10D03000DBB271B102F803B0E31CDBB24FEA2B2183
:10D04000D154631D0434E4B24FEA2B4B02F804B010
:10D05000DBB21C46414698E59DF8133043F01003BF
:10D060008DF813302946D9E710238DF8133059462F
:10D07000D4E7AB46F6E74FF0000B8DF813B0555CE4
:10D0800003F1020815F003055FFA88F87ED1DFF896
:10D0900024B14FF001098BF82C90D81C12F808101D
:10D0A000CBF82410C0B203F10B08105C01EB002197
:10D0B000181DC0B2CBF82410105C01EB0041581DC4
:10D0C000C0B2CBF82410105C01EB00613A48084470
:10D0D000991DC9B2CBF82400505CC0F30210ABF824
:10D0E0003600515C01F00F018BF82810D91DC9B230
:10D0F00003F10800515CCBF83010C0B25FFA88F839
:10D10000105C41EA002103F10900C0B2CBF83010F5
:10D11000105C0A3341EA004164204143DBB2CBF8A2
:10D120003010D35C8BF834300DF113020BF12C016D
:10D13000284602F065FB70BB05A807F0BDFFDBF8D1
:10D140002420059BA2EB030BBBF1000F16DD4FF46F
:10D150007A7101FB0BF11948039108F0B9F91748EE
:10D1600008F07CF903990091154B29462A460220C4
:10D1700007F038FD4946BA68052351E79DF813309A
:10D1800043F010038DF813302946F4E710238DF88F
:10D1900013305946EFE7AB46F6E70024094F054E3A
:10D1A000FF252346F2E407F01DFD94F93430009387
:10D1B000054B79E598210020803DD5128021002083
:10D1C00051630308F00100200E6403080048704713
:10D1D000B8010020044B054A93F81831022B18BF00
:10D1E000062382F8903470473C280020002E00204F
:10D1F000034BD3F8483313B15B6903B11847704749
:10D20000002E0020034A137843F004031370FFF745
:10D21000EFBF00BFE42100201FB50A4B8DF80900C5
:10D2200093F87C208DF80A2093F88C2093F848001E
:10D230000D3202A98DF8082003F082FDC0B205B0BE
:10D240005DF804FB3C28002008B5074808F0B8F852
:10D25000064B93F81A2412B1012283F81924BDE871
:10D260000840FFF7C5BF00BF00320020002E00209D
:10D2700010B50C4CD4F8403343F08003C4F840336D
:10D2800094F81A3413B10020FFF7DEFF94F89134BC
:10D2900023F0120343F0120384F89134BDE81040E8
:10D2A000FFF798BF002E00202DE9F041DFF8AC8099
:10D2B00098F81831022B06460D4602D0284BDB6A3F
:10D2C000984702F078FE044628B1022002F069FE79
:10D2D000002002F06BFE98F81831012B17D102F0F4
:10D2E0006CFE074630B1002002F05CFE002002F028
:10D2F0005EFE3C4602F063FE48B1002002F053FEA1
:10D30000002002F055FEBDE8F041FFF763BF002C9E
:10D31000F9D1144C94F8902494F81A34BAB90BB19A
:10D3200084F84164304602F0EBFFD8F82C0008F096
:10D330000DF8D4F8B4339842E5D30B4808F040F820
:10D3400094F8913443F0100384F89134DBE70BB187
:10D3500084F84154284602F0D3FFF1E73C2800202E
:10D36000646B0308002E002098310020074A10B596
:10D37000137843F002031370FFF73AFFBDE8104043
:10D38000034B01220021022007F02CBCE4210020E5
:10D3900037640308074A10B5137843F00803137085
:10D3A000FFF726FFBDE81040034B012200210220B9
:10D3B00007F018BCE4210020476403082DE9F04180
:10D3C0000F4616461D46804607F0B6FF0B4A0C4C2A
:10D3D0001378278123F0110343F01103C4E90008F7
:10D3E000137066812573FFF703FFBDE8F041054B1D
:10D3F00001220021022007F0F5BB00BFE42100203C
:10D40000D02100205764030813B507F095FF0D4B9A
:10D410006C461860204607F04FFE94E803000A4A65
:10D420000A4B83E80300137843F020031370FFF7DF
:10D43000DFFE074B01220021022002B0BDE81040B0
:10D4400007F0D0BBE0210020E4210020383100208B
:10D45000646403082DE9F04192B0064602F0ABFD8A
:10D46000002840F05881AD4D95F81831012B09D0B6
:10D470002B6BAB4C93B194F80431BBB1042B6FD040
:10D48000032003E002F099FD18B10F2012B0BDE8AF
:10D49000F08102F094FD0028EAD0F6E7B5F82031DB
:10D4A000D4F81C24013B53432B63E4E79D4803F06D
:10D4B0007EFB002840F0128194F80C3123802B6B06
:10D4C0000C930DF1180895F839308DF83830404636
:10D4D00095F81C318DF83A3007F014FED5F8283154
:10D4E000009302AF98E80600D5F82431384607F0DB
:10D4F0009FFD97E803000FAB83E80300EB6A0D93F1
:10D5000000238DF844302388ADF8463095F830314B
:10D5100001228DF839201BB98DF844208DF839305F
:10D52000814B0093814B95F84800A3F179020CA937
:10D5300003F07BFCC0B10B28A8D1D4F8941499B1A6
:10D54000002EA3D0D4F84033794843F02003C4F828
:10D55000403307F0BDFF764807F080FF002095E7D5
:10D56000704803F058FBA4E795F8487095F96930C6
:10D5700095F9392095F87D106E4E384603F062FC1F
:10D58000009641B2EB6C95F850203846183603F0FF
:10D59000FDFB0096EB6C95F8502095F9701095F80E
:10D5A000480003F0F3FBD4F8C413AB6DD4F8DC23CC
:10D5B0000B44C4F8B033EB6D1344C4F8B43394F89F
:10D5C0000431042B07D02B6E0B44C4F8B0336B6EC0
:10D5D0001344C4F8B4330023089395F83031002B7A
:10D5E00040D100238DF8133095F839308DF8213073
:10D5F00095F838308DF82230D5F880300993D5F879
:10D6000084300A932388ADF82C3095F8303194F8A3
:10D610001B648DF82E3095F84800474B8DF820603C
:10D620000DF1130208A903F0C5FB012384F841346E
:10D6300095F8393084F842349DF8133084F8433437
:10D64000D4F81C34C4F85064C4F84834C4F85834CE
:10D6500002F0B7FCC8B1D4F81C0402F0C4FCA0B1BD
:10D66000102013E708A802F07BFD60B995F9390096
:10D6700094F837629DF82070FFF7CEFD3E44B0422B
:10D68000AFD2082002E7132000E795F81831012BEC
:10D6900001D102F0AAFC02F097FC0023059394F854
:10D6A000043195F9395094F81B649BB1042B7FF435
:10D6B000E7AE05A802F088FF58BB94F8183413B100
:10D6C000059B013B0593174B05983246E9B202F0E2
:10D6D000E1FF02E0134802F0B1FF08B11120D5E6E6
:10D6E000D4F8403394F80C11218043F00203C4F8BD
:10D6F000403394F8183411480133DBB284F81834FD
:10D7000084F845340E4B00259B6AC4F8985498471A
:10D7100024E71220BAE60E20B8E600BF3C2800201D
:10D72000002E0020082F00206C28002094320020BA
:10D7300068310020B83100201C320020022E002069
:10D74000646B030873B5134D134E0096EB6C95F89C
:10D75000502095F9781095F8480003F017FB95F8DC
:10D760003031337595F8480040F2012306F13C0250
:10D770003146738203F016FB50B196F83C3086F8C0
:10D780008230064B00205B6B9847F37C86F8A8300C
:10D7900002B070BD3C280020E8310020646B030813
:10D7A000F8B5324C94F81831012B05460ED0022BF7
:10D7B0004ED0002B57D138B9D4E91B0104F17403C2
:10D7C00083E803000020F8BD012806D102F0FEFB2B
:10D7D0000028F8D184F81851F5E7022843D1244EE7
:10D7E00084F8180106F5747CBCE80F0006F57A771A
:10D7F0000FC79CE8030094F8E92094F8003187E80B
:10D80000030086F8FB53D2B1022B18D1D4F80431AF
:10D810006367C6F8EC3394F87D3094F8082186F8F5
:10D82000F83394F88C3084F8782086F8F93396F839
:10D830001B2486F8E82340F20133A6F8FA330023CC
:10D8400086F81A340B4BDB6A9847FFF77BFFB9E782
:10D8500048B9074B84F81801062283F89024054B39
:10D86000DB6A9847AEE70320ADE700BF3C28002005
:10D87000002E0020646B0308F0B5504C504EB4F8F5
:10D88000DC202287D4E92D0194F8B12084F86920A6
:10D8900004F16C0282E80300D4E92F0104F1740260
:10D8A00082E80300B4F8C420A4F87C2091B0D4F836
:10D8B000CC20D4F8C810C4F884200025D4F8D02097
:10D8C000C4F888200123A4F82031C4F8801084F81B
:10D8D0003051A56284F81B5184F83A5084F81D51E8
:10D8E00084F81E51C4F83451C6F89854A6F8185458
:10D8F00086F81A54A4F838518DF8183004F50973D5
:10D90000039304F50A7394F84800049303A92D4B7C
:10D9100084F84551C4E94F55A4F84651059303F0E6
:10D920001DFAE36EC6F8D43394F87D3086F8E03300
:10D9300094F88C3086F8E1334FF48073A6F8E23324
:10D9400086F8D05394F8303186F8E43306F57477CE
:10D950000FCF06F57A740FC497E8030040F2012355
:10D9600084E80300A6F8FA33D6F8483386F81B5447
:10D97000CDE901551BB15A685B6901920293124BC4
:10D980000793A3F148020892A3F1140209920F4AE7
:10D990000B9229330A93A2F19C030C93A2F19803F2
:10D9A0000D93131D0E9301A902F14C0307A802F574
:10D9B00099620F9302F0F4FA11B0F0BD3C280020F8
:10D9C000002E0020E82100206832002020290020BD
:10D9D000F8B50D4F0D4E0C4607F0F2FC3B6B984727
:10D9E0000B4A96F84800214603F0DCF950B1094D86
:10D9F000706D95F8243485F86A347B6B9847E37C26
:10DA000085F89034F8BD00BF646B03083C28002003
:10DA100024320020002E00200F4890F81B3480F89C
:10DA2000B8330E4B93F8692080F8BB2393F87D2020
:10DA300080F8C82393F88C2080F8C92393F83031FC
:10DA400080F8CC330022A0F8CA2300F56E7100F5EF
:10DA50006070FFF7BDBF00BF002E00203C280020F3
:10DA6000114890F89034EBB190F81B3480F8D03323
:10DA70000E4BDA6EC0F8D42393F87D2080F8E023B3
:10DA800093F88C2080F8E12393F8303180F8E43368
:10DA90004FF48072A0F8E22300F5747100F566700F
:10DAA000FFF796BF704700BF002E00203C280020E3
:10DAB00070B5344C2421204605F0BEF8636A9842C4
:10DAC00018BF60624FF01C012F4814BF01250025CC
:10DAD00005F0B2F8636C984218BF60644FF480712F
:10DAE0002A4818BF45F0020505F0A6F8D4F84831D9
:10DAF000984218BFC4F848014FF0D401244818BF19
:10DB000045F0040505F098F8D4F82032984218BF83
:10DB1000C4F820024FF000011E4818BF45F0080568
:10DB200005F08AF8D4F82432984218BFC4F82402C9
:10DB30004FF46071184818BF45F0100505F07CF8E7
:10DB4000D4F8A835984218BFC4F8A8054FF01401BE
:10DB5000124818BF45F0200505F06EF8D4F8C0351E
:10DB600098420F4B18BFC4F8C005D3F8483318BF0C
:10DB700045F040052BB11B691BB12846BDE870403C
:10DB8000184770BD3C28002064280020842800200D
:10DB900088290020602A0020642A0020E82D002027
:10DBA000002E00202DE9F04F8FB04FF00009012B1F
:10DBB00006460F4690468DF80D90ADF8109002D8AD
:10DBC0004C46BC4202D30FB0BDE8F08F305D02F08E
:10DBD00007FB2044B842F6DC335D651C023BEDB226
:10DBE000112BF0D801A252F823F000BF35DC000859
:10DBF0005FDC00085DDD000885DD000803DE00084D
:10DC000029DE00088FDE0008B7DE00083DDF0008CF
:10DC1000C7DB0008C7DB000891DF0008C7DB00088E
:10DC2000C7DB000839E0000861E0000899E000085F
:10DC3000CDE00008052002F07BFB70B1052100203B
:10DC400002F03CFB725DBA4BE51C0234E4B283F88F
:10DC50005C24325D83F85D24EDB22C46B1E70023ED
:10DC60008DF80E308DF80F308DF814308DF8183097
:10DC7000B9F1000F6DD1AF4C4FF0050994F87C203D
:10DC80008DF831206B1E94F839208DF83320334401
:10DC900094F838200B938DF8342094F81A3194F8C6
:10DCA00068208DF83520D4F82C218DF832300A9276
:10DCB00073B37B1C5B1BDBB28DF8303006AB01937A
:10DCC00005AB009394F848000DF10F030DF10E021F
:10DCD0000AA903F07BF88DF80D0000F00700072873
:10DCE00013D194F939209DF90E3084F839309A42D5
:10DCF0009DF80F3084F83830B8BF01229DF81430F9
:10DD0000B8BF84F81D2184F868304FF0000A09E09C
:10DD10000523D1E701220DF10D01032002F078F96E
:10DD20000AF1010A5FFA8AF29DF81830B3FBF9F1A3
:10DD30009142EFD82B44DDB26B1EDBB29F420BD970
:10DD4000F25C032A9AD0AF4288BF1D464FF001090A
:10DD500083E70534E5B2F9E71D46F7E7735D7549DA
:10DD600003F00F03012281F81B31023402FA03F39E
:10DD7000A1F82031E4B2002204A9042002F048F9FD
:10DD800025466AE707238DF80D30735DC3F3021251
:10DD900003F00F038DF82830E31CDBB28DF8292047
:10DDA000F25C231DDBB2651DF35C0234E4B21B049C
:10DDB00043EA0223325D5F4C13436422534394F8D9
:10DDC00048000B930AA903F010F800F00703072B93
:10DDD000EDB28DF80D000CD19DF8283084F870302C
:10DDE00084F878300B9BE36663679DF8293084F8EC
:10DDF00069308DF81000012204A9052002F008F90D
:10DE00002BE74B4BD3F8483363B11B6853B19847AA
:10DE100008F03F038DF810008DF81130022204A99C
:10DE20000620EBE7FF20F3E703238DF80D30735D49
:10DE30008DF81C300AAB0693E31CDBB2A51DF25C27
:10DE4000231DDBB206A9F35C1B0443EA0223A21CD8
:10DE5000D2B20534B25C134364225343E4B20A9352
:10DE600000230B93335D8DF83030324B93F848002C
:10DE700002F0C1FFC3B20028EDB28DF80D30FFF6FD
:10DE8000ECAE8DF81030012204A90720B6E7735DCF
:10DE900003F00F03012B4FF47A7238BF0123534371
:10DEA000244A0234936503F57A73D365E4B2002201
:10DEB00004A9082062E7735D1E4DC3F340128DF87C
:10DEC000152095F84800C3F3001205A903F00F03CD
:10DED0008DF814208DF8163002F093FF02340130D3
:10DEE000E4B23FF44DAFBDF81430134AA5F87C30CE
:10DEF0009DF816309DF814A0D05CF4F75BF802236F
:10DF0000C5F880000AA995F848008DF828308DF8EA
:10DF10002AA002F015FF95F93930069040B29842D8
:10DF2000B8BF184685F83900002204A9092025E762
:10DF3000002E00203C2800207164030803238DF884
:10DF40000D30735D8DF82830E31CDBB2651DF25C8B
:10DF5000231DDBB20234F35CE4B21B0443EA022368
:10DF6000325D1343642253430B93644B0AA993F825
:10DF7000480002F04CFFC3B20028EDB28DF80D301E
:10DF8000FFF66BAE8DF81030012204A90A2035E7A8
:10DF9000092002F0CDF9DFF868B1002849D0092145
:10DFA000002002F08BF90023ADF81E30A31CDBB279
:10DFB000F25CE31CDBB216F803A0735D4FEA0A4A79
:10DFC0004AEA022A4AEA030A231DDBB2A51D0534E8
:10DFD000F35CE4B24AEA036A335D4FF47A72534366
:10DFE0000AAC1B122046ADF81C3007F065F8454B13
:10DFF00053440693DBF83C3300930DF1180A9AE87A
:10E000000600DBF8383308A807F012F8099B0093E4
:10E0100094E80600089B504606F0EFFF9AE80300DC
:10E0200007F022F801F0DCFF0123EDB28BF8383461
:10E0300013E68BF8380410E60C2002F079F900287A
:10E040003FF40BAE0C21002002F038F92C4B93F872
:10E050009034043B012B7FF600AE01F0BDFFFCE5E0
:10E06000A31CDBB2725DF15CE31CDBB2651DF35CEB
:10E070000434E4B21B04305D43EA012313436421FA
:10E08000594300F00F0001F0A8FFEDB28DF8100029
:10E09000012204A91120B1E60D2002F049F900285F
:10E0A0003FF4DBAD0D21002002F008F9A31CDBB228
:10E0B000154AF05C735D1268251D0334E4B243EA2F
:10E0C0000020315DEDB201F08AFFC6E5725DA31C50
:10E0D000251D0334DBB2E4B2F15C335D1B0443EA7B
:10E0E000012313436420584301F07BFFEDB28DF808
:10E0F0001000012204A9132080E600BF3C28002064
:10E10000002E0020803DD512D02100200E4B93F828
:10E110009124920703D593F88F24012A08D90B493B
:10E1200091F81A2122B18A6A501C18BF01328A6202
:10E130000022A3F8182483F81A24D3F8402322F0ED
:10E140000202C3F840237047002E00203C28002024
:10E1500070B5184C1848194D07F032F9D4F840330F
:10E16000D4F89804D5F8906023F02003C4F8403325
:10E1700038B107F0EBF8864203D2002385F83A3035
:10E1800070BD0120FFF766F90028F9D00B28F7D001
:10E1900095F8393084F84234092094F8183484F81A
:10E1A000453484F8410402F0ABF8BDE87040FFF755
:10E1B000ADBF00BF002E0020683100203C280020A9
:10E1C000094BD3F84023012A0AD008490978C90726
:10E1D00008D43AB993F89204013818BF0120704767
:10E1E0000020704701207047002E0020E42100200D
:10E1F000034BD3F84003431E58425841704700BFB9
:10E20000002E00202DE9F04FA9B0EFF3108272B676
:10E21000DFF8F0B20021DBF80030CBF8001082F319
:10E220001088B94C002B00F0E180DAB29B06039213
:10E2300064D5B64D95F81831022B02D0B44BDB6A89
:10E240009847EFF3108872B6B24F07F075F83E6842
:10E25000D4F8B013361A3144AF4807F039F9AE4854
:10E2600007F0FCF8D4F8B413AC48314407F030F9A7
:10E27000AA4807F0F3F888F3108894F81A34002BB2
:10E2800000F06B81152312A995F848008DF84830ED
:10E2900002F056FDD4F8B4130F900144A04807F0E3
:10E2A00017F99F4807F0DAF83B6894F81B24EB62F3
:10E2B0000DAF38468DF870201D9306F023FFD5F87A
:10E2C0002831009306AE97E80600D5F82431304691
:10E2D00006F0AEFE96E803001FAB83E80300D4F817
:10E2E0001C341E9395F8303195F84800003B18BF58
:10E2F00001231CA98DF8713002F02BFD039BDF0672
:10E3000048D5824DDFF81CA2D5F8E42004929BF892
:10E310000020BAF90A809AF90C90A4F88C840023A2
:10E3200063F300020A9384F84434A4F8223484F896
:10E330002534C4F82834A4F82C3484F82E34C4F8D6
:10E34000303484F82034C4F8343484F83834C4F8D1
:10E350003C346F4B8BF8002094F89024DB6A84F8EF
:10E360008E9484F88F24DAF80470BAF8086098471D
:10E3700094F88F3413B9694807F022F831463846CB
:10E3800001F017FE8346002800F0EA80A4F87E849E
:10E3900084F88094039B19071AD55C4B93F81831C5
:10E3A000022B02D05A4BDB6A98470220FEF712FF7D
:10E3B00084F8410401F0A4FF94F81A3413B1012346
:10E3C00084F8193494F8913443F0100384F89134AC
:10E3D000039B5A0703D506210520FEF765FF039B23
:10E3E0009B0703D504210320FEF75EFF01F000FE2A
:10E3F00094F89124D7065FD5002384F89234D4F89A
:10E4000040331E0644BF23F08203C4F8403312F0A9
:10E41000050F00F0FB820B2001F08AFF002800F0BE
:10E42000F58294F89134DD0700F1F082580740F14D
:10E430000783D4F8403323F00203C4F84033D4F800
:10E44000402382BB94F8915415F001011EBF2B4666
:10E4500062F3000384F8913494F891345E0744BF6A
:10E460006FF3820384F89134012384F8923421B14C
:10E47000D4F844332C481B6898476D070BD52B48BC
:10E4800001F062FF01F090FF28B194F8913443F05D
:10E49000040384F8913401F098FD94F891346FF3FB
:10E4A000041384F89134012384F8923494F891345D
:10E4B00043F0200384F8913494F8913418070AD576
:10E4C0006FF3C3031A4984F89134D4F84433A1F1AB
:10E4D0002400DB68984794F8913499070AD56FF3C4
:10E4E0004103134984F89134D4F84433A1F16C000A
:10E4F0005B68984794F89034022B1BD1FFF722F900
:10E5000018E000BFE4210020002E00203C2800205D
:10E51000646B0308E0210020803100209831002046
:10E5200000320020D0210020403200205432002050
:10E530008C32002094F891349A0640F1C4826FF333
:10E54000451384F89134D4F84033002B40F0BB825B
:10E5500029B0BDE8F04FFFF7ABBA84F84134A3E629
:10E5600095F81831012B0CD101F027FD804668B1D8
:10E57000584601F017FD584601F019FD042384F8B0
:10E580008F347EB9012384F821344FE101F017FD67
:10E590000028F6D0404601F006FD404601F008FD97
:10E5A0000523ECE73B7805935B09013B062B00F262
:10E5B0001782DFE813F0070015029500150292009C
:10E5C00015020602102EDDD995F830311297F6B2F9
:10E5D0008DF84C60002BD5D11CA804F03FFA12AA8C
:10E5E0001CA9FF2002F072F99DF85830C3F3030311
:10E5F00007468DF82C3095F8480095F87D308DF859
:10E600002D3007220BA902F0AEFB002F5DD10028B0
:10E610005BD09DF853309DF852201599C5F8E41051
:10E620001B0443EA02239DF8512002201343C5F83E
:10E63000E03004F021FA9DF8583095F8480085F84C
:10E640002E71C3F30212C3F3030385F8703085F80B
:10E6500078309DF8593085F86920012B38BF0123A7
:10E660004FF47A725343AB651344EB650DF15A03D3
:10E670004FF001081093113E94F81B348DF83C3094
:10E680000FA985F868808DF8446002F074FB0223BE
:10E69000404685F8303101F04BFE18B1414638460E
:10E6A00001F00CFE94F88F34012B00F2A78194F84E
:10E6B0001A34002B40F09A8194F8913443F01003FF
:10E6C00084F89134FEF786FD64E6012001F030FE07
:10E6D0000028E7D001210720E2E7012384F8203455
:10E6E00095F87D308DF82E3094F824348DF82D3047
:10E6F00095F88C3095F848000D330BA98DF82C3027
:10E7000002F01EFBA6F10D031BB2099023EAE3738E
:10E7100000B283423FF736AF0B2E7FF633AFBA4BD2
:10E7200025931CA8FF231C978DF874608DF89830F2
:10E7300002F0E2F9074600287FF424AF95F818317B
:10E74000012B13D101F039FC002872D0384601F0BA
:10E7500029FC384601F02BFC04239DF87C101E9800
:10E7600084F88F34C1F3001101F041FC9DF87C3036
:10E770001E99C4F8341413F00F0203D09DF89000D2
:10E78000002862D19DF89800002861D0002A7FF40B
:10E79000F9AE9DF89020002A14BF4FF003084FF007
:10E7A000020800220A92D5F8EC2095F8E90091427F
:10E7B00051D100284FD0D5F80C1195F8EAB009686E
:10E7C0000A9195F81811022902D1032184F88F14B7
:10E7D000B8F1030F7FF4D6AE13F0600F7FF4D2AE22
:10E7E0000492012795F82E31BBF1000F36D0BBF112
:10E7F000010F13D1012B33D16FF0090646FA08F649
:10E8000006F00106C6F10206F6B2BDF87E100AAAAD
:10E81000304601F0E5FE38B3072823D0012384F801
:10E8200021340A9BC4F83034C4F86C34FEF720FD60
:10E83000B0E501F0C4FB002898D0384601F0B3FBE6
:10E84000384601F0B5FB052387E74FF00008A8E73D
:10E850004FF00108A5E74FF0010BC3E70426D4E70A
:10E860000326D2E70823DAE71CAB009304990A9B3E
:10E870003246584601F076FF20B1022814BF0B2320
:10E880000A2380E60A9BC4F83034C4F86C349DF83F
:10E890007C3084F82104C3F3401384F82E3484F8C8
:10E8A000443494F88F3484F82274012B9EBF0122E3
:10E8B000A86285F81E21012FC4F8280484F82C04CE
:10E8C00084F8410438D1022284F8202495F83A20B3
:10E8D000002A4AD19DF87C20D60646D4012B94F814
:10E8E00040149DF87C2005D8012901D1900601D55E
:10E8F00001F020FCB8F1020F94F88F3443D0B8F146
:10E90000030F0AD09DF87C10B8F1010F4A4601F0C0
:10E910000F0120A83BD0FFF745F99DF8903084F80F
:10E920002334259BC4F828349DF8983084F82C347F
:10E93000012384F82D3430E0059A02F0E002A02A89
:10E940001BD195F82E11012285F83A2009B9279993
:10E950006963012B84F8202407D9D5F89020C4F8E6
:10E960003C24DAF80020C4F8982495F81821002AED
:10E97000B4D1012284F82524B0E7002285F83A209A
:10E9800084F82024A6E79DF8981025984A46FFF7BA
:10E9900009F99DF8903084F823349DF89020E02AFE
:10E9A00008D195F81F312BB984F82324C4F82834F2
:10E9B000A4F82C3494F8913443F0020384F8913491
:10E9C00070E6114D013EB2B2791C284604F01EF9E2
:10E9D0000323A4F82034C4F8285484F82C64E9E70D
:10E9E000012384F82134FEF743FC5BE694F84434B9
:10E9F000002B3FF461AE0020FEF726FC94F88F3424
:10EA0000022B3FF45FAE57E63830002094F8913483
:10EA1000590715D5012001F08BFC60B1012001F0F0
:10EA20005FFC08B984F81804D4F8403323F00203DB
:10EA3000C4F8403304E0062001F07AFC0028F3D14A
:10EA400094F89134DA077FF5FAAC94F840240AB1CF
:10EA5000032A18D11D4A94F8181492F8682091429C
:10EA600005D29B0723D594F88F34012B1FD8184863
:10EA700006F0A6FCD4F8403323F02003C4F840335A
:10EA8000FFF744FBDBE4012A11D194F81924002A92
:10EA90003FF4D5AC0D4A94F8181492F868209142CE
:10EAA000E5D29F0703D594F84434002BDFD194F8C6
:10EAB000913400206FF3041384F8913484F819041E
:10EAC000FFF746FBBBE429B0BDE8F08F3C280020EF
:10EAD000683100202DE9F04F89468DB090460746F9
:10EAE000002800F08F81002900F08C810368002B42
:10EAF00000F088814368002B00F084818368002B3C
:10EB000000F08081C368002B00F07C81104602F089
:10EB100013F9002800F07881BD4CBE4D384601F055
:10EB200083FB40F2C4520021204604F083F840F2F7
:10EB30001C520021284604F07DF8B74BC4F82C3154
:10EB400004F50973089304F50A73002640460993F7
:10EB500008A9B24B84F848800A9384F8186184F8B5
:10EB60008C608DF82C6002F0F9F80F2306A994F858
:10EB700048008DF8183002F0E3F8801B18BF012020
:10EB80004FF00A0B84F81C0106A994F848008DF890
:10EB900018B002F0D5F84FF0060A84F8DC0006A998
:10EBA00094F848008DF818A002F0CAF8102384F8F1
:10EBB000DD0006A994F848008DF8183002F0C0F87E
:10EBC0001123C4F89C0006A994F848008DF8183069
:10EBD00002F0B6F81223C4F8A00006A994F8480081
:10EBE0008DF8183002F0ACF81323C4F8A40006A97D
:10EBF00094F848008DF8183002F0A2F81423C4F8F5
:10EC0000A80006A994F848008DF8183002F098F88A
:10EC10001623C4F8AC0006A994F848008DF8183003
:10EC200002F08EF8172384F8B10006A994F8480082
:10EC30008DF8183002F084F818230DEB0301C4F8A6
:10EC4000B400C4F8BC0094F848008DF8183002F005
:10EC500077F8C0B21D2384F8B80084F8C00006A974
:10EC600094F848008DF8183002F06AF81E2384F8F2
:10EC7000C40006A994F848008DF8183002F060F836
:10EC80001F2384F8C50006A994F848008DF81830B1
:10EC900002F056F82023C4F8C80006A994F84800EA
:10ECA0008DF8183002F04CF80B23C4F8CC0006A9FC
:10ECB00094F848008DF8183002F042F80C2306A9A9
:10ECC000A4F8D00094F848008DF8183002F038F815
:10ECD000D4F89C306365D4F8A030A365D4F8A43090
:10ECE000E365D4F8A83023664FF00108D4F8AC30BF
:10ECF0000590A4F8D200636684F8B080C4F894B09C
:10ED000084F898A0C4F84CB084F850A084F86880C7
:10ED100084F81F81C5F84893FEF7AEFDC5F844732B
:10ED2000C4E90B663E4B84F8198185F89164C5F8F7
:10ED3000408332464FF0FF31009605F55A7006F0D9
:10ED4000E1FA384B009632464FF0FF3105F560701E
:10ED500006F0D8FA344B009632464FF0FF3105F5F5
:10ED6000667006F0CFFA02AF304B009632464FF095
:10ED7000FF3105F5806006F0C5FA384606F0C2F9A5
:10ED800097E8030004F5927383E80300284B294FAA
:10ED90001E60294BC5F84C33284BC5F85433284B1B
:10EDA000C5F85C33274BC5F85033274BC5F85833AB
:10EDB00005F553703B68984704F5A67003F06AFCAC
:10EDC00020B1112630460DB0BDE8F08F204601F08D
:10EDD000D7FB0028F5D101F00DF9B8B91B4801F0B7
:10EDE00021FC06460028ECD17B69984703F0ECFE35
:10EDF000BB6D94F819019847FB6A9847012385F881
:10EE00009234DFE70326DDE70926DBE71326D9E79F
:10EE10003C280020002E002000040001E8210020F2
:10EE200051E1000819DA000861DA000849D2000847
:10EE3000E4210020646B030809D40008BDD3000856
:10EE400005D2000895D300086DD3000824290020BE
:10EE500008B5034B0020C3F84003FEF7BBF908BD1B
:10EE6000002E002010B5FFF7ABF90A4C60B90A4B31
:10EE700093F81831022B02D1084BDB6A9847012323
:10EE8000C4F84033002010BDD4F84003013818BF47
:10EE90000120F8E7002E00203C280020646B0308C6
:10EEA00038B5124C204606F08BFA04F1180006F033
:10EEB00087FA04F1300006F083FA04F1980006F0B6
:10EEC0007FFA01F081F80A4B0025DB6A984744F885
:10EED000285CFEF7EDFD0749074840F2C45203F0F5
:10EEE00095FE012344F8283C284638BD68310020AF
:10EEF000646B03083C2800207822002070B52E4B5C
:10EF00008AB0054693F8DD008DF8090093F8DC001F
:10EF10008DF80A0029489A6A90F81804039200268E
:10EF20008DF80B0004960C46002940D00692D3F8C9
:10EF3000882007921A8F93F81A118DF8151052BA7B
:10EF4000ADF8202093F87C2093F848308DF82430D9
:10EF500003AB8DF822008DF8232000930DF10A02F7
:10EF60000DF10B030DF1090105A88DF8146000F0F7
:10EF7000A9FF9DF90900FEF74FF9607004A801F0A0
:10EF8000EFF8B0B9049A0F2A0DD863789A420AD8DC
:10EF90001544AB42A3EB02012CBF002001202170DD
:10EFA000C0000AB070BD002323700820F9E70320D9
:10EFB000F7E71320F5E700BF3C280020002E0020D3
:10EFC0001FB50446002800F010810378412B00F2A1
:10EFD0000781DFE813F0420049004D005100550061
:10EFE00059005E0005010501050105010501050146
:10EFF00005010501650069006D0078007F00820051
:10F0000085008A0088008C0090009300960099008B
:10F010009C009F00AE00B200BA00B600BE00C10066
:10F02000C500CE00CA00CC000501D20005010501D3
:10F0300005010501050105010501050105010501A0
:10F0400005010501050105010501DA00DE00E20008
:10F05000E700EB00EF00F300FC00664B93F818317B
:10F060002371002004B010BD624B93F83031F7E7F4
:10F07000406803F0ADFCF4E7406803F0EFFCF0E714
:10F080005C4B93F81A31EBE75A4BD3F8E0306360EE
:10F09000E7E7584B011D93F8300103F0F7FCE0E778
:10F0A000544B93F81931DBE7524B93F88C30D7E788
:10F0B0001C238DF808304F4B02A993F8480001F04B
:10F0C0003FFE6060CDE74C4B043493E8030084E8D6
:10F0D0000300C6E7494B0434F7E7494B0434F4E72F
:10F0E000484B0434F1E71A23E3E71923E1E7414BE6
:10F0F00093F86830B4E73F4B5B6DC8E73D4B9B6DC1
:10F10000C5E73C4BDB6DC2E73A4B1B6EBFE7394BA3
:10F110005B6EBCE702238DF80830364B02A993F8EA
:10F120007C2093F848008DF80A2001F009FE207138
:10F1300097E7304B93F8DD3092E72E4B93F8393058
:10F140008EE72C4B93F8DC308AE72A4B93F8383063
:10F1500086E7284BDB6C9AE7264B93F850307FE725
:10F16000244BD3F8843063607BE7224B8FE7264B38
:10F170008DE7204BD3F8CC30F5E71E4BD3F82C317C
:10F18000436001F06BFEA0606BE71A4BD3F8903040
:10F190007DE7184B93F81F3162E7164BB3F88830C0
:10F1A000A3805EE7134BB3F88A30F9E7114BB3F84D
:10F1B000D030F5E70F4BB3F8D230F1E70D4B93F8B1
:10F1C00048200AB1062A12D1B3F8A035E8E7094B66
:10F1D00093F848200AB1062A09D1D3F8A43556E796
:10F1E00004B0BDE8104000F0F3BE03203AE7182059
:10F1F00038E700BF3C280020A8280020F028002085
:10F20000B0280020F8280020782200207FB504468E
:10F2100010B9032004B070BDA34DD5F840339A0750
:10F2200000F16F820278412A00F26882DFE812F072
:10F230004200470055005B005F00640069007600F3
:10F24000810087008D00930099009F00A500AB000E
:10F25000B5006602BA00DC00EF0016013801290192
:10F2600042014B014F01530157015B0166025F01EF
:10F27000710199018701AB01B101B801BD01C20162
:10F28000660228026602660266026602660266027C
:10F29000660266026602660266026602660266022E
:10F2A00066026602340239023E02430248024D02FF
:10F2B00052025C020079FEF773FA30B1AAE70379D3
:10F2C000022BA6D0794A82F8303195F8913443F078
:10F2D000200385F8913400209CE7406803F06AFB26
:10F2E0000028F2D095E7406803F0A8FBF8E76F4BE1
:10F2F000027983F81A21E8E76C4B4268C3F8E020F2
:10F30000E3E76A4E416896F8300103F0B5FB002848
:10F310007FF47FAF6368C6F8E430D6E74168002920
:10F320003FF477AF002001F0B1FA0028CDD01120D2
:10F3300070E7416800293FF46CAF0120F3E74168B2
:10F3400000293FF466AF0820EDE7416800293FF44B
:10F3500060AF0920E7E7416800293FF45AAF0C206D
:10F36000E1E7416800293FF454AF0D20DBE7416835
:10F3700000293FF44EAF0E20D5E7416800293FF445
:10F3800048AF0F20CFE74A4C484B007983F819016A
:10F39000A36D9847E36A984797E7444B027983F84F
:10F3A0008C2092E7414E037A8DF8043096F848009D
:10F3B00096F87D308DF80530072201A901F0D3FCC5
:10F3C00000283FF426AF636896F8480001930022B6
:10F3D00001A901F0C8FC00283FF41BAF6C36D4E94A
:10F3E000010186E8030070E7304E037A8DF804309F
:10F3F00096F8480096F87D308DF80530072201A96F
:10F4000001F0B1FC00283FF404AFB436E7E7274E23
:10F41000037A8DF8043096F8480096F87D308DF820
:10F420000530072201A901F09EFC00283FF4F1AE4F
:10F43000D4E9010106F1740383E8030096F818315A
:10F44000022B7FF442AF96F83031002B3FF43DAFF2
:10F45000174BDB6A9847FEF775F936E7134E037AC8
:10F460008DF8043096F8480096F87D308DF8053018
:10F47000072201A901F077FC00283FF4CAAEBC3690
:10F48000ADE74368029301238DF80C30074B02A9C6
:10F4900093F8480001F074FC00287FF416AFB8E63A
:10F4A000436802930023EFE7002E00203C28002051
:10F4B000646B030803795A1E0E2A3FF6AAAE934ADC
:10F4C00082F8683001E7914B42685A65FDE68F4B40
:10F4D00042689A65F9E68D4B4268DA65F5E68B4B32
:10F4E00042681A66F1E6894B42685A66EDE6874C37
:10F4F000037994F848008DF80430062201A901F040
:10F5000032FC00283FF485AE9DF8043084F8DD30ED
:10F51000DBE67E4C03798DF8043094F8480094F8CB
:10F520007C308DF80630052201A901F01CFC002872
:10F530003FF46FAE9DF8043084F83930C5E6734C63
:10F54000037994F848008DF804300A2201A901F0EB
:10F550000AFC00283FF45DAE9DF8043084F8DC30EE
:10F56000B3E66A4C037994F848008DF80430092218
:10F5700001A901F0F8FB00283FF44BAE9DF80430E0
:10F5800084F83830A1E6614B4268C3F89420DA640D
:10F590009BE65E4B027983F8982083F8502094E62E
:10F5A0005A4B4268C3F884208FE6584B4268C3F830
:10F5B000CC208AE6012B40F0A480554C2421204623
:10F5C00003F03AFB636A984201D0172022E61C211F
:10F5D00004F1280003F030FB636C9842F5D14FF43E
:10F5E000807104F1480003F027FBD4F848319842B9
:10F5F000EBD1D42104F5A67003F01EFBD4F8203221
:10F600009842E2D1002104F5097003F015FBD4F80B
:10F6100024329842D9D14FF4607104F50A7003F096
:10F620000BFBD4F8A8359842CFD1142104F2AC508A
:10F6300003F002FBD4F8C0359842C6D1334E2146C0
:10F64000304640F2C45203F0E1FA204640F2C45280
:10F65000002103F0EFFA95F81B3485F8E833736F57
:10F66000C5F8EC3396F87D3085F8F83340F2012385
:10F67000A5F8FA33274B96F819019B6D984724E6B5
:10F680008379012B3FF6C5AD204B42684068C3F833
:10F690002C2100F091FF48E61C4B4268C3F89020F3
:10F6A00013E61A4B027983F81F210EE6174B828866
:10F6B000A3F8882009E6154B8288A3F88A2004E67F
:10F6C000124B8288A3F8D020FFE5104B8288A3F864
:10F6D000D220FAE50D4B93F848200AB1062A12D140
:10F6E000A288A3F8A025F0E5084B93F848200AB1BA
:10F6F000062A08D16268C3F8A425E6E500F06AFC92
:10F70000DBE5012086E5182084E500BF3C280020C9
:10F7100078220020646B0308DFF880C0F8B5DCF8BD
:10F7200040339B07064635D48778002F34D10546F1
:10F730000FCD1B4C0FC40FCD0FC42B6823609CF85A
:10F740009134B16843F020038CF891343378BBB125
:10F750000D2001F09BF810B111273846F8BD7168F3
:10F76000B07801F031F90028F6D1B2780D4B302194
:10F7700001FB02334FF0FF32D3F80C311A60ECE793
:10F780000E2001F083F80028E6D1F1680F2001F087
:10F790007DF8E8E70127E0E71627DEE7002E0020E6
:10F7A000242900203C280020F0B5134FD7F840331F
:10F7B0009B078BB006461AD4D8B9104C94F8E930A0
:10F7C000BBB10146242201A801AD03F033FA0FCDED
:10F7D000E8340FC40FCD0FC42B68236097F8913421
:10F7E00043F0200387F8913430460BB0F0BD01267A
:10F7F000FAE71626F8E700BF002E00203C2800207C
:10F8000000F00303F7B51C33294F13701546D7F8E2
:10F81000402392070C4647D40A78013A012A03D9BB
:10F820000325284603B0F0BD00283FD1214E96F8AD
:10F83000E920002A3AD003F00F032B7091F9083029
:10F840008DF8043096F8480096F87D308DF8053034
:10F85000072201A901F087FA18B12B7823F00403DD
:10F860002B70636896F848000193002201A901F00B
:10F870007AFA18B12B7823F008032B702D78002D1D
:10F88000CED194E807000C4B83E8070097F8912449
:10F8900042F0200287F891242278012AC1D1A3F1F5
:10F8A000180000F0A3FBBCE70125BAE71625B8E76E
:10F8B000002E00203C2800203C2900202DE9F043A8
:10F8C00087B00023ADF800300646002800F0EE8037
:10F8D0000361FEF775FC20B10124204607B0BDE8A6
:10F8E000F08300F067FD0028F6D100F05DFD0146D1
:10F8F00018B96F48142203F09DF96E4D95F89134B4
:10F90000012243F0040385F8552485F891343378B7
:10F910008DF804300021013B8DF80520ADF806106C
:10F920000C2B00F2BB80DFE803F007B9B9B979828C
:10F93000B9B990B9AD9AA900D5F8407317F020076E
:10F94000CAD196F80480B8F1020F46D1DFF8688179
:10F950005A4CFDF791FF96F9051098F848003A4681
:10F9600001F05BFA88F83900B37988F83830384606
:10F9700007238DF80530FDF713FFFF2304F586708C
:10F98000A5F80C31C5F8084185F8047103F066F854
:10F9900004F58A7003F01CF83846FDF75BFD044659
:10F9A000002839D096F9051098F84800012201F096
:10F9B00034FA88F83900D5F894343361002C71D0CA
:10F9C00000F0F2FC002888D195F8913485F81A04EB
:10F9D00060F3820385F891347FE7B8F1010F4FF0AF
:10F9E0000204E8D1DFF8D0908DF8144099F848006F
:10F9F00089F81D7102A901F0B1F9337989F8303124
:10FA00008DF805708DF80680FDF7F2FB95F89134BE
:10FA100043F0100385F891340024CCE700226946B6
:10FA2000022000F0F5FA0028F6D01324C3E7244B97
:10FA3000B288DB6B96F90C10B0689847D5F8403364
:10FA400043F00203C5F84033E6E702A90D2000F0B9
:10FA500055FB0028E0D0002269460D20E1E7164B57
:10FA600093F81831D3B9347904F0070000F0ABFAF9
:10FA70008DF80040012269461020D2E70022694635
:10FA80001220CEE78DF8072000F08EFA044638B930
:10FA900000F087FA204600F089FABDE702248AE7E1
:10FAA000012488E701A800F0D3FB16E7032414E73C
:10FAB00054320020002E00203C280020022E00207E
:10FAC000646B03082DE9F04F99B08046059118B991
:10FAD000032019B0BDE8F08F00230361FEF770FB2F
:10FAE0000446002840F0A58046460FCE0EAD0FC557
:10FAF0001422524898F800A0B8F80C7098F90EB08B
:10FB00004F4E214603F096F84E4B012283F84124D4
:10FB100096F83021022A25460BD196F81821022AA0
:10FB200007D196F81E2122B9BAF1010F38BF4FF064
:10FB3000010ABAF1010F2BD0BAF1030F2AD0BAF1A2
:10FB4000000F33D102229DF83C30DDF84090029343
:10FB500062F34715012496F87C108DF832100222CA
:10FB60000CA996F848008DF8302001F0E9F896F8D5
:10FB70001A3196F830C196F81D1140B2002B63D0AF
:10FB8000BCF1010F57D1002955D1002C61D153E0B0
:10FB90000422D8E70023DDF83C90BDF840709DF9C1
:10FBA00042B0029365F01F050124D4E74FF0000B2B
:10FBB000D946CDF808B0CEE74FF0010084F81A041A
:10FBC000D2E005F29A420BA900F0D6FA002800F024
:10FBD00015811320049B33871A4B002283F81A24C3
:10FBE00023E105F29A452A460BA900F0C5FA002840
:10FBF000EFD10B9B84F82801C4F82C5184F83031E4
:10FC0000FCE0B9F1000F00F0F980002A00F0F68066
:10FC10004946E01C02F0FAFF94F8373201332380A2
:10FC2000ECE01220D6E70220D4E70720D4E7132027
:10FC3000D2E701204DE7FCB90220F6E04032002077
:10FC40003C280020002E0020002CF5D05845B8BFDD
:10FC5000584696F87C308DF82000052296F848002A
:10FC60008DF8223008A901F07EF800283FF430AF6B
:10FC70009DF8203086F839306F4A704BD2F89804DE
:10FC8000D3F8904038B105F061FB6C4B84423CBF27
:10FC9000002283F83A20198F1A8F93F830010491CB
:10FCA000996A099152BA0028BFD093F81B0100B994
:10FCB000186393F81801ADF85820013893F87C20A8
:10FCC00093F81A411491D0F1000BD3F888108DF8F5
:10FCD0005B204BEB000B93F8482093F83A0093F825
:10FCE00068308DF85A3009AB0093554B03904FF0B4
:10FCF00001008DF84C0015918DF85C20A3F12F01C7
:10FD0000A3F1300213A88DF84D4000F0DBF8039BFF
:10FD10004FEA0B1B4BEA431B00264BEA801B4BEAC6
:10FD2000C413B145444C039308BF37463A4649468D
:10FD300004F59C70CDE90A669B46268084F81A6417
:10FD400002F064FFE9B2A570C5F34215FAB2042DC2
:10FD50003A4E039B84F837223FF42EAF072D3FF431
:10FD600050AF022D7FF45FAF364D84F80D110420A3
:10FD7000029984F80401FF2084F80C0184F828110A
:10FD800084F81431D6F8E410C4F8085105F59B73D3
:10FD90000AA8C4F8101184F83021C4F82C3100F0FE
:10FDA00013FC00287FF43DAF0A9BA4F844040BA881
:10FDB000A4F81631C4F84C3400F0D2F900287FF4CE
:10FDC00008AF0B9BD3B196F93900FDF725FA94F8EB
:10FDD0003732002B3FF405AF0B9B0F2B3FF6F1AEF4
:10FDE00005F58B720BA90F2000F0C6F900287FF4EF
:10FDF000F0AE0B9B63F3030B84F814B10598FDF789
:10FE000029FB00287FF4E6AE099B86F83A00B3622E
:10FE100000F082F900287FF40AAF94F8913484F856
:10FE200040A443F0010384F89134034BD3F8943495
:10FE3000C8F810304DE600BF002E00203C280020FE
:10FE4000A4280020022E002037B50B4D8DF80400A9
:10FE500004460F2295F8480001A900F084FF40B144
:10FE6000064A85F81C4192F8913443F0200382F849
:10FE7000913403B030BD00BF3C280020002E00208C
:10FE800010B5FEF7EFFF044688B90A4805F098FA66
:10FE9000094805F095FA094805F092FA00F094F83F
:10FEA000FDF7EAFC064BDB6A9847204610BD0124AB
:10FEB000FBE700BF6831002080310020983100202E
:10FEC000646B03082DE9F04F8BB047780093149BC7
:10FED00090F90C8090F90D6090F80EB08A46416858
:10FEE000196004469146002F58D002238DF8103037
:10FEF00004A9C37B007C8DF8123000F021FFB4F818
:10FF000008C0618943B26068984545466144B8BFFE
:10FF10001D46604534BF00270127884209D30A21C6
:10FF20008DF81010207C019304A900F009FF019BBB
:10FF300046B2B4F808C0608961680CEB400E7145A8
:10FF400019D3A1EB0C01B1FBF0FC00FB1C1191B922
:10FF5000984503DC2378CBB94FF0010B21238DF8B2
:10FF60001030207CE37B8DF8115004A98DF81230FD
:10FF700000F0E6FE45B2009B8AF80050384689F84A
:10FF8000006083F800B00BB0BDE8F08F0223207C46
:10FF90008DF8243006A900F0E1FEDDE74546EAE7EA
:10FFA0007047704770477047002070477047704730
:10FFB00070470020704700207047002070470020E5
:10FFC00070470020704770477047704702207047A5
:10FFD000022070470220704770470020704770472A
:10FFE0007047002070470020704770477047704787
:10FFF0007047000010B5054C4FF4037220460021F5
:020000040801F1
:1000000002F018FE0020C4E9000010BD1C330020DF
:100010002DE9F8438146904600293CD01F4C20230F
:10002000224604F1100012F8017F6FBB8242FAD120
:100030001B4E3368013403B93460736803B11C602C
:1000400000252560C4F8088074601FFA88F284F8DF
:100050000490601D02F0DAFDB9F1110F4FF00003BA
:1000600098BF104D6373D6F8083298BF25FA09F58A
:1000700003F1010398BF05F0010543442573C6F859
:1000800008323846BDE8F883013B13F0FF0304460D
:10009000C6D10227F5E70127F3E700BF233300208D
:1000A0001C3300202007020010B518B3124A136851
:1000B000984204D103681360002305E00B46002B2F
:1000C000FAD019688842F9D15168884208BF536054
:1000D0000BB101681960D2F808328168013B002435
:1000E0005B1A04602146C2F80832102202F0A2FD19
:1000F000204610BD0120FCE71C330020054B1B6887
:1001000013B11A798242FAD1002B0B600CBF032085
:10011000002070471C33002010B5054B186800B94B
:1001200010BD037B04680BB9FFF7BEFF2046F6E75E
:100130001C33002038B5084B084C186800B938BD8E
:1001400003790568112B05D824FA03F3DB0701D5E1
:10015000FFF7AAFF2846F1E71C3300202007020022
:1001600028B1044BD3F80832036000207047012007
:10017000704700BF1C3300202DE9F04107460E46B2
:10018000154642B339B3154B1C6800232CB93046D1
:10019000FFF7E6FF0020BDE8F081A268F91A0132FE
:1001A000914215D32279EA54581C22895FFA80F8CB
:1001B000611D55FA80F002F029FDA3682468984477
:1001C0005FFA88F3E2E720462568FFF76DFF2C46CB
:1001D000002CF8D1DBE70120DDE700BF1C33002055
:1001E0000238C0B211289ABF014B185C002070473A
:1001F0008164030830B50B4B93F820200446084671
:1002000072B100211C330578A54208D00131984213
:10021000CDB214BF04301038AA42F4D8002030BD4B
:100220001046FCE72835002010B5084C002320605C
:10023000142204F10C00FF2184F82030C4E90100ED
:1002400002F0F8FC012384F8213010BD283500208D
:1002500010B50E4A92F82010042915D89368047836
:100260001C7044785C70C478807898700131DC70C0
:1002700082F8201002F11C018B4214BF043302F1FA
:100280000C039360012010BD0020FCE728350020FE
:10029000094B93F8200068B15A6803F11C018A42A7
:1002A00000F1FF3014BF043203F10C0283F8200088
:1002B0005A600120704700BF2835002010B5074B59
:1002C00093F820200446084632B15968FFF792FFA0
:1002D00010B101234470837010BD00BF2835002089
:1002E00008B5064B93F820202AB15968FFF782FF22
:1002F00008B1407808BD0120FCE700BF2835002088
:1003000030B50A4A92F82010536882F8210061B192
:10031000916801241C32DD78587005B99C709342B5
:1003200014BF0433103B9942F5D130BD283500206D
:1003300008B5044B5968FFF75DFF003818BF01206E
:1003400008BD00BF28350020F7B50422154E04462D
:1003500000210DEB020096F8207002F06BFC0025E6
:10036000EBB29F4201D803B0F0BD736819782170D9
:100370005A786270987838B1336820469B689847FD
:10038000FFF786FF0135EBE7DB788DF804108DF879
:1003900005208DF80730FFF77BFF01A8FFF758FF16
:1003A000F0E700BF28350020014B93F8200070478C
:1003B00028350020034B93F82000042894BF002028
:1003C00001207047283500201FB50024CDE90244E4
:1003D000C41F8DF800408DF801100C0AADF8042000
:1003E000090C120C8DF803108DF806208DF80730DB
:1003F00002461B0A012168468DF802408DF808303C
:1004000002F073FA002818BF0E2004B010BD2DE9C9
:10041000F04188B090460D460F9A0746002847D015
:1004200000240121CDE904448DF810109DF8381006
:100430008DF81510ADF81630190CCDE900441B0EDF
:10044000CDE902448DF81930ADF81A20130C120EC4
:1004500007948DF818108DF81C308DF81D20E3B22C
:100460001E01002DF6B203DC002008B0BDE8F081CB
:10047000013310218DF81F3042466B460DEB010011
:1004800002F0C9F90346A8B9102D28463E44A8BF7A
:1004900010206946327811F801CB013382EA0C0250
:1004A000984206F8012BF5DC103D2DB20134D6E759
:1004B0000920DAE70E20D8E70138032815D8DFE84D
:1004C00000F002080C100A4B1B681B690B6000202F
:1004D0007047074B1B685B69F8E7054B1B689B6916
:1004E000F4E7034B1B68DB69F0E70520704700BFAA
:1004F0004C3500202DE9F041C4B00C464A9E174609
:100500001D468046B8B3B1F5807F36D84FF4887267
:100510000021684602F08EFB492300934FF480735C
:10052000ADF804302B0C8DF80830330CADF80650C4
:10053000ADF80A608DF80C3022460023414604A82D
:100540002D0E360E8DF80E308DF809508DF80D6099
:100550008DF80F4002F05AFB04F110014B9A3B4614
:1005600089B2684602F041F910B1012818BF0E2087
:1005700044B0BDE8F0810920FAE70D20F8E700005B
:1005800010B590B10A4C28220021206002F052FBE5
:100590002368084A1A6000204FF0FF32C3E90302C3
:1005A000C3E90522C3E9072210BD0820FCE700BF0C
:1005B0004C35002000010101024B1B68186000202F
:1005C000704700BF4C35002030B1044B1B68DB681E
:1005D0000133036000207047092070474C3500202C
:1005E00013B500230C460193CAB101A9FFF764FFBC
:1005F00018B9019B591C02D1146002B010BD99B208
:10060000611A002901DD5C18F6E702D113600720AA
:10061000F3E71B0C1B0403F580331C44ECE70920B3
:10062000EBE7000028B1044B1B681C334362002039
:1006300070470920704700BF4C3500201FB50446A5
:1006400000B3002303A8039302F0A6F9104ABDF8F3
:100650000C30126820469380E38200F0A8FA98B923
:1006600004F11803009321680123132202F0B2F869
:1006700060B9204600F09BFA003818BF0120000145
:1006800004B010BD0920FBE71020F9E70E20F7E7C2
:100690004C350020F0B5054687B01C4613B909203B
:1006A00007B0F0BD2E4E3368DB68834255D894F80E
:1006B0002020002A0CBF08220922834205D32046AD
:1006C00000F0A9FA68B11020EAE700230190009336
:1006D000A36894F82810606AFFF799FE0028EED00E
:1006E000DEE723792168B4F808C0A768043B9AB212
:1006F0000029D4D0B2F5807F2DD8ADF80EC08DF88A
:1007000017304FEA174C04F12C033F0E8DF811708F
:1007100000932F0C08234FF0490EADF80C008DF814
:1007200014708DF816002F0E0DEB0300CDF808E0C5
:100730008DF810C0ADF812508DF8157002F04AF81F
:1007400008B10E20ACE7204600F065FA0028BAD1C7
:100750003368DD60A4E70D20A2E70620A0E700BF14
:100760004C3500202DE9FF410A9D80460F46164674
:100770001C46002D5AD0002303A910460393FFF70F
:100780009BFE18B1062004B0BDE8F081039B9C429B
:1007900001D80133F6D1284600F0AEF9002847D140
:1007A000264B1A78424503D01A79424542D101209E
:1007B000AA68BA4240D103EB8002EB6A92F801804A
:1007C0002979CDE900430439927828683B4689B2FB
:1007D000FFF790FE0028D6D195F820300194002B29
:1007E0004FF00103009314BF4246082295F82810E9
:1007F000686A3B46FFF70BFE0028C4D1013E032E7A
:10080000C1D8DFE806F002070B0F0D4B1B681C6117
:100810001C62B8E70A4B1B685C61F9E7084B1B6870
:100820009C61F5E7064B1B68DC61ACE70920AAE791
:100830000F20A8E70B20A6E70220A4E7FC01002078
:100840004C3500201FB50B294FF00003CDE90033D4
:10085000CDE902330A4607D00C2914D00A2910D05A
:100860000A2005B05DF804FB012802D120238DF891
:1008700000300021684602F038F8002818BF0E202A
:10088000EFE73023F3E70B21F4E7000038B5054626
:1008900002F026F8044610B10E24204638BD002D83
:1008A000FBD1094B1B680B219878FFF7CBFF002881
:1008B000F2D10C21FFF7C6FF0028EDD10A21FFF786
:1008C000C1FF0028E9D0E7E74C3500202DE9F043CF
:1008D00080468FB00C461746002A6BD0002969D09D
:1008E000002529461D2206A805951EF097F88DF8CB
:1008F0001350344D2B680DF114099E88CDF80490E7
:100900000DF1130302933B7900933B683246214675
:10091000404602F006F800284ED138683A79494638
:1009200002F074F9384600F099F8002846D13C7A74
:10093000FA79BB79240444EA02241C432B689A68A0
:1009400094423DD99C609DF813000B21FFF77AFF7C
:10095000034658BB0C21FFF775FF034630BB0A2145
:10096000FFF770FF034608BB7B7ABA7AFF7A3F0431
:1009700047EA02271F433A46334621460920FFF73C
:1009800023FD034690B933463A4621460820FFF737
:100990001BFD034650B92A689DF813109170002181
:1009A000D1604FF0FF31C2E90411916118460FB0D8
:1009B000BDE8F0830923F9E70E23F7E70F23F5E7F6
:1009C0000323F3E74C35002070B588B000293FD0F1
:1009D000214C2378834231D0237983423AD10122BA
:1009E0000023CDE90133CDE9053304EB8204039301
:1009F00007930123C1F30720CDB28DF80030C1F376
:100A00000743090E8DF802008DF8041002268DF8B8
:100A100012008DF814106278E1788DF80150684664
:100A20008DF803308DF810608DF811508DF813306B
:100A300001F05BFF20B10E2008B070BD0022CFE7AF
:100A4000A278E17804A801F050FF0028F4D0F2E782
:100A50000920F1E70B20EFE7FC01002010B5044668
:100A6000002845D00168002942D011F8013B4371AC
:100A70000322063002F0CAF82046032250F8091B70
:100A8000043102F0C3F82168CB79E3600A7A43EAC3
:100A90000223E3604A7A43EA0243E3608A7A43EA44
:100AA0000263E360CB7A23740B7B63742379212B7D
:100AB0001AD110220D3104F1120002F0A7F81D2204
:100AC0002168501C8B5C6362085C43EA0023901C25
:100AD0006362085C033243EA004363628A5C43EA70
:100AE00002636362002010BD112B03DC0D22E7E7D7
:100AF0000220F8E70120F6E710B50446002854D09C
:100B00000168002951D00B7843714B7883608A7853
:100B100043EA02238360CA7843EA024383600A7986
:100B200043EA026383604B7903738B79C381CA798B
:100B300043EA0223027BC38102F00F020831103026
:100B400002F064F8237B002203F00F0384F82020D6
:100B500084F82820227903F10800111A04290DDDF8
:100B600021680933043AD21A085C84F82000D2B212
:100B7000606A84F82820194402F048F82379226832
:100B80001A44002012F8043CE36212F8031C43EA02
:100B90000123E36212F8021C43EA0143E36212F804
:100BA000012C43EA0263E36210BD0220FCE710B5AA
:100BB000044660B3036853B30279162A29D94279EF
:100BC0001A700146082251F8060B013002F028F88D
:100BD0002146082251F80E0B093002F021F8236853
:100BE000E28A5A74E38A22681B0A93742368A26912
:100BF000DA74A36922681B0A13752368628B5A751D
:100C00002368E27E9A7517232371002010BD01200E
:100C1000FCE70220FAE738B50446002863D00168F3
:100C2000002960D0037B90F8282003F00F03002AEE
:100C300057D10833207904321344984255D363794D
:100C40000B702368A2685A70A36822681B0A93700D
:100C500023686289DA702368E27A1A712368227B3A
:100C60005A712368E2899A71E38922681B0A214636
:100C7000D371227B51F8100B02F00F02083001F003
:100C8000C5FF237B94F8282003F00F0303F1080528
:100C90002AB1226894F82010515503F10905206803
:100CA00094F82820616A284401F0B0FF94F82830B5
:100CB0002268E16A2B44D1545A1CE16A206892B23E
:100CC000090A81549A1C2168E08D92B28854DA1C7A
:100CD000216894F82F0092B20433885423710020C5
:100CE00038BD0933A6E70120FAE70220F8E7000043
:100CF000024B1A8810431880704700BF50350020FF
:100D000008B5074B1B883BB1FEF7ACF8002814BFB1
:100D10006FF00200002008BD6FF00100FBE700BF8C
:100D20005035002010B5034B00241C80FEF790F8CE
:100D3000204610BD50350020B0FA80F040097047C1
:100D400082B018B9084602B000F0CAB8002002B05C
:100D5000704710B9084600F079B9704710B90846D5
:100D600000F090B970470346084611460BB900F0F1
:100D7000DDB90020704710B9084600F039BD704752
:100D800010B9084600F0FEB90020704710B40446C0
:100D9000084611461A46019B14B910BC00F00CBA63
:100DA00010BC70470346084611460BB900F036BA2E
:100DB0000020704710B40446084611461A4614B97C
:100DC00010BC00F0A3BA002010BC704730B4054638
:100DD000084611461A46DDE902341DB9029430BCBA
:100DE00000F022BB002030BC704710B9084600F06C
:100DF000D3BB0020704710B9084600F037BD002073
:100E0000704710B9084600F0E2BB0020704710B9E7
:100E1000084600F0DFBB0020704703460846114635
:100E20000BB900F0F9BB0020704710B40446084627
:100E300011461A46019B14B910BC00F0EFBB092003
:100E400010BC704710B40446084611461A4614B93F
:100E500010BC00F02DBDC8B210BC704700487047F0
:100E600001000102064B10B51B6A0446984730B1D9
:100E70000448054B204498428CBF0020012010BD3F
:100E8000646B0308403576C9405DC600F0B5114B70
:100E900085B00C4610491F56054601F017F80F4B58
:100EA000E4B25E6A072D4FF00103CDE9024301462B
:100EB0000AD105220023CDE900234FF47A727A4348
:100EC0001846B04705B0F0BD08220020CDE900204B
:100ED0003A46F5E74C6503082C650308646B030884
:100EE0001FB5002300930378013B372B21D8DFE89F
:100EF00003F01C242020201E202020204143454EAA
:100F00002055585B5E6164206C1E6E73787A7D207C
:100F10007F83262020202020202020202020202009
:100F200085878C2020858C208E92C3780BB102237C
:100F30000093009805B05DF804FB8378F6E74378EA
:100F40008DF8043007238DF805308378003B18BFF7
:100F500001235B008DF8063010238DF80730314BEC
:100F60001B6801A803F55872CDE9022300F08EFF3B
:100F70000090DEE74023DBE72023D9E7827890F971
:100F8000013012B9284AD35CD2E7284AFBE78278BD
:100F900090F90130002AF8D1254AF4E740F6B83339
:100FA000C6E74FF47A73C3E74FF4FA63C0E741F240
:100FB0008833BDE741F27073BAE71E484FF47A7187
:100FC00001F008FE00F5FA60D2E71B4BB0E7154BC5
:100FD0001B6803F55873ABE7124B1B6803F55B7393
:100FE000A6E71023A4E70F4B1B68A1E701239FE7A7
:100FF0004FF0834300939CE7104BFBE7104B97E7C0
:1010000040F21113ADF8003093E7032390E790F915
:1010100001300C4AB7E70C4990F9010000F056FF87
:10102000A6E700BF583500202365030813650308B1
:101030001B65030818FCFFFF00EA06379A99094070
:1010400040F709374C6503082C65030837B50B4B8F
:1010500002781B680C2101FB02335B7A03EB43042B
:10106000074B1D6803690093C3684278816805EBEC
:10107000C40000F0A7FC03B030BD00BF583500200D
:101080005435002030B587B0027B6423ADF80030C2
:10109000012A4FF00003CDE90133CDE903338DF888
:1010A00002308DF8143028D0022A2FD01ABB0368E2
:1010B0000BB34368FBB11A4C80682360194B1822AC
:1010C0006946186001F0A2FD174B246893E80700F9
:1010D0000C3384E8070093E8070004F10C050323B0
:1010E00085E80700A4F86C33012204F55B7104F570
:1010F000587000F058FC07B030BD094908684360DB
:10110000036100F55B7100F55870F2E7044B1B6852
:10111000B3F86023B3F86C130A43A3F86023EAE73B
:1011200058350020543500204020030808B50346F8
:101130000A2924D8DFE801F006232323230B161BFA
:1011400023212100BDE808400068FFF78BBE90F91D
:1011500000009978072271B900F0E5FB003818BF4C
:10116000012008BD052293F900000021F4E790F961
:1011700000005978EEE70221EEE70722F3E70020AE
:10118000EFE7000008B502791AB1012A0BD0002060
:1011900008BD084B01681B68012203F5587000F078
:1011A00002FC0120F4E7034B01681B6803F55B7048
:1011B000F5E700BF58350020F7B50728144D1C4649
:1011C000A8BF072058700E462946174600F07EFE3D
:1011D00094F90130A070072B13D1322000F076FD76
:1011E0000C4BDB6D0546984704F10C0208340346AE
:1011F000019200943A463146284600F06CFD03B057
:10120000F0BD054A55F82310D05C00F057FDE7E724
:101210002C650308646B03084C6503082DE9F04F47
:10122000344F90F901607B68D0F804908BB004468D
:10123000884698470546002859D1E37C73B92E4A61
:101240002378126803EB4303990002EB8303D3F87E
:101250000490B9F1000F01D152F80190274B484694
:1012600013F906B0FB689847A37C2289D7F818A029
:101270000993072E28D100230121CDE90223204A1A
:101280000693CDE90431CDE907330521CDE90021ED
:101290004FF47A7202FB0BF24CF250311846D047F1
:1012A000637C13B3174B995D7B6D0D31C9B2284632
:1012B0009847E07C3246494600F01AFE88F8006004
:1012C00001200BB0BDE8F08F002101250823CDE9F6
:1012D0000013CDE90715CDE90511CDE903110292FF
:1012E000A1782B465A462846D9E7074BDBE7002072
:1012F000E7E700BF646B0308583500204C6503081E
:10130000854501001B650308236503082DE9F04F9F
:101310008DB090F90130DFF8FCA0DFF8FC90CDE94A
:101320000A123E4A12F903B00278DAF800300C25AE
:1013300005FB02333A4A5B7A126803EB430302EB84
:10134000C303044693F9021090F9020000F0B9FDBE
:101350003449064694F9010000F0B8FDA2686168BE
:101360008046304600F0DFFC2178DAF80020D9F81A
:101370000C306943074650589847D9F81C309C46B2
:1013800094F901300025072B4FF47A63CDE9075318
:10139000CDE905552DD10123CDE903530523CDE931
:1013A00001534FF47A7303FB0BF300933946434622
:1013B00046F2A81228466746B8472378DAF8002094
:1013C0000C214B4394F90110D05800F0B3FDA189D2
:1013D00094F90100FFF75AFD0B9B217B1860D9F8A7
:1013E0005430284698470A9B01201E700DB0BDE876
:1013F000F08F01200823CDE90350CDE901032A46EF
:10140000CDF800B0654643463946A8470120054659
:10141000D3E700BF58350020646B03084C65030810
:10142000543500202C6503082DE9F04F8FB00024BF
:1014300005468A46914698460494ADF81440ADF8A6
:10144000024007264FF0010B2B7AA34206D96868A9
:1014500004A9204400F0CAFB00285DD102238DF8C6
:10146000083002A86B7A8DF80A30FFF739FDAB7AA5
:101470008DF81D309DF811308DF81E309DF812301A
:101480008DF81F309DF810308DF82030EB7A8DF8F4
:1014900021302B7B8DF822306B7B8DF8233010238D
:1014A0008DF81C608DF824303A4E8DF82C000DF12B
:1014B00002030A93072332688DF82D30ADF83430DB
:1014C0002B680C9206930DF1120204AB0DF1110181
:1014D00006A800F0A5FB072805460BD130680C22B2
:1014E000002100F5587001F0A5FB3368BDF802201B
:1014F000A3F860239DF811308AF800309DF812306F
:1015000089F800309DF8103088F80030189B284684
:101510001C700FB0BDE8F08F9DF81330BDF814704B
:10152000ADF802702044C4B2F3B917B3194A0020D1
:101530001168072602464FF00C0C062B1BD10CFB42
:1015400000FE51F80EE0BEF1000F04D00BFA00F2DD
:101550003A4397B2012201301028EED1002A3FF41D
:1015600073AFADF802706FE75A1E042A01D9062B3B
:10157000DCD0062668E747FA00FE1EF0010FEAD02D
:101580000CFB00FE51F80EE0BEF1000F08BF06266E
:10159000E1E700BF5835002038B505464068FFF741
:1015A00061FC0722841D002195F90000E4B200F0DF
:1015B000BAF908B904F0FD0495F9010007220021E9
:1015C00000F0B1F908B904F0FB04204638BD002052
:1015D0007047000010B503780F2B044618D84068F8
:1015E000FFF740FC22780B4902EB42020968831C9A
:1015F00001EB820051F82220DBB21AB903F0FD039F
:1016000058B210BD032B06BF626842600223F7E7A1
:101610000020F6E758350020022070472DE9F04100
:101620003A4D0446286896B00E46904600211F4663
:101630000122032300F55870CDE90411CDE906110C
:101640008DF80C108DF80D10ADF80E3000F08DF9FE
:1016500030B92A68B2F8603343F00303A2F860336C
:101660002A68637A8DF8203002F55871CDE90912A5
:10167000274A94F9083012680B921022ADF83020F6
:101680000DF10E020D9222680E9262680F92D4E95B
:101690000301A27A8DF8402001228DF8412011AA81
:1016A00082E80300227DE18A8DF8213018468DF80A
:1016B0004C20FFF7EBFB08AB15930DF10D031490D5
:1016C0000093CDF8048003AB04AA39460EA800F0BD
:1016D00099FB044678B99DF80C10013901F07AFAAB
:1016E00000F158030DEB030010F8483C337020461E
:1016F00016B0BDE8F0810C2801BF2A68B2F860334B
:1017000043F00303A2F86033F1E700BF583500202F
:1017100054350020F8B50679012E054648D90F2E1C
:1017200048D80368187A40F303000722002140B22A
:1017300000F0F9F82B680446187A40F303100722EA
:10174000002140B200F0EFF8B8B1B4FA84F46409B3
:1017500029680B7A086843F3030243F303135BB26F
:1017600052B29A42C8BF0124FFF77CFB80F001030C
:10177000DBB224B10533D8B2F8BD0124E8E7DBB908
:101780000E4F29683B6806EB460003EB80000C22F5
:1017900001F03CFA3A680C2303FB062320465C72F6
:1017A000B2F860130123B3400B43A2F86033E3E7C0
:1017B0000620E1E70320DFE70420DDE758350020BD
:1017C00010B4017801290ED9084B18680C234B433B
:1017D000C4180022C250C4E9012200F5587010BCA0
:1017E000102200F0A9B8002010BC70475835002026
:1017F0002DE9F04186B050238DF81430037A102B78
:10180000074630D14368DD7B6DBB0224A8466426C1
:10181000062C14D87A68535D03932A44517843EA1E
:1018200001230393927843EA02437343CDE90338DB
:1018300063B968468DF80040FFF7C2FF0DE0CDF8B0
:101840000C808DF81480CDF81080F2E703AB01A86E
:1018500001938DF80840FFF75DFF0134E4B2102CCE
:1018600005F10305D4D106B0BDE8F0811FB50268CB
:101870000379116849B901A88DF80430FFF7A0FF7A
:1018800078B1032005B05DF804FB02A802928DF840
:101890000C30FFF73FFF042805D0052805D00028AD
:1018A000EFD00020EEE70220ECE70120EAE700009D
:1018B000C90020B9034B0B449856C0B27047024B85
:1018C000F9E700BFD364030893640308F0B59A42B4
:1018D000069D03DB9DF914309A4220DD0020F0BD07
:1018E00003EB430331F814C005EB830300264CFAE5
:1018F00006F7FF0707D51F7A07F00F0E964502DCA3
:10190000B2EB171F0DDD0136102E03F10C03EED1E3
:101910000134E4B22301DBB29842E1D8DEE70024CF
:10192000F8E70120DBE7884204DB9042CCBF0020CF
:10193000012070470020704710B51409B4EB111F47
:1019400003464FEA11100ED391420CD202B201F0BD
:101950000F0133F81240012000FA01F124EA0101DD
:1019600023F8121010BD0020FCE7F0B528B100EB01
:10197000410501270020914200D3F0BD002435F835
:1019800002CB234607FA04F636EA0C0608BF0133F9
:1019900004F1010408BFDBB2102CF3D1184401316B
:1019A000C0B2C9B2E7E710B500B149B910BD31F80E
:1019B000134020F813400133DCB2A242F7D8F5E718
:1019C0000023F9E782B030B504880493D2B9B3F5A7
:1019D000616F15D349F6AF2542F21072AB4298BF42
:1019E0004FF47A72944238BF14466143BDE83040E8
:1019F000C3688B428CBF5B1A0023C36002B0704780
:101A00006422EFE7012C38BF0124EEE72DE9F04F07
:101A10008FB01546199F03939DF8603007930C46CD
:101A2000804603F089FC6A4A0590A7F5F633303BFF
:101A3000B3FBF2F3534303F5F63B0493182313FB74
:101A400005430BF1300B069300254FF0FF3A069B40
:101A50009C4207D1002D14BF50464FF0FF300FB00D
:101A6000BDE8F08FBDF96830ADF8243009991997B9
:101A70003846089703F05CFB2688B8F1000F5FD169
:101A8000B7F5616F5AD349F6AF2242F2107397420D
:101A900098BF4FF47A739E4238BF1E46642E59D1C8
:101AA000DFF83091A060A1680CA803F063FB0D9BE8
:101AB0000093DDE908120C9B0AA803F0B9FA039A17
:101AC0000A9B0AB9079A2AB122694A4502D1424AB9
:101AD00093420ED9414BC4F80C909F4209D9002380
:101AE000ADF82C300B99CDF828B0584603F020FB08
:101AF000A060606808B9C4F80C90C4F81090B8F100
:101B0000000F04D003F022FCE3680344E360D4E94F
:101B100003329342059B88BFE26063601B9BE168D0
:101B20007343994204D20398E8B9B8F1000F1AD070
:101B300001231D442375EDB2183488E76423AAE716
:101B4000039B0BB9234BE360012EDFF8889038BF6D
:101B50000126CEE7B6F57A7F0ABFDFF88490DFF87A
:101B60008490A0609FE700209342207506D85B1AFE
:101B70009A4505F1010528BF9A46EDB2B8F1000F6C
:101B8000DAD1642E184AADF82C801DD049F6B02366
:101B9000B6F57A7F18BF1346974281BF049A02F5C3
:101BA000A83202F5C0729B180A931A9B00930AAEE2
:101BB00096E80600199B304603F03AFA96E80300CF
:101BC00003F0B6FA8246B7E74FF46163E4E700BF7B
:101BD0008051010040771B007F5101002FEC010074
:101BE00080A81201002E930230EC01000378032B31
:101BF00014D1437803F00F021B098A704B7083786D
:101C00008B80C27843EA02238B800379C3F30212EC
